:040000037000CE8932
:020000040000FA
:1000000000040020810A000015070000610A0000BA
:100010001F07000029070000330700000000000050
:10002000000000000000000000000000A50A000021
:100030003D070000000000004707000051070000D6
:100040005B070000650700006F07000079070000EC
:10005000830700008D07000097070000A10700003C
:10006000AB070000B5070000BF070000C90700008C
:10007000D3070000DD070000E7070000F1070000DC
:10008000FB070000050800000F0800001908000029
:10009000230800002D080000370800004108000078
:1000A0004B080000550800005F08000069080000C8
:1000B000730800007D080000870800009108000018
:1000C0009B080000A5080000AF080000B908000068
:1000D000C3080000CD080000D7080000E1080000B8
:1000E000EB080000F5080000FF0800000909000007
:1000F000130900001D090000270900003109000054
:100100003B0900001FB500F003F88DE80F001FBD8C
:1001100000F0ACBC40F6FC7108684FF01022401CA7
:1001200008D00868401C09D00868401C04D0086842
:1001300000F037BA9069F5E79069F9E7704770B554
:100140000B46010B184400F6FF70040B4FF0805073
:100150000022090303692403406943431D1B104621
:1001600000F048FA29462046BDE8704000F042BA47
:10017000F0B54FF6FF734FF4B4751A466E1E11E0DA
:10018000A94201D3344600E00C46091B30F8027B3B
:10019000641E3B441A44F9D19CB204EB134394B25D
:1001A00004EB12420029EBD198B200EB134002EBB2
:1001B000124140EA0140F0BDF34992B00446D1E952
:1001C0000001CDE91001FF224021684600F0F4FB58
:1001D00094E80F008DE80F00684610A902E004C8FB
:1001E00041F8042D8842FAD110216846FFF7C0FF7C
:1001F0001090AA208DF8440000F099F9FFF78AFFCB
:1002000040F6FC7420684FF01025401C0FD0206889
:1002100010226946803000F078F92068401C08D030
:100220002068082210A900F070F900F061F9A869AF
:10023000EEE7A869F5E74FF080500369406940F6A2
:10024000FC71434308684FF01022401C06D0086838
:1002500000F58050834203D2092070479069F7E788
:100260000868401C04D00868401C03D00020704778
:100270009069F9E70420704770B504460068C34DE3
:10028000072876D2DFE800F033041929631E250021
:10029000D4E9026564682946304600F062F92A46CE
:1002A0002146304600F031F9AA002146304600F0E0
:1002B00057FB002800D0032070BD00F009FC4FF46C
:1002C000805007E0201D00F040F90028F4D100F034
:1002D000FFFB60682860002070BD241D94E80700C3
:1002E000920000F03DFB0028F6D00E2070BDFFF715
:1002F000A2FF0028FAD1D4E901034FF0805100EBAE
:10030000830208694D69684382420ED840F6F8704E
:1003100005684FF010226D1C09D0056805EB8305B8
:100320000B6949694B439D4203D9092070BD55694A
:10033000F4E70168491C03D00068401C02D003E0C8
:100340005069FAE70F2070BD2046FFF735FFFFF731
:1003500072FF0028F7D1201D00F0F7F80028F2D135
:1003600060680028F0D100F0E2F8FFF7D3FE00F05B
:10037000BFF8072070BD10B50C46182802D0012028
:10038000086010BD2068FFF777FF206010BD41684E
:10039000054609B1012700E0002740F6F8742068FF
:1003A0004FF01026401C2BD02068AA68920000F065
:1003B000D7FA38B3A86881002068401C27D020688D
:1003C000FFF7BDFED7B12068401C22D026684FF051
:1003D0008050AC686D68016942695143A9420DD9EA
:1003E000016940694143A14208D92146304600F0E5
:1003F000B8F822462946304600F087F800F078F831
:100400007069D2E700F093F8FFF784FEF6E77069B1
:10041000D6E77669DBE740F6FC7420684FF01026DB
:10042000401C23D02068401C0CD02068401C1FD0EA
:100430002568206805F18005401C1BD027683879A5
:10044000AA2819D040F6F8700168491C42D001680A
:10045000491C45D00168491C3ED001680968491C07
:100460003ED00168491C39D000683EE0B069DAE747
:10047000B569DEE7B769E2E710212846FFF778FEA5
:100480003968814222D12068401C05D0D4F8001080
:1004900001F18002C03107E0B169F9E730B108CA63
:1004A00051F8040D984201D1012000E000208A4259
:1004B000F4D158B1286810B1042803D0FEE72846CB
:1004C000FFF765FF3149686808600EE0FFF722FE1C
:1004D00000F00EF87169BBE77169BFE7706904E06D
:1004E0004FF480500168491C01D000F0CBFAFEE7C0
:1004F000BFF34F8F26480168264A01F4E06111439B
:100500000160BFF34F8F00BFFDE72DE9F0411746B3
:100510000D460646002406E03046296800F054F8EF
:10052000641C2D1D361DBC42F6D3BDE8F08140F69B
:10053000FC700168491C04D0D0F800004FF48051D1
:10054000FDE54FF010208069F8E74FF080510A690F
:10055000496900684A43824201D810207047002050
:10056000704770B50C4605464FF4806608E0284693
:1005700000F017F8B44205D3A4F5806405F5805562
:10058000002CF4D170BD0000F40A0000000000202F
:100590000CED00E00400FA05144801680029FCD0C5
:1005A0007047134A0221116010490B68002BFCD0E0
:1005B0000F4B1B1D186008680028FCD0002010603D
:1005C00008680028FCD07047094B10B501221A605A
:1005D000064A1468002CFCD0016010680028FCD08A
:1005E0000020186010680028FCD010BD00E4014015
:1005F00004E5014070B50C46054600F073F810B9EB
:1006000000F07EF828B121462846BDE8704000F091
:1006100007B821462846BDE8704000F037B8000012
:100620007FB5002200920192029203920A0B000B06
:100630006946012302440AE0440900F01F0651F80C
:10064000245003FA06F6354341F82450401C8242F8
:10065000F2D80D490868009A10430860081D016827
:10066000019A1143016000F03DF800280AD00649C4
:1006700010310868029A10430860091D0868039A3F
:10068000104308607FBD00000006004030B50F4CED
:10069000002200BF04EB0213D3F800582DB9D3F8A1
:1006A000045815B9D3F808581DB1521C082AF1D3C3
:1006B00030BD082AFCD204EB0212C2F80008C3F8CD
:1006C00004180220C3F8080830BD000000E0014013
:1006D0004FF08050D0F83001082801D0002070473A
:1006E000012070474FF08050D0F83011062905D016
:1006F000D0F83001401C01D0002070470120704725
:100700004FF08050D0F830010A2801D00020704707
:100710000120704708208F490968095808471020B0
:100720008C4909680958084714208A4909680958FA
:100730000847182087490968095808473020854923
:100740000968095808473820824909680958084744
:100750003C20804909680958084740207D490968BC
:100760000958084744207B49096809580847482028
:1007700078490968095808474C207649096809589A
:10078000084750207349096809580847542071499F
:1007900009680958084758206E49096809580847E8
:1007A0005C206C4909680958084760206949096854
:1007B00009580847642067490968095808476820AC
:1007C00064490968095808476C2062490968095852
:1007D000084770205F4909680958084774205D4937
:1007E00009680958084778205A490968095808478C
:1007F0007C205849096809580847802055490968EC
:10080000095808478420534909680958084788202F
:1008100050490968095808478C204E490968095809
:10082000084790204B4909680958084794204949CE
:10083000096809580847982046490968095808472F
:100840009C204449096809580847A0204149096883
:1008500009580847A4203F49096809580847A820B3
:100860003C49096809580847AC203A4909680958C1
:100870000847B0203749096809580847B420354966
:10088000096809580847B8203249096809580847D3
:10089000BC203049096809580847C0202D4909681B
:1008A00009580847C4202B49096809580847C82037
:1008B0002849096809580847CC2026490968095879
:1008C0000847D0202349096809580847D4202149FE
:1008D000096809580847D8201E4909680958084777
:1008E000DC201C49096809580847E02019490968B3
:1008F00009580847E4201749096809580847E820BB
:100900001449096809580847EC2012490968095830
:100910000847F0200F49096809580847F4200D4995
:10092000096809580847F8200A490968095808471A
:10093000FC2008490968095808475FF48070054998
:10094000096809580847000003480449024A034B54
:100950007047000000000020000B0000000B0000AA
:1009600040EA010310B59B070FD1042A0DD310C82C
:1009700008C9121F9C42F8D020BA19BA884201D97E
:10098000012010BD4FF0FF3010BD1AB1D30703D0C6
:10099000521C07E0002010BD10F8013B11F8014B7C
:1009A0001B1B07D110F8013B11F8014B1B1B01D198
:1009B000921EF1D1184610BD02F0FF0343EA032254
:1009C00042EA024200F005B87047704770474FF0A6
:1009D00000020429C0F0128010F0030C00F01B800C
:1009E000CCF1040CBCF1020F18BF00F8012BA8BF1A
:1009F00020F8022BA1EB0C0100F00DB85FEAC17CDE
:100A000024BF00F8012B00F8012B48BF00F8012B90
:100A100070474FF0000200B51346944696462039C1
:100A200022BFA0E80C50A0E80C50B1F12001BFF4A7
:100A3000F7AF090728BFA0E80C5048BF0CC05DF80D
:100A400004EB890028BF40F8042B08BF704748BF5B
:100A500020F8022B11F0804F18BF00F8012B7047CF
:100A6000014B1B68DB6818470000002009480A4951
:100A70007047FFF7FBFFFFF745FB00BD20BFFDE719
:100A8000064B1847064A1060016881F308884068E1
:100A900000470000000B0000000B000017040000DE
:100AA000000000201EF0040F0CBFEFF30881EFF3ED
:100AB0000981886902380078182803D100E0000015
:100AC000074A1047074A12682C3212681047000084
:100AD00000B5054B1B68054A9B58984700BD0000B0
:100AE0007703000000000020F00A0000040000006E
:100AF000001000000000000000FFFFFF0090D00386
:1010000080130020194B020005C000007F4A020037
:1010100005C0000005C0000005C000000000000081
:10102000000000000000000000000000754B0200FE
:1010300005C000000000000005C0000005C0000061
:10104000DD4B0200E34B020005C0000005C00000BC
:1010500005C0000005C0000005C0000005C000007C
:10106000E94B020005C0000005C00000EF4B020084
:1010700005C00000F54B0200FB4B0200014C0200D2
:1010800005C0000005C0000005C0000005C000004C
:1010900005C0000005C0000005C0000005C000003C
:1010A00005C00000074C020005C0000005C000009C
:1010B00005C0000005C0000005C0000005C000001C
:1010C0000D4C020005C0000005C0000005C0000076
:1010D00005C0000005C0000005C0000005C00000FC
:1010E00005C0000005C0000005C0000005C00000EC
:1010F00005C0000005C0000005C0000005C00000DC
:1011000005C0000005C0000000F002F823F0F3FC69
:101110000AA090E8000C82448344AAF10107DA4552
:1011200001D123F0E8FCAFF2090EBAE80F0013F08A
:10113000010F18BFFB1A43F001031847C03F02001C
:10114000E03F02000A444FF0000C10F8013B13F09E
:10115000070408BF10F8014B1D1108BF10F8015B10
:10116000641E05D010F8016B641E01F8016BF9D103
:1011700013F0080F1EBF10F8014BAD1C0C1B09D15A
:101180006D1E58BF01F801CBFAD505E014F8016BCC
:1011900001F8016B6D1EF9D59142D6D3704700005E
:1011A0000023002400250026103A28BF78C1FBD870
:1011B000520728BF30C148BF0B6070471FB500F011
:1011C0003DF88DE80F001FBD1EF0040F0CBFEFF3BC
:1011D0000880EFF30980014A1047000047BF000074
:1011E000F0B44046494652465B460FB402A0013077
:1011F00001B50648004700BF01BC86460FBC8046CB
:10120000894692469B46F0BC7047000009110000D9
:101210008269034981614FF001001044704700006A
:101220002512000001B41EB400B514F047FD01B44E
:101230000198864601BC01B01EBD000023F058BCD9
:1012400070B51A4C054609202070A01C00F0D1F89A
:101250005920A08029462046BDE8704008F0C4B857
:1012600008F0CDB870B50C461149097829B1A0F144
:1012700060015E2908D3012013E0602804D06928AA
:1012800002D043F201000CE020CC0A4E94E80E009C
:1012900006EB8000A0F58050241FD0F8806E284611
:1012A000B047206070BD012070470000080000209A
:1012B00018000020584C02003249884201D2012017
:1012C00070470020704770B50446A0F500002E4E10
:1012D000B0F1786F02D23444A4F500042948844266
:1012E00001D2012500E0002500F043F848B125B9FE
:1012F000B44204D32548006808E0012070BD0020F6
:1013000070BD002DF9D1B442F9D321488442F6D200
:10131000F3E710B50446A0F50000B0F1786F03D2F2
:1013200019480444A4F5000400F023F84FF080416C
:1013300030B11648006804E08C4204D2012003E07A
:1013400013488442F8D2002080F0010010BD10B58F
:1013500020B1FFF7DEFF08B1012010BD002010BD55
:1013600010B520B1FFF7AFFF08B1012010BD00207C
:1013700010BD084808490068884201D10120704723
:101380000020704700600200000000201C000020C8
:101390000800002054000020BEBAFECA10B5044662
:1013A0000021012000F03DF800210B2000F039F869
:1013B0000421192000F035F804210D2000F031F847
:1013C00004210E2000F02DF804210F2000F029F850
:1013D0000421C84300F025F80621162000F021F86A
:1013E0000621152000F01DF82046FFF729FF0020F8
:1013F00010BDB72101807047FFF732BF1148704719
:1014000010487047104A10B514680F4B0F4A083344
:101410001A60FFF727FF0C48001D046010BD7047DD
:1014200070474907090E002804DB00F1E02080F82E
:101430000014704700F00F0000F1E02080F8141D48
:101440007047000003F9004210050240010000014E
:10145000FE48002101604160018170472DE9F7439A
:10146000044692B091464068FFF771FF40B1606852
:10147000FFF776FF20B9607800F00300022801D062
:10148000012000E00020F14E30724846FFF71BFFBC
:1014900018B1102015B0BDE8F0834946012001F0D5
:1014A0008EFE0028F6D101258DF842504FF4C05031
:1014B000ADF84000002210A9284606F0FFFB0028E6
:1014C000E8D18DF842504FF428504FF00008ADF8A5
:1014D000400047461C216846CDF81C8023F0A3FA43
:1014E0009DF81C0008AA20F00F00401C20F0F0001E
:1014F00010308DF81C0020788DF81D0061789DF863
:101500001E0061F3420040F001008DF81E009DF8BE
:1015100000000AA940F002008DF800002089ADF813
:101520003000ADF83270608907AFADF834000B972A
:10153000606810AC0E900A94684606F0B2F9002874
:10154000A8D1BDF8200030808DF8425042F601202D
:10155000ADF840009DF81E0008AA20F00600801C8F
:1015600020F001008DF81E000220ADF83000ADF82B
:10157000340013A80E900AA9684606F092F90028D4
:1015800088D1BDF820007080311D484600F033F945
:10159000002887D18DF8425042F6A620ADF84000D1
:1015A0001C216846CDF81C8023F03DFA9DF81C00F4
:1015B000ADF8345020F00F00401C20F0F000103047
:1015C0008DF81C009DF81D0008AA20F0FF008DF882
:1015D0001D009DF81E000AA920F0060040F0010041
:1015E000801C8DF81E009DF800008DF8445040F0DE
:1015F00002008DF80000CDE90A4711A80E90ADF861
:101600003050684606F04DF9002899D1BDF8200009
:10161000F08000203EE73EB504460820ADF800000B
:101620002046FFF750FE08B110203EBD21460120A4
:1016300001F0C5FD0028F8D12088ADF804006088CD
:10164000ADF80600A088ADF80800E088ADF80A0003
:101650007E4801AB6A468088002106F02BFDBDF86C
:1016600000100829E1D003203EBD1FB5044600202C
:1016700002900820ADF80800CDF80CD02046FFF706
:1016800022FE10B1102004B010BD704802AA81885B
:101690004FF6FF7006F050FF0028F4D1BDF8081097
:1016A000082901D00320EEE7BDF800102180BDF825
:1016B00002106180BDF80410A180BDF80610E18021
:1016C000E1E701B582B00220ADF800005F4802AB4F
:1016D0006A464088002106F0EDFCBDF800100229A2
:1016E00000D003200EBD1CB5002100910221ADF8F1
:1016F00000100190FFF70DFE08B110201CBD5348EB
:101700006A4641884FF6FF7006F016FFBDF80010DC
:101710000229F3D003201CBDFEB54C4C06461546ED
:10172000207A0F46C00705D00846FFF7CCFD18B158
:101730001020FEBD0F20FEBDF82D01D90C20FEBDEE
:101740003046FFF7C0FD18BB208801A905F0AEFDAB
:101750000028F4D130788DF80500208801A906F022
:1017600087FC0028EBD100909DF800009DF8051043
:1017700040F002008DF80000090703D040F0080097
:101780008DF800002088694606F00FFC0028D6D1AD
:10179000ADF8085020883B4602AA002106F08AFCDA
:1017A000BDF80810A942CAD00320FEBD7CB505468D
:1017B0000020009001900888ADF800000C462846F3
:1017C0000195FFF7C4FD18B92046FFF7A2FD08B147
:1017D00010207CBD15B1BDF8000050B11B486A4611
:1017E00001884FF6FF7006F0A7FEBDF800102180BB
:1017F0007CBD0C207CBD30B593B0044600200D4666
:101800000090142101A823F00EF91C2108A823F050
:101810000AF99DF80000CDF808D020F00F00401C18
:1018200020F0F00010308DF800009DF8010020F04D
:10183000FF008DF801009DF8200040F002008DF8B7
:10184000200001208DF8460002E000002002002068
:1018500042F60420ADF8440011A801902088ADF8AC
:101860003C006088ADF83E00A088ADF84000E088FC
:10187000ADF842009DF8020006AA20F00600801C88
:1018800020F001008DF802000820ADF80C00ADF842
:1018900010000FA8059001A908A806F002F800287A
:1018A00003D1BDF818002880002013B030BD00001F
:1018B000F0B5007B059F1E4614460D46012800D05A
:1018C000FFDF0C2030803A203880002C08D0287AA6
:1018D000032806D0287B012800D0FFDF1720608175
:1018E000F0BDA889FBE72DE9F04786B0144691F8D2
:1018F0000C900E9A0D46B9F1010F0BD01021007B10
:101900002E8A8846052807D0062833D0FFDF06B088
:10191000BDE8F0870221F2E7E8890C2100EB4000E6
:1019200001EB4000188033201080002CEFD0E889B4
:10193000608100271AE00096688808F1020301AA76
:10194000696900F084FF06EB0800801C07EB470183
:1019500086B204EB4102BDF8040090810DF106014E
:1019600040460E3212F04FFC7F1CBFB26089B84275
:10197000E1D8CCE734201080E889B9F1010F11D00B
:10198000122148430E301880002CC0D0E8896081B5
:101990004846B9F1010F00D00220207300270DF155
:1019A000040A1FE00621ECE70096688808F10203AC
:1019B00001AA696900F04BFF06EB0800801C86B2A3
:1019C000B9F1010F12D007EBC70004EB4000BDF8DE
:1019D0000410C18110220AF10201103022F082FFAE
:1019E0007F1CBFB26089B842DED890E707EB4701A1
:1019F00004EB4102BDF80400D0810AF10201404627
:101A0000103212F000FCEBE72DE9F0470E4688B0EB
:101A100090F80CC096F80C80378AF5890C20109944
:101A200002F10C044FF0000ABCF1030F08D0BCF126
:101A3000040F3ED0BCF1070F7DD0FFDF08B067E791
:101A400005EB850C00EB4C00188031200880002A43
:101A5000F4D0A8F1060000F0FF09558125E0182117
:101A600001A822F0E0FF00977088434601AA71693F
:101A700000F0EDFEBDF804002080BDF80600E08017
:101A8000BDF808002081A21C0DF10A01484612F0A1
:101A9000BAFBB9F1000F00D018B184F804A0A4F883
:101AA00002A007EB080087B20A346D1EADB2D6D291
:101AB000C4E705EB850C00EB4C0018803220088051
:101AC000002ABBD0A8F1050000F0FF09558137E0DE
:101AD00000977088434601AA716900F0B8FE9DF82E
:101AE0000600BDF80410E1802179420860F300018E
:101AF00062F34101820862F38201C20862F3C3010A
:101B0000020962F30411420962F34511820962F38A
:101B100086112171C0096071BDF80700208122463D
:101B20000DF10901484612F06EFB18B184F802A0CD
:101B3000A4F800A000E007E007EB080087B20A3431
:101B40006D1EADB2C4D279E7A8F1020084B205FBE4
:101B500008F000F10E0CA3F800C035230B80002A1A
:101B6000A6D055819481009783B270880E32716936
:101B700000F06DFE62E72DE9F84F1E460A9D0C4607
:101B800081462AB1607A00F58070D080E0891081AA
:101B900099F80C000C274FF000084FF00E0A0D28A2
:101BA00073D2DFE800F09E070E1C28303846556AD5
:101BB00073737300214648460095FFF779FEBDE830
:101BC000F88F207B9146082802D0032800D0FFDF41
:101BD000378030200AE000BFA9F80A80EFE7207BB9
:101BE0009146042800D0FFDF378031202880B9F1EA
:101BF000000FF1D1E3E7207B9146042800D0FFDFFE
:101C000037803220F2E7207B9146022800D0FFDFA8
:101C100037803320EAE7207B1746022800D0FFDF19
:101C20003420A6F800A02880002FC8D0A7F80A808A
:101C3000C5E7207B1746042800D0FFDF3520A6F833
:101C400000A02880002FBAD04046A7F80A8012E0F2
:101C5000207B1746052802D0062800D0FFDF102081
:101C6000308036202880002FA9D0E0897881A7F81D
:101C70000E80B9F80E00B881A1E7207B91460728B5
:101C800000D0FFDF37803720B0E72AE04FF01200A6
:101C900018804FF038001700288090D0E0897881B4
:101CA000A7F80E80A7F8108099F80C000A2805D034
:101CB0000B2809D00C280DD0FFDF80E7207B0A28F5
:101CC00000D0FFDF01200AE0207B0B2800D0FFDFDF
:101CD000042004E0207B0C2800D0FFDF05203873AF
:101CE0006DE7FFDF6BE770B50C46054601F0ABFB17
:101CF00020B10078222804D2082070BD43F20200EF
:101D000070BD0521284610F0F1FC206008B10020CC
:101D100070BD032070BD30B44880087820F00F00FB
:101D2000C01C20F0F000903001F8080B1DCA81E8BB
:101D30001D0030BC07F0D9BB2DE9FF4784B0002758
:101D40008246029707989046894612300AF0AAF90F
:101D5000401D20F00306079828B907A95046FFF751
:101D6000C2FF002854D1B9F1000F05D00798017BBC
:101D700019BB052504681BE098F80000092803D06A
:101D80000D2812D0FFDF46E0079903254868B0B35D
:101D9000497B42887143914239D98AB2B3B2011D5D
:101DA00010F017FB0446078002E0079C0425083466
:101DB0000CB1208810B1032D29D02CE00798012107
:101DC00012300AF0A1F9ADF80C00024602AB294628
:101DD000504608F0F0F9070001D1A01C02900798C6
:101DE0003A461230C8F80400A8F802A003A94046F9
:101DF000029B0AF096F9D8B10A2817D200E006E053
:101E0000DFE800F007091414100B0D14141213204E
:101E100014E6002012E6112010E608200EE643F238
:101E200003000BE6072009E60D2007E6032005E680
:101E3000BDF80C002346CDE900702A4650460799AC
:101E400000F015FD57B9032D08D10798B3B2417BB7
:101E5000406871438AB2011D10F0CFFAB9F1000F4A
:101E6000D7D0079981F80C90D3E72DE9FE4F914622
:101E70001A881C468A468046FAB102AB494608F0E9
:101E80009AF9050019D04046A61C278810F072FD6B
:101E90003246072629463B46009610F080F92088F6
:101EA0002346CDE900504A465146404600F0DFFC4B
:101EB000002020800120BDE8FE8F0020FBE710B548
:101EC00086B01C46AAB104238DF800301388ADF803
:101ED00008305288ADF80A208A788DF80E200988DB
:101EE000ADF80C1000236A462146FFF725FF06B027
:101EF00010BD1020FBE770B50D46052110F0F6FB74
:101F0000040000D1FFDF294604F11200BDE8704053
:101F10000AF0E3B82DE9F8430D468046002607F0A5
:101F2000E1FA04462878102878D2DFE800F0773B01
:101F30003453313112313131083131313131287975
:101F4000001FC0B2022801D0102810D114BBFFDF3F
:101F500035E004B9FFDF0521404610F0C7FB007BE8
:101F6000032806D004280BD0072828D0FFDF072637
:101F700055E02879801FC0B2022820D050B1F6E782
:101F80002879401FC0B2022819D0102817D0EEE7D8
:101F900004B9FFDF13E004B9FFDF287901280ED16F
:101FA000172137E00521404610F0A0FB070000D1C3
:101FB000FFDF07F1120140460AF06CF82CB12A4607
:101FC00021464046FFF7A7FE29E01321404602F0D4
:101FD000F1FC24E004B9FFDF0521404610F086FB48
:101FE000060000D1FFDF694606F112000AF05CF836
:101FF000060000D0FFDFA988172901D2172200E0D0
:102000000A46BDF80000824202D9014602E005E01E
:102010001729C5D3404600F03AFCD0E7FFDF304631
:10202000BDE8F883401D20F0030219B102FB01F066
:10203000001D00E000201044704713B5009848B11F
:102040000024684610F06FF9002C02D1F74A00997D
:1020500011601CBD01240020F4E72DE9F0470C4677
:1020600015462421204622F0DEFC05B9FFDFA878C2
:1020700060732888DFF8B4A3401D20F00301AF7817
:102080008946DAF8000010F06CF9060000D1FFDF95
:102090004FF000082660A6F8008077B109FB07F131
:1020A000091D0AD0DAF8000010F05BF9060000D133
:1020B000FFDF6660C6F8008001E0C4F8048029886C
:1020C00004F11200BDE8F04709F0D6BF2DE9F04752
:1020D000804601F112000D46814609F0E3FF401DE4
:1020E000D24F20F003026E7B14462968386810F046
:1020F00063F93EB104FB06F2121D03D0696838682B
:1021000010F05AF9052010F099FA0446052010F055
:102110009DFA201A012802D1386810F017F94946B3
:102120004046BDE8F04709F0BCBF70B50546052143
:1021300010F0DCFA040000D1FFDF04F112012846A0
:10214000BDE8704009F0A6BF2DE9F04F91B04FF007
:10215000000BADF834B0ADF804B047880C46054626
:1021600092460521384610F0C1FA060000D1FFDF83
:1021700024B1A780A4F806B0A4F808B029780922F1
:102180000B20B2EB111F7DD12A7A04F11001382700
:102190004FF00C084FF001090391102A73D2DFE8C9
:1021A00002F072F2F1F07F08D2888D9F3DDBF3EEF2
:1021B000B6B6307B022800D0FFDFA88908EBC0014B
:1021C000ADF804103021ADF83410002C25D060811A
:1021D000B5F80E9000271DE004EBC708317C88F8A5
:1021E0000E10F189A8F80C10CDF80090688804232F
:1021F00004AA296900F02BFBBDF81010A8F81010F4
:1022000009F10400BDF812107F1C1FFA80F9A8F82C
:102210001210BFB26089B842DED80DE1307B0228CF
:1022200000D0FFDFE98908EBC100ADF804003020E1
:10223000ADF83400287B0A90001FC0B20F90002C2C
:10224000EBD06181B5F81090002725E0CDF8009023
:102250006888696903AA0A9B00F0F9FA0A9804EBF6
:10226000C70848441FFA80F908F10C0204A90F9826
:1022700011F0C9FF18B188F80EB0A8F80CB0BDF87D
:102280000C1001E0D4E0CFE0A8F81010BDF80E105B
:102290007F1CA8F81210BFB26089B842D6D8CBE034
:1022A0000DA8009001AB224629463046FFF71BFBE4
:1022B000C2E0307B082805D0FFDF03E0307B082830
:1022C00000D0FFDFE8891030ADF804003620ADF80B
:1022D0003400002C3FD0A9896181F189A18127E0D8
:1022E000307B092800D0FFDFA88900F10C01ADF890
:1022F00004103721ADF83410002C2CD06081E8890F
:102300000090AB89688804F10C02296956E0E889DD
:102310003921103080B2ADF80400ADF83410002C33
:1023200074D0A9896181287A0E280AD002212173EC
:10233000E989E181288A0090EB8968886969039AB4
:102340003CE00121F3E70DA8009001AB22462946AD
:102350003046FFF759FB6FE0307B0A2800D0FFDFE3
:102360001220ADF80400ADF834704CB3A989618136
:10237000A4F810B0A4F80EB084F80C905CE020E053
:1023800002E031E039E042E0307B0B2800D0FFDF93
:10239000288AADF834701230ADF8040084B10421FD
:1023A0002173A9896181E989E181298A2182688A69
:1023B00000902B8A688804F11202696900F047FADC
:1023C0003AE0307B0C2800D0FFDF1220ADF804008B
:1023D000ADF834703CB305212173A4F80AB0A4F819
:1023E0000EB0A4F810B027E00DA8009001AB224673
:1023F00029463046FFF75CFA1EE00DA8009001ABBD
:10240000224629463046FFF7B6FB15E034E03B2173
:10241000ADF80400ADF8341074B3A4F80690A4F835
:1024200008B084F80AB007E0FFDF05E010000020E4
:10243000297A012917D0FFDFBDF80400AAF80000AF
:102440006CB1BDF834002080BDF804006080BDF898
:102450003400392803D03C2801D086F80CB011B0E4
:102460000020BDE8F08F3C21ADF80400ADF8341039
:1024700014B1697AA172DFE7AAF80000EFE72DE94D
:10248000F84356880F46804615460521304610F021
:102490002DF9040000D1FFDF123400943B46414681
:1024A00030466A6809F071FFBAE570B50D4605213E
:1024B00010F01CF9040000D1FFDF294604F11200DE
:1024C000BDE8704009F0FBBD70B50D46052110F068
:1024D0000DF9040000D1FFDF294604F11200BDE828
:1024E000704009F019BE70B50546052110F0FEF8E0
:1024F000040000D1FFDF04F1080321462846BDE8AF
:1025000070400422B1E470B50546052110F0EEF8E4
:10251000040000D1FFDF214628462368BDE8704053
:102520000522A2E470B50646052110F0DFF804008C
:1025300000D1FFDF04F1120009F0B4FD401D20F0CE
:10254000030511E0011D008803224318214630468F
:10255000FFF78BFC00280BD0607BABB2684382B2E4
:102560006068011D0FF07FFF606841880029E9D194
:1025700070BD70B50E46054606F0B4FF040000D1EC
:10258000FFDF0120207266726580207820F00F0046
:10259000C01C20F0F00030302070BDE8704006F024
:1025A000A4BF2DE9F0438BB00D461446814606A921
:1025B000FFF799FB002814D14FF6FF7601274FF45F
:1025C00020588CB103208DF800001020ADF81000C9
:1025D00007A8059007AA204604A911F033FE78B198
:1025E00007200BB0BDE8F0830820ADF808508DF847
:1025F0000E708DF80000ADF80A60ADF80C800CE0AC
:102600000698A17801742188C1818DF80E70ADF80B
:102610000850ADF80C80ADF80A606A4602214846C1
:10262000069BFFF789FBDCE708B501228DF8022045
:1026300042F60202ADF800200A4603236946FFF77E
:102640003EFC08BD08B501228DF8022042F60302C7
:10265000ADF800200A4604236946FFF730FC08BDA8
:1026600000B587B079B102228DF800200A88ADF854
:1026700008204988ADF80A1000236A460521FFF7B3
:102680005BFB07B000BD1020FBE709B1072316E490
:102690000720704770B588B00D461446064606A957
:1026A000FFF721FB00280ED17CB10620ADF80850C1
:1026B0008DF80000ADF80A40069B6A460821DC81CF
:1026C0003046FFF739FB08B070BD05208DF80000DB
:1026D000ADF80850F0E700B587B059B107238DF881
:1026E0000030ADF80820039100236A460921FFF766
:1026F00023FBC6E71020C4E770B588B00C46064639
:10270000002506A9FFF7EFFA0028DCD10698012181
:10271000123009F0F9FC9CB12178062921D2DFE8BA
:1027200001F0200505160318801E80B2C01EE28845
:1027300080B20AB1A3681BB1824203D90C20C2E760
:102740001020C0E7042904D0A08850B901E0062079
:10275000B9E7012913D0022905D004291CD0052985
:102760002AD00720AFE709208DF800006088ADF877
:102770000800E088ADF80A00A068039023E00A2072
:102780008DF800006088ADF80800E088ADF80A0018
:10279000A0680A25039016E00B208DF800006088E1
:1027A000ADF80800A088ADF80A00E088ADF80C008C
:1027B000A0680B25049006E00C208DF800006078DE
:1027C0008DF808000C256A4629463046069BFFF71F
:1027D000B3FA78E700B587B00D228DF80020ADF888
:1027E000081000236A461946FFF7A6FA49E700B524
:1027F00087B071B102228DF800200A88ADF8082058
:102800004988ADF80A1000236A460621FFF794FABA
:1028100037E7102035E770B586B0064601200D4633
:10282000ADF808108DF80000014600236A463046D6
:10283000FFF782FA040008D12946304605F054FC1F
:102840000021304605F06EFC204606B070BDF8B59C
:102850001C4615460E46069F10F07AF82346FF1DCB
:10286000BCB231462A4600940FF065FCF8BD30B486
:102870001146DDE902423CB1032903D0002330BCFC
:1028800008F024BB0123FAE71A8030BC704770B50A
:102890000C460546FFF72FFB2146284605F033FC82
:1028A0002846BDE87040012105F03CBC4FF0E02215
:1028B0004FF400400021C2F88001BFF34F8FBFF3F7
:1028C0006F8F1748016001601649900208607047D9
:1028D000134900B500220A600A60124B4FF0607283
:1028E0001A60002808BF00BD0F4A104BDFF840C037
:1028F00001280CD002281CBFFFDF00BD03200860A8
:102900001A604FF4000000BFCCF8000000BD0220A8
:1029100008601A604FF04070F6E700B5FFDF00BDB9
:1029200000F5004008F50140A002002014F5004029
:1029300004F5014070B50B2000F0BDF9082000F04F
:10294000BAF900210B2000F0D4F90021082000F092
:10295000D0F9F44C01256560A5600020C4F8400161
:10296000C4F84401C4F848010B2000F0B5F9082070
:1029700000F0B2F90B2000F091F9256070BD10B5A0
:102980000B2000F098F9082000F095F9E5480121A6
:1029900041608160E4490A68002AFCD10021C0F846
:1029A0004011C0F84411C0F848110B2000F094F910
:1029B000BDE81040082000F08FB910B50B2000F0E2
:1029C0008BF9BDE81040082000F086B900B530B1A1
:1029D000012806D0022806D0FFDF002000BDD34822
:1029E00000BDD34800BDD248001D00BD70B5D1491F
:1029F0004FF000400860D04DC00BC5F80803CF4829
:102A000000240460C5F840410820C43500F053F9A3
:102A1000C5F83C41CA48047070BD08B5C14A0021E0
:102A200028B1012811D002281CD0FFDF08BD4FF4C7
:102A30008030C2F80803C2F84803BB483C3001604C
:102A4000C2F84011BDE80840D0E74FF40030C2F8AA
:102A50000803C2F84803B44840300160C2F844118A
:102A6000B3480CE04FF48020C2F80803C2F84803D2
:102A7000AD4844300160C2F84811AD48001D0068FF
:102A8000009008BD70B516460D460446022800D9D0
:102A9000FFDF0022A348012304F110018B4000EB6B
:102AA0008401C1F8405526B1C1F84021C0F8043373
:102AB00003E0C0F80833C1F84021C0F8443370BDCA
:102AC0002DE9F0411D46144630B1012833D00228CB
:102AD00038D0FFDFBDE8F081891E002221F07F4160
:102AE0001046FFF7CFFF012D23D00020944D924FC9
:102AF000012668703E61914900203C39086002203F
:102B0000091D08608D490420303908608B483D3428
:102B1000046008206C6000F0DFF83004C7F804039C
:102B2000082000F0BBF88349F007091F08602E70E9
:102B3000D0E70120DAE7012B02D00022012005E0D6
:102B40000122FBE7012B04D000220220BDE8F04166
:102B500098E70122F9E774480068704770B500F003
:102B6000D8F8704C0546D4F840010026012809D158
:102B7000D4F80803C00305D54FF48030C4F8080327
:102B8000C4F84061D4F8440101280CD1D4F80803FA
:102B9000800308D54FF40030C4F80803C4F844613A
:102BA000012012F025FBD4F8480101280CD1D4F8FB
:102BB0000803400308D54FF48020C4F80803C4F884
:102BC0004861022012F014FB5E48056070BD70B5CC
:102BD00000F09FF85A4D0446287850B1FFF706FFE1
:102BE000687818B10020687012F002FB5548046044
:102BF00070BD0320F8E74FF0E0214FF40010C1F85A
:102C000000027047152000F067B84B4901200861A9
:102C1000082000F061B848494FF47C10C1F808035F
:102C20000020024601EB8003C3F84025C3F8402191
:102C3000401CC0B20628F5D37047410A43F609523A
:102C40005143C0F3080010FB02F000F5807001EB67
:102C50005020704710B5430B48F2376463431B0C98
:102C60005C020C60384C03FB0400384B4CF2F72438
:102C700043435B0D13FB04F404EB402000F580702C
:102C80004012107008681844086010BD2C48406855
:102C9000704729490120C1F800027047002809DB6C
:102CA00000F01F02012191404009800000F1E02066
:102CB000C0F80011704700280DDB00F01F02012151
:102CC00091404009800000F1E020C0F88011BFF37E
:102CD0004F8FBFF36F8F7047002809DB00F01F0292
:102CE000012191404009800000F1E020C0F88012ED
:102CF00070474907090E002804DB00F1E02080F846
:102D00000014704700F00F0000F1E02080F8141D5F
:102D100070470C48001F00680A4A0D49121D1160D7
:102D20007047000000B0004004B500404081004002
:102D300044B1004008F5014000800040408500405B
:102D40003400002014050240F7C2FFFF6F0C0100A1
:102D5000010000010A4810B5046809490948083112
:102D6000086012F0D9FA0648001D046010BD06493B
:102D7000002008604FF0E0210220C1F88002704777
:102D80001005024001000001FC1F004010B50D209D
:102D900000F077F8C4B26FF0040000F072F8C0B22F
:102DA000844200D0FFDF3E490120086010BD70B5AD
:102DB0000D2000F048F83B4C0020C4F8000101252C
:102DC000C4F804530D2000F04FF825604FF0E021C7
:102DD0006014C1F8000170BD10B50D2000F033F88B
:102DE0003048012141600021C0F80011BDE81040C9
:102DF0000D2000F039B82C4810B504682A492B483A
:102E0000083108602749D1F80001012804D0FFDF0C
:102E10002548001D046010BD2148001D00680022E7
:102E2000C0B2C1F8002112F0C3FEF1E710B51D4891
:102E3000D0F800110029FBD0FFF7DDFFBDE81040FE
:102E40000D2000F011B800280DDB00F01F02012159
:102E500091404009800000F1E020C0F88011BFF3EC
:102E60004F8FBFF36F8F7047002809DB00F01F0200
:102E7000012191404009800000F1E020C0F880125B
:102E80007047002804DB00F1E02090F8000405E022
:102E900000F00F0000F1E02090F8140D4009704799
:102EA00004D5004000D000401005024001000001A0
:102EB0004FF0E0214FF00070C1F8800101F5C071C2
:102EC000BFF34F8FBFF36F8FC1F80001384B8022E3
:102ED00083F8002441F8800C704700B502460420B6
:102EE000344903E001EBC0031B792BB1401EC0B293
:102EF000F8D2FFDFFF2000BD41F8302001EBC00118
:102F000000224A718A7101220A7100BD294A0021FA
:102F100002EBC0000171704710B50446042800D3CD
:102F2000FFDF244800EBC4042079012800D0FFDF34
:102F30006079A179401CC0B2814200D060714FF02D
:102F4000E0214FF00070C1F8000210BD2DE9F04102
:102F500019480568184919480831086014480426BA
:102F600090F80004134F4009154C042818D0FFDFD7
:102F700016E0217807EBC1000279012A08D14279D5
:102F800083799A4204D04279827157F831008047A0
:102F90002078401CC0B22070042801D3002020708B
:102FA000761EF6B2E5D20448001D0560BDE8F0814A
:102FB00019E000E0D80500201005024001000001E2
:102FC000500000200548064A0168914201D10021C5
:102FD000016004490120086070470000540000208F
:102FE000BEBAFECA40E5014070B50C46054609F080
:102FF00069FB21462846BDE870400AF04EBC704788
:103000002CFFFFFFDBE5B15100600200B700FFFFBE
:103010008400000069915B00935FFEEDA0843C7327
:10302000F87462145E06C0CB72F2136030B5F84DCE
:103030000446062CA9780ED2DFE804F0030E0E0E2B
:103040000509FFDF08E0022906D0FFDF04E00329BD
:1030500002D0FFDF00E0FFDFAC7030BD30B50446CA
:103060001038EB4D07280CD2DFE800F0040C060CFA
:103070000C0C0C00FFDF05E0287E112802D0FFDFDA
:1030800000E0FFDF2C7630BD2DE9F04111F044FA6D
:10309000044612F01DFC201AC5B206200FF0CEFA2D
:1030A000044606200FF0D2FA211AD94C207E1228AD
:1030B00018D000200F1807200FF0C0FA064607208E
:1030C0000FF0C4FA301A3918207E13280CD00020D3
:1030D0000144A078042809D000200844281AC0B26E
:1030E000BDE8F0810120E5E70120F1E70120F4E7E8
:1030F000C74810B590F825004108C54800F12600E2
:1031000005D00DF0A8FABDE8104006F001B80DF0AA
:1031100083FAF8E730B50446A1F120000D460A28ED
:103120004AD2DFE800F005070C1C2328353A3F445B
:10313000FFDF42E0207820283FD1FFDF3DE0B448A8
:103140008178052939D0007E122836D020782428AD
:1031500033D0252831D023282FD0FFDF2DE0207851
:1031600022282AD0232828D8FFDF26E0207822280A
:1031700023D0FFDF21E0207822281ED024281CD075
:1031800026281AD0272818D0292816D0FFDF14E0C7
:103190002078252811D0FFDF0FE0207825280CD0DB
:1031A000FFDF0AE02078252807D0FFDF05E0207840
:1031B000282802D0FFDF00E0FFDF257030BD1FB5FB
:1031C00004466A46002001F036FEB4B1BDF8022084
:1031D0004FF6FF700621824201D1ADF80210BDF812
:1031E0000420824201D1ADF80410BDF808108142DC
:1031F00003D14FF44860ADF8080068460DF0A7FF12
:1032000005F086FF04B010BD70B514460D460646A5
:10321000FEF759F858B90DB1A54201D90C2070BD7F
:10322000002408E056F82400FEF74DF808B11020FD
:1032300070BD641CE4B2AC42F4D3002070BD2DE933
:10324000F04105461F4690460E4600240068FEF7F2
:1032500087F830B9A98828680844401EFEF780F82E
:1032600008B110203CE728680028A88802D0B8429E
:1032700002D850E00028F5D0092031E72968085D20
:10328000B8B1671CCA5D152A2ED03CDC152A3AD28B
:10329000DFE802F03912222228282A2A313139396E
:1032A00039393939393939392200085D30BB641C64
:1032B000A4B2A242F9D833E00228DDD1A01C085CF8
:1032C00088F80000072801D2400701D40A2007E748
:1032D000307840F0010015E0C143C90707E001283C
:1032E00007D010E00620FBE60107A1F1805100297C
:1032F000F5D01846F4E63078810701D50B20EFE6CB
:1033000040F0020030702868005D384484B2A8881C
:10331000A04202D2B0E74FF4485382B2A242ADD8E5
:103320000020DDE610B5027843F2022354080122A2
:10333000022C12D003DC3CB1012C16D106E0032C88
:1033400010D07F2C11D112E0002011E080790324ED
:10335000B4EB901F09D10A700BE08079B2EB901F9B
:1033600003D1F8E780798009F5D0184610BDFF2019
:103370000870002010BD08B500208DF8000024481A
:1033800090F82E1049B190F82F0002280ED0032893
:103390000ED0FFDF9DF8000008BD1D4869462530AE
:1033A00001F098FD0028F5D0FFDFF3E7032000E0EF
:1033B00001208DF80000EDE738B50C46054669465A
:1033C00001F088FD00280DD19DF80010207861F3F0
:1033D0004700207055F8010FC4F80100A888A4F830
:1033E0000500002038BD38B51378A8B1022813D0E5
:1033F000FF281AD007A46D46246800944C7905EB89
:103400009414247864F347031370032809D00FE061
:10341000EC0100200302FF0123F0FE0313700228D9
:10342000F3D1D8B240F0010005E043F0FE00107087
:10343000107820F0010010700868C2F80100888838
:10344000A2F8050038BD02210FF050B938B50C467E
:103450000978222901D2082038BDADF800008DF886
:10346000022068460DF039F905F052FE050003D13F
:1034700021212046FFF74EFE284638BD1CB500200E
:103480008DF80000CDF80100ADF80500FE4890F879
:103490002E00022801D0012000E000208DF8070056
:1034A00068460DF083FA002800D0FFDF1CBD002223
:1034B0000A80437892B263F3451222F040020A80F8
:1034C00000780C282BD2DFE800F02A06090E11162E
:1034D000191C1F220C2742F0110009E042F01D00C8
:1034E00008800020704742F0110012E042F0100006
:1034F00040F00200F4E742F01000F1E742F0010072
:10350000EEE742F0010004E042F00200E8E742F09A
:10351000020040F00400E3E742F00400E0E7072087
:1035200070472DE9FF478AB00025BDF82C60824620
:103530001C4690468DF81C50700703D56068FDF757
:10354000C2FE68B9D04F4FF0010997F82E0058B16C
:1035500097F82F00022807D16068FDF701FF18B126
:1035600010200EB0BDE8F087300702D5A089802872
:1035700016D8700705D4B8F1000F02D097F82400D0
:1035800070B1E07DC0F300108DF81B00617D072055
:1035900041B1012906D00229E3D00429E1D12CE070
:1035A0000720DEE749468DF81790F00609D4A27D82
:1035B000072032B1012A04D0022A05D0042AD0D132
:1035C0001BE08DF8191002E002208DF819008DF82B
:1035D00015806068B0B107A9FFF7A4FE0028C0D12C
:1035E0009DF81C00FF280AD0606850F8011FCDF834
:1035F0000F108088ADF8130008E00620B1E743F211
:103600000220AEE7CDF80F50ADF81350E07B002854
:10361000F3D1207C0028F0D1607C0028EDD1A07C83
:103620000028EAD1E07CC006E7D18DF800A0BDF803
:103630002C00ADF80200A0680190A068029004F18F
:103640000F0001F03BFC8DF80C00FFF794FE8DF8A5
:103650000D009DF81C008DF80E008DF816508DF8A9
:103660001850E07D08A900F00F008DF81A00684698
:103670000DF0B7FE05F04CFD73E7F0B58FB00025F7
:103680008DF830508DF814508DF8345006468DF872
:103690002850019502950395049519B10FC901AC05
:1036A00084E80F00784CA078052801D004280CD1BC
:1036B00001986168884200D120B90398E168884286
:1036C00003D110B108200FB0F0BD207DC00601D598
:1036D0001F2700E0FF273B460DAA05A903A8FFF717
:1036E000AEFD0028EFD1A08AC10702D0C00600D4E9
:1036F000EE273B460AAA0CA901A8FFF7A0FD002867
:10370000E1D19DF81400C00701D00A20DBE7A08AB0
:10371000410708D4A17D31B19DF82810890702D056
:1037200043F20120CFE79DF82810C90709D04007D0
:1037300007D4208818B144F25061884201D907208B
:10374000C1E78DF818508DF81960BDF80800ADF884
:103750001A000198079006A80DF05DFE05F0D8FC50
:103760000028B0D18DF820508DF82160BDF81000F0
:10377000ADF822000398099008A80DF06BFE05F043
:10378000C7FC00289FD101AD241D95E80F0084E8F7
:103790000F00002097E770B586B00D46040005D0F5
:1037A000FDF7DEFD20B1102006B070BD0820FBE75C
:1037B0002078C107A98802D0FF2902D303E01F297E
:1037C00001D20920F0E780073BD4FFF75DFC38B158
:1037D0002178C1F3C100012804D0032802D005E0FC
:1037E0001320E1E7284890F82400C8B1C8074FF03B
:1037F00001064FF0000502D08DF80F6001E08DF852
:103800000F50FFF7B8FD8DF8000020786946C0F32F
:10381000C1008DF8010060788DF80250C20801D017
:103820000720C1E778B1C20701D08DF80260820796
:1038300005D59DF8022042F002028DF802204007D3
:1038400003D50620B0E78DF80260002022780B181F
:10385000C2F38002DA7001EB40026388D380401C1F
:10386000A388C0B253810228F0D3207A0028E8D17F
:10387000607A0028E5D1A07A0028E2D1E07A002819
:10388000DFD1207BC00601E0EC010020D9D104F19A
:10389000080001F013FB8DF80E0068460DF0B1F939
:1038A00005F036FC00288DD18DF810608DF8115090
:1038B000E088ADF81200ADF8145004A80DF0F4F94A
:1038C00005F026FC00288CD12078C00701D01520F7
:1038D00000E01320FFF7C2FB002065E72DE9FF475A
:1038E0000220FC4E8DF804000027708EADF8060013
:1038F000B84643F202094CE001A80EF05EFE050056
:1039000006D0708EA8B3A6F83280ADF806803EE0EF
:10391000039CA07F01072DD504F124000090A28E06
:10392000BDF80800214604F1360301F05CFC0500F7
:1039300005D04D452AD0112D3CD0FFDF3AE0A07FC5
:1039400020F00801E07F420862F3C711A1778108E7
:1039500061F30000E07794F8210000F01F0084F884
:1039600020002078282826D129212046FFF7D2FBE5
:1039700021E014E040070AD5BDF8080004F10E016B
:1039800001F0B2FA05000DD04D4510D100257F1C85
:10399000FFB202200EF052FE401CB842ACD8052DFA
:1039A00011D008E0A07F20F00400A07703E0112DE3
:1039B00000D0FFDF0025BDF806007086052D04D07D
:1039C000284604B0CEE5A6F832800020F9E770B5AD
:1039D0000646FFF738FD054605F084FD040000D1DA
:1039E000FFDF6680207820F00F00801C20F0F000C0
:1039F000203020700320207295F83E006072BDE8F0
:103A0000704005F072BD2DE9F04786B0040000D18A
:103A1000FFDF2078AF4D20F00F00801C20F0F00079
:103A20007030207060680178491F1B2933D2DFE8AD
:103A300001F0FC32323255FB320EFBFB42FA3232DD
:103A40003278FAFAF9F83232FAFAF7F6FA00C6885A
:103A50003046FFF7F8FC0546304607F035F9E0B18F
:103A60006068007A85F83E0021212846FFF752FB66
:103A70003046FEF75AFB304603F058FE314601202F
:103A800012F056FBA87F20F01000A877FFF726FF62
:103A9000002800D0FFDF06B064E5207820F0F000B9
:103AA000203020700320207266806068007A607287
:103AB00005F01BFDD8E7C5882846FFF7C4FC00B910
:103AC000FFDF60680079012800D0FFDF6068017ABD
:103AD00006B02846BDE8F04707F0D5BCC68830469A
:103AE000FFF7B1FC050000D1FFDF05F0FEFC6068C8
:103AF00031460089288160684089688160688089D2
:103B0000A881012012F014FB0020A875A87F00F006
:103B100003000228BFD1FFF7E1FE0028BBD0FFDF82
:103B2000B9E700790228B6D000B1FFDF05F0DDFC6F
:103B30006668B6F806A0307A361D012806D0687E81
:103B4000814605F051FA070003D101E0E878F7E774
:103B5000FFDF0022022150460EF0BFFD040000D11D
:103B6000FFDF22212046FFF7D5FA3079012800D067
:103B70000220A17F804668F30101A177308B20816C
:103B8000708B6081B08BA08184F822908DF80880C2
:103B9000B8680090F86801906A46032150460EF01C
:103BA0009CFD00B9FFDFB888ADF81000B8788DF83B
:103BB000120004AA052150460EF08FFD00B9FFDF68
:103BC000B888ADF80C00F8788DF80E0003AA04212F
:103BD00050460EF082FD00B9FFDF062106F112000B
:103BE00001F0A0F940B37079800700D5FFDF71794B
:103BF000E07D61F34700E075D6F80600A0617089AA
:103C0000A083062106F10C0001F08CF9F0B195F8C3
:103C100025004108607861F34700607006E040E0ED
:103C200038E070E058E04DE02EE042E0D5F82600A4
:103C3000C4F80200688D12E0E07D20F0FE00801CD8
:103C4000E075D6F81200A061F08AD9E7607820F01C
:103C5000FE00801C6070F068C4F80200308AE080CA
:103C6000B8F1010F04D0B8F1020F05D0FFDF12E761
:103C70000320FFF7DBF90EE7287E122800D0FFDFD4
:103C80001120FFF7EBF906E706B02046BDE8F04744
:103C900001F032BD05F029FC15F8300F40F00200AC
:103CA00005E005F022FC15F8300F40F00400287004
:103CB000F1E6287E13280AD01528D8D15FF0160027
:103CC000FFF7CCF906B0BDE8F04705F00EBC1420B4
:103CD000F6E70000EC010020A978052909D00429A5
:103CE000C5D105F002FC022006B0BDE8F047FFF7A1
:103CF0009DB900790028BAD0E87801F0C6F805F03F
:103D0000F4FB0320F0E7287E122802D1687E01F040
:103D1000BCF81120D4E72DE9F047054600784FF0B4
:103D200000080009DFF8C0A891460C464646012865
:103D300075D0022874D007280AD00A2871D0FFDF76
:103D4000A9F8006014B1A4F800806680002009E49E
:103D50006968012704F108000A784FF0020C4FF659
:103D6000FF73172A7ED00EDC142A32D006DC052A17
:103D700068D0092A10D0102A75D120E0152A73D0F6
:103D8000162AF9D1F8E0183A082A6CD2DFE802F0D6
:103D9000F36B6B0ACAF2DFF1C8884FF012081026E5
:103DA00021468DE14FF01C080A26BCB38888A0800C
:103DB0006868807920726868C0796072C0E74FF0E7
:103DC0001B08142654B30320207268688088A080E2
:103DD000B6E70A793C2AB3D00D1D4FF010082C2607
:103DE000E4B16988A180298B6182298B2182698B4A
:103DF000A182A98BE1826B790246A91D1846FFF7C3
:103E0000F2FA2979002001290CD084F80FC0FF2193
:103E10002176E06120626062A06291E70FE02EE10E
:103E200051E18CE1E77320760AF1040090E80E007E
:103E3000DAF81000C4E90930C4E9071280E7A9F8EC
:103E4000006083E72C264FF01D08002CF7D00546B4
:103E5000A380887B2A880F1D60F300022A80887B5C
:103E6000400802E09DE007E1BEE060F341022A80E5
:103E7000887B800860F382022A80887BB91CC00896
:103E800060F3C3022A80B87A0011401C60F3041268
:103E900002F07F0028807878AA1CFFF7A4FA387D0A
:103EA00005F1090207F11501FFF79DFA387B01F0D2
:103EB00048F82874787B01F044F86874F87EA87498
:103EC000787AE874387F2875B87B6875388AE88214
:103ED000DAF81C00A861B87A524697F808A0C0F337
:103EE0004111012904D0108C504503D2824609E0CB
:103EF000FFDF10E0022903D0288820F0600009E0ED
:103F0000504504D1288820F06000403002E0288825
:103F100040F060002880A4F824A0524607F11D015B
:103F2000A86996E011264FF02008002C87D0A380C6
:103F3000686804F10A02007920726868007B607288
:103F400069688B1D48791946FFF74DFAF8E60A268D
:103F50004FF02108002CE9D08888A080686880791B
:103F600020726868C07960729AF8301021F00401FC
:103F70009FE065E04CE06FE00B264FF02208002C3C
:103F8000D4D0C888A0806868007920726868007AF8
:103F900000F0D7FF60726868407A00F0D2FFA0722C
:103FA000CEE61C264FF02608002CBFD0A380686800
:103FB000407960726868007AA0720AF1040090E8A3
:103FC0000E00DAF81000C4E90530C4E9031268688D
:103FD00000793C2803D0432803D0FFDFB0E62772E6
:103FE000AEE684F808C0ABE610264FF02408002C9B
:103FF0009CD08888A0806868807920816868807AF1
:10400000608168680089A08168688089E08197E69E
:1040100010264FF02308002C88D08888A08068687C
:10402000C088208168680089608168684089A081B3
:1040300068688089E0819AF8301021F0020138E048
:1040400030264FF02508002C85D0A38069682822EF
:10405000496820F047FC73E614264FF01B08002C3B
:104060008ED0A380686800790128BAD02772DAE977
:104070000710C4E9031063E64A46214660E0287A47
:10408000012803D0022817D0FFDF59E610264FF091
:104090001F08002C89D06888A080A8892081E88921
:1040A0006081288AA081688AE0819AF8301021F026
:1040B00001018AF8301043E64FF012081026688894
:1040C00000F01DFF3CE6287AC8B3012838D002284A
:1040D00036D0032801D0FFDF32E609264FF0110861
:1040E000002C85D06F883846FFF7ADF990F822A0F4
:1040F000A780687A2072042138460EF009FB05215A
:1041000038460EF005FB002138460EF001FB012178
:1041100038460EF0FDFA032138460EF0F9FA022176
:1041200038460EF0F5FA062138460EF0F1FA07216E
:1041300038460EF0EDFA504600F0A7FE00E6FFE725
:104140002846BDE8F04701F061BC70B5012803D0F6
:10415000052800D0FFDF70BD8DB22846FFF773F948
:10416000040000D1FFDF20782128F4D005F0BAF94F
:1041700080B1017821F00F01891C21F0F00110318C
:1041800001700221017245800020A075BDE87040D9
:1041900005F0ABB921462846BDE870401322FFF771
:1041A00055B92DE9F04116460C00804600D1FFDFDD
:1041B000307820F00F00801C20F0F00010303070BC
:1041C0002078012804D0022818D0FFDFBDE8F08154
:1041D0004046FFF738F9050000D1FFDF0320A8753E
:1041E00005F083F994E80F00083686E80F00FE48D2
:1041F00010F8301F41F001010170E7E74046FFF77A
:1042000022F9050000D1FFDFA1884FF6FF700027DB
:10421000814202D1E288824203D0814201D1E0880A
:1042200040B105F062F994E80F00083686E80F0007
:10423000AF75CBE7A87D0128C8D17823002241467D
:1042400011F0CCFE0220A875C0E738B505460C4633
:104250000846FDF738F818BB203D062D4AD2DFE8A6
:1042600005F0031B373C42300021052011F036FFDA
:1042700008B1112038BDA01C0CF0BCFF04F048FFB1
:10428000050038D1002208231146052011F0A6FEB2
:10429000052830D0FFDF2EE06068FDF758F808B140
:1042A000102038BD618820886A460DF054FA04F069
:1042B0002FFF05001FD16068E8B1BDF80010018034
:1042C00019E0A07800F0010120880DF075FA0EE0E9
:1042D000206801F047FE05460DE0207800F001005F
:1042E0000CF082F903E0618820880DF0B0F904F049
:1042F0000FFFF0E70725284638BD70B505460C4688
:104300000846FDF706F808B1102070BD202D07D033
:10431000212D0DD0222D0BD0252D09D0072070BDC9
:104320002088A11C0CF036FABDE8704004F0F0BE05
:10433000062070BDAC482530704708B53421AA4826
:1043400020F071FB0120FEF771FE1120FEF786FEC2
:10435000A5496846263105F05BF8A3489DF8002082
:1043600010F8251F62F3470121F0010101700021BF
:1043700041724FF46171A0F8071002218172FEF7BB
:10438000B7FE00B1FFDFFDF763F801F080F908BD6B
:1043900010B50C464021204620F023FBA07F20F0E2
:1043A0000300A077202020700020A07584F823004F
:1043B00010BD70472DE9FC410746FCF784FF10B1A2
:1043C0001020BDE8FC81884E06F12501D6F82500B5
:1043D0000090B6F82950ADF8045096F82B408DF8AF
:1043E00006403846FEF7E8FF0028EAD1FEF780FED7
:1043F0000028E6D0009946F8251FB580B471E0E7A3
:1044000010B50446FCF785FF08B1102010BD7648B2
:104410007549224690F8250026314008FEF7E3FF53
:10442000002010BD3EB504460D460846FCF771FF5E
:1044300008B110203EBD14B143F204003EBD6A48ED
:104440008078052803D0042801D008203EBD6946A5
:1044500002A80AF069FA2A4669469DF80800FEF7A4
:10446000C2FF00203EBDFEB50D4604004FF0000720
:1044700011D00822FEF7C8FE002811D1002608E05E
:1044800054F826006946FEF74DFF002808D1761C37
:10449000F6B2AE42F4D30BF0F1FF10B143F20320B9
:1044A000FEBD514E86F824700CB300271BE000BF00
:1044B00054F8270002A9FEF735FF00B1FFDF9DF891
:1044C00008008DF8000054F8270050F8011FCDF8BF
:1044D00001108088ADF8050068460BF0F4FF00B1CC
:1044E000FFDF7F1CFFB2AF42E2D386F824500020EA
:1044F000FEBD2DE9F0478AB01546894604001ED05E
:104500000F4608222946FEF77FFE002811D100261B
:1045100013E000BF54F826006946103000F0DAFCC2
:10452000002806D13FB157F82600FCF7CCFE10B1A9
:1045300010200AB00BE4761CF6B2AE42EAD3002695
:10454000A5F101081CE000BF06F1010A0AF0FF070F
:1045500012E000BF54F82600017C4A0854F82710E6
:104560000B7CB2EB530F05D106221130113120F034
:104570008DF958B17F1CFFB2AF42EBD30AF0FF06B2
:104580004645E1DB4E4624B1012003E043F205201D
:10459000CFE700200BF0BCFF10B90BF0C5FF10B146
:1045A00043F20420C5E774B300270DF1170828E093
:1045B00054F827006946103000F08CFC00B1FFDF92
:1045C00054F82700102250F8111FCDF801108088F0
:1045D000ADF8050054F827100DF1070020F082F91E
:1045E000AEB156F8271001E0EC0100201022404641
:1045F00020F078F968460BF04BFF00B1FFDF7F1C1D
:10460000FFB2AF42D4D3FEF739FF002091E7404616
:1046100001F09CFCEEE730B585B00446FCF753FE94
:1046200018B96068FCF79CFE10B1102005B030BDD1
:1046300060884AF2B811884206D82078F84D28B12F
:10464000012806D0022804D00720EFE7FEF750FD2E
:1046500018E06078022804D0032802D043F2022038
:10466000E4E785F82F00C1B200200090ADF8040007
:1046700002292CD0032927D0FFDF68460BF0EBFF7F
:1046800004F046FD0028D1D1606801F052FC20788A
:1046900058B101208DF800000DF1010001F056FC29
:1046A00068460DF0EDF800B1FFDF207885F82E00A8
:1046B000FEF7E4FE608860B1A88580B20BF020FFB1
:1046C00000B1FFDF0020B1E78DF80500D5E74020FD
:1046D000FAE74FF46170EFE710B50446FCF719FEF6
:1046E00020B9606838B1FCF732FE08B1102010BD67
:1046F000606801F02BFCCA4830F82C1F6180C1783B
:10470000617080782070002010BD2DE9F8431446B8
:1047100089460646FCF7FDFDA0B94846FCF720FE99
:1047200080B92046FCF71CFE60B9BD4DA878012871
:1047300000D13CB13178FF2906D049B143F20400E1
:10474000BDE8F8831020FBE7012801D00420F7E73B
:10475000CCB3052811D004280FD069462046FEF7B7
:10476000A6FE0028ECD1217D49B1012909D00229FA
:1047700009D0032909D00720E2E70820E0E7024634
:1047800004E0012202E0022200E0032280462346E8
:10479000174600200099FEF7C4FE0028D0D1A0895A
:1047A0002880A07BE875BDF80000A882AF75BDF831
:1047B0000010090701D5A18931B1A1892980C0075D
:1047C00004D0032003E006E08021F7E70220FEF793
:1047D0002DFC86F800804946BDE8F8430020FEF72E
:1047E0004CBF7CB58E4C05460E46A078022803D0FF
:1047F000032801D008207CBD15B143F204007CBD24
:1048000007200DF023FF10B9A078032806D0FEF78B
:104810003BFC28B1A078032804D009E012207CBD1D
:1048200013207CBD304600F013FB0028F9D1E67060
:10483000FEF7A1FD09F0B5FF01208DF800008DF80D
:1048400001008DF802502088ADF80400E07D8DF85D
:10485000060068460CF0BEFE04F05AFC0028E0D1C9
:10486000A078032804D00420FEF7E0FB00207CBDE4
:10487000E07800F0FDFA0520F6E71CB510B143F230
:1048800004001CBD664CA078042803D0052801D084
:1048900008201CBD00208DF8000001218DF80110BA
:1048A0008DF8020068460CF095FE04F031FC0028FB
:1048B000EFD1A078052805D05FF00200FEF7B6FB27
:1048C00000201CBDE07800F0E0FA0320F6E72DE9B7
:1048D000FC4180460E4603250846FCF741FD0028B2
:1048E00066D14046FEF7AFFD040004D020782228B0
:1048F00004D2082065E543F2020062E5A07F00F0E3
:1049000003073EB1012F0CD000203146FEF757FCC3
:104910000500EFD1012F06D0022F1AD0FFDF284665
:104920004FE50120F1E7A07D3146022801D011B109
:1049300007E0112045E56846FCF797FE0028D9D12D
:104940006946404606F062FD0500E8D10120A075E9
:10495000E5E7A07D032804D1314890F83000C00776
:1049600001D02EB30EE026B1A07F40071ED4002157
:1049700000E00121404606F069FD0500CFD1A07599
:10498000002ECCD03146404600F0AEFA0546112844
:10499000C5D1A07F4107C2D4316844F80E1F7168A9
:1049A000616040F0040020740025B8E71125B6E7E7
:1049B000102006E570B50C460546FEF744FD0100E3
:1049C00005D022462846BDE87040FEF73FBD43F2C1
:1049D000020070BD10B5012807D1114B9B78012B47
:1049E00000D011B143F2040010BD0BF0BBFDBDE8D7
:1049F000104004F08DBB012300F051BA00231A4689
:104A0000194600F04CBA70B506460C460846FCF74D
:104A10005AFC18B92068FCF77CFC18B1102070BD56
:104A2000EC010020F84D2A7E112A04D0132A00D36D
:104A30003EB10820F3E721463046FEF7ACFE60B1F8
:104A4000EDE70920132A0DD0142A0BD0A188FF29E5
:104A5000E5D31520FEF702FB0020D4E90012C5E9DA
:104A60000712DCE7A1881F29D9D31320F2E71CB570
:104A7000E548007E132801D208201CBD00208DF8D7
:104A8000000068460CF010F904F042FB0028F4D155
:104A90001120FEF7E3FA00201CBD2DE9F04FDFF8EE
:104AA00068A3814691B09AF818009B4615460C46BB
:104AB000132803D3FFF7DBFF00281FD12046FCF7A4
:104AC00002FC78BB2846FCF7FEFB58BB20784FF071
:104AD0000107C0074FF0000102D08DF83A7001E0E5
:104AE0008DF83A1020788846C0F3C1008DF8000098
:104AF00060788DF80910C10803D0072011B0BDE817
:104B0000F08F80B1C10701D08DF80970810705D5FC
:104B10009DF8091041F002018DF80910400704D5F5
:104B20000620EBE720E08DF809709DF80900810769
:104B300003D540F001008DF8090000206E4606EB19
:104B4000400162884A81401CA288C0B20A820328C0
:104B5000F5D32078C0F3C100012821D003281FD04D
:104B60004846FCF7B0FB08B11020C7E799F80000F1
:104B7000400808D0012809D0022807D0032805D012
:104B800043F20220BAE78DF8028001E08DF802704E
:104B9000484650F8011FCDF803108088ADF8070093
:104BA000FEF7E9FB8DF801000020424606EB4001CC
:104BB0002B88CB826B888B83AB884B84EB880B85EF
:104BC000401CCA85C0B28A860328EFD3E088ADF8BE
:104BD0003C0068460CF083F900288ED19AF8180042
:104BE0005546112801D0082088E706200DF02EFD3B
:104BF00038B12078C0F3C100012804D0032802D0C6
:104C000006E012207AE795F8240000283FF475AFFB
:104C1000FEF73AFA022801D213206FE7584600F057
:104C200017F90028A1D185F819B068460CF069FA87
:104C300004F06EFA040098D1687E00F019F9122091
:104C4000FEF70CFA204659E770B56F4D287E122802
:104C500001D00820E3E60CF057FA04F059FA0400FA
:104C600005D1687E00F011F91120FEF7F7F9204612
:104C7000D5E670B5064615460C460846FCF749FBD6
:104C800018B92846FCF745FB08B11020C7E62A46AC
:104C9000214630460CF03FFD04F03AFA0028F5D1E9
:104CA00021787F29F2D10520B9E67CB505460C466E
:104CB0000846FCF708FB08B110207CBD2846FEF72B
:104CC000C2FB20B10078222804D208207CBD43F228
:104CD00002007CBD4C4890F83000400701D51120FF
:104CE0007CBD2178C80802D16078C20801D00720B5
:104CF0007CBD890801D1800801D006207CBDADF8BB
:104D0000005020788DF8020060788DF803000220B2
:104D1000ADF8040068460BF0E3FE04F0F9F97CBD41
:104D200070B586B014460D460646FEF78CFB28B1DA
:104D30000078222805D2082006B070E643F202006F
:104D4000FAE72846FCF70CFB20B944B12046FCF7F3
:104D5000FEFA08B11020EFE700202060A0802A486A
:104D600090F83000800701D51120E5E703A930460F
:104D70000BF05CFD18B100BF04F0CAF9DCE7ADF838
:104D80000060BDF81400ADF80200BDF81600ADF8E3
:104D90000400BDF81000BDF81210ADF80600ADF823
:104DA00008107DB1298809B1ADF80610698809B1EC
:104DB000ADF80210A98809B1ADF80810E98809B169
:104DC000ADF80410DCB1BDF80610814201D9081A13
:104DD0002080BDF80210BDF81400814201D9081AE4
:104DE0006080BDF80800BDF80410BDF8162001442D
:104DF000BDF812001044814201D9081AA08068460B
:104E00000BF0D3FDB8E70000EC0100201CB55249BF
:104E10000968CDE9001068460CF063F804F078F9F1
:104E20001CBD1CB500200090019068460CF059F89C
:104E300004F06EF91CBD108008885080488890806E
:104E4000C88810818888D080002050819081704768
:104E500010B5044604F0C8F830B1407830B12046AF
:104E600004F0E7FB002010BD052010BD122010BD8E
:104E700010B504F0B9F8040000D1FFDF607800B984
:104E8000FFDF6078401E607010BD10B504F0ACF814
:104E9000040000D1FFDF6078401C607010BD1CB5BD
:104EA000ADF800008DF802308DF803108DF8042065
:104EB00068460CF0F3FB04F02BF91CBD0CB527A2DF
:104EC000D2E90012CDE900120079694601EB5010D9
:104ED00000780CBD0278520804D0012A02D043F2B7
:104EE00002207047FEF71EBA1FB56A46FFF7A3FF00
:104EF00068460CF03CF904F00BF904B010BD70B535
:104F00000C0006460DD0FEF79EFA050000D1FFDF2B
:104F1000A68028892081288960816889A081A88944
:104F2000E0817CE510B500231A4603E0845C23434E
:104F3000521CD2B28A42F9D30BB1002010BD01201D
:104F400010BD00B530B1012803D0022801D0FFDF29
:104F5000002000BDFF2000BDCC4D02000706050467
:104F60000302010010B50446FCF7ADF908B11020AA
:104F700010BD2078C0F30210042807D860780728F5
:104F800004D3A178102901D8814201D2072010BD95
:104F9000E078410706D421794A0703D4000701D4F9
:104FA000080701D5062010BD002010BD10B51378EC
:104FB0005C08837F64F3C713837713789C08C37FEF
:104FC00064F30003C3771078C309487863F34100A2
:104FD000487013781C090B7864F347130B7013782F
:104FE000DB0863F3000048705078487110BD10B5BD
:104FF000C4780B7864F300030B70C478640864F31E
:1050000041030B70C478A40864F382030B70C47866
:10501000E40864F3C3030B700379117863F30001B0
:10502000117003795B0863F34101117003799B08E8
:1050300063F3820111700079C00860F3C30111703D
:1050400010BD70B514460D46064604F04BFA80B10B
:105050000178182221F00F01891C21F0F001A03104
:1050600000F8081B21461FF082FCBDE8704004F0E8
:105070003CBA29463046BDE870401322FEF7E6B937
:105080002DE9F047064608A8894690E830041F46F7
:105090009046142128461FF0C6FC0021CAF80010D3
:1050A000B8F1000F03D0B9F1000F03D114E0387844
:1050B000C00711D02068FCF72CF9C0BBB8F1000F75
:1050C00007D120681230286020681430686020689A
:1050D000A8602168CAF800103878800724D5606875
:1050E000FCF735F918BBB9F1000F21D0FFF722F911
:1050F0000168C6F868118188A6F86C11807986F875
:105100006E0101F0F8FCF94FEF60626862B196F849
:10511000680106F2691140081032FEF764F91022A6
:10512000394660681FF0DEFB0020BDE8F08706E02E
:10513000606820B1E8606068C6F86401F4E7102098
:10514000F3E730B5054608780C4620F00F00401C08
:1051500020F0F001103121700020607095F82300DC
:1051600030B104280FD0052811D0062814D0FFDF55
:1051700020780121B1EB101F04D295F8200000F037
:105180001F00607030BD21F0F000203002E021F0FF
:10519000F00030302070EBE721F0F0004030F9E70C
:1051A000F0B591B0022715460C4606463A46ADF8D2
:1051B0000870092103AB04F0FEFF0490002810D012
:1051C00004208DF804008DF80170E03409960594F0
:1051D0008DF818500AA968460EF078FF00B1FFDF7D
:1051E000012011B0F0BD10B588B00C460A99ADF899
:1051F0000000C3B11868CDF802005868CDF8060069
:10520000ADF80A20102203A81FF06CFB68460CF0D2
:105210001EF803F07DFF002803D1A17F41F01001AB
:10522000A17708B010BD0020CDF80200E6E72DE917
:10523000F84F0646808A0D4680B28246FEF703F993
:1052400004463078DFF8A48200274FF00209A8F165
:1052500020080F2870D2DFE800F06FF23708387DA1
:105260008CC8F1F0EFF35FF3F300A07F00F00300D0
:10527000022809D05FF0000080F0010150460DF0D7
:1052800035FA050003D101E00120F5E7FFDF98F8CA
:105290005C10C90702D0D8F860000BE0032105F1CB
:1052A0001D0010F066FCD5F81D009149B0FBF1F22D
:1052B00001FB1200C5F81D0070686867B068A86738
:1052C0002078252800D0FFDFCAE0A07F00F003008F
:1052D000022809D05FF0000080F0010150460DF077
:1052E00005FA060003D101E00120F5E7FFDF307881
:1052F000810702D52178252904D040F001003070C3
:10530000BDE8F88F85F80090307F287106F11D0008
:105310002D36C5E90206F3E7A07F00F0030002285E
:1053200008D0002080F0010150460DF0DFF90400A4
:1053300004D102E00120F5E7A7E1FFDF2078C106F4
:1053400004D5072028703D346C60D9E740F0080090
:105350002070D5E7E07F000700D5FFDF307CB28802
:1053600000F0010301B05046BDE8F04F092105F0FF
:10537000ADBD04B9FFDF716821B1102204F1240032
:105380001FF0B0FA28212046FDF7C4FEA07F00F0F0
:10539000030002280ED104F12400002300901A46D5
:1053A00021465046FFF71FFF112807D0292120462C
:1053B000FDF7B0FE307A84F82000A1E7A07F000757
:1053C00000D5FFDF14F81E0F40F008002070E782C0
:1053D000A761E761C109607861F34100014660F3AC
:1053E00082016170307AE0708AE7A07F00F00300EC
:1053F000022809D05FF0000080F0010150460DF056
:1054000075F9040003D101E00120F5E7FFDF022177
:1054100004F1850010F0ADFB0420287004F5B47091
:105420006860B4F885002882304810387C346C619C
:10543000C5E9028064E703E024E15BE02DE015E0CC
:10544000A07F00F00300022807D0002080F00101B7
:1054500050460DF04BF918B901E00120F6E7FFDFE7
:10546000324621465046BDE8F84FEAE504B9FFDF71
:1054700020782128A1D93079012803D1E07F40F09C
:105480000800E077324621465046FFF7DAFD204615
:10549000BDE8F84F2321FDF73DBE3279AA8005F122
:1054A00008030921504604F086FEE86010B105208B
:1054B000287025E7A07F00F00300022808D0002014
:1054C00080F0010150460DF011F9040003D101E014
:1054D0000120F5E7FFDF04F1620102231022081F1B
:1054E0000CF08BFF07703179417009E74C02002006
:1054F00040420F00A07F00F00300022808D00020E7
:1055000080F0010150460DF0F1F8050003D101E0F3
:105510000120F5E7FFDF95F8840000F00300012883
:105520007AD1A07F00F00307E07F10F0010602D0DF
:10553000022F04D133E095F8A000C0072BD0D5F896
:10554000601121B395F88320087C62F3870008740A
:10555000A17FCA09D5F8601162F341000874D5F83B
:10556000601166F300000874AEB1D5F86001102236
:1055700004F1240188351FF0B5F9287E40F00100C0
:105580002876287820F0010005F8880900E016B197
:10559000022F04D02DE095F88800C00727D0D5F859
:1055A0005C1121B395F88320087C62F387000874AE
:1055B000A17FCA09D5F85C1162F341000874D5F8DF
:1055C0005C1166F3000008748EB1D5F85C011022FE
:1055D00004F1240188351FF085F9287840F0010096
:1055E00005F8180B287820F0010005F8A009022F13
:1055F00044D0002000EB400005EBC00090F888008C
:10560000800709D595F87C00D5F86421400805F19C
:105610007D011032FDF7E7FE8DF8009095F88400CB
:105620006A4600F003008DF8010095F888108DF8A7
:10563000021095F8A0008DF803002146504601F0B5
:1056400043FA2078252805D0212807D0FFDF2078CD
:10565000222803D922212046FDF75CFDA07F00F01F
:10566000030002280CD0002080F0010150460DF00C
:105670004FF800283FF44FAEFFDF41E60120B9E7C5
:105680000120F1E7706847703AE6FFDF38E670B551
:10569000FE4C002584F85C5025660EF0E4FC04F115
:1056A0001001204603F0DAFE84F8305070BD70B56A
:1056B0000D46FDF7C8FE040000D1FFDF4FF4B871BE
:1056C00028461FF0B0F904F124002861A07F00F003
:1056D0000300022808D0012105F1E0000EF0C4FC0F
:1056E000002800D0FFDF70BD0221F5E70A46014621
:1056F00002F1E0000EF0D8BC70B50546406886B0F7
:1057000001780A2906D00D2933D00E292FD0FFDFCA
:1057100006B070BD86883046FDF795FE040000D1C6
:10572000FFDF20782128F3D028281BD168680221C8
:105730000E3001F0BEF9A8B168680821801D01F0A3
:10574000B8F978B104F1240130460BF045FF03F0BD
:10575000DFFC00B1FFDF06B02046BDE87040292124
:10576000FDF7D8BC06B0BDE8704003F0BEBE012115
:1057700001726868C6883046FDF765FE040000D1F6
:10578000FFDFA07F00F00301022902D120F010000A
:10579000A077207821280AD06868017A09B10079B9
:1057A00080B1A07F00F00300022862D0FFDFA07F5D
:1057B00000F003000228ABD1FEF790F80028A7D034
:1057C000FFDFA5E703F091FEA17F08062BD5E07F60
:1057D000C00705D094F8200000F01F00102820D04A
:1057E0005FF0050084F82300207829281DD02428A4
:1057F000DDD13146042010F09BFC22212046FDF72C
:1058000089FCA07F00F00300022830D05FF0000088
:1058100080F0010130460CF07BFF0028C7D0FFDF8D
:10582000C5E70620DEE70420DCE701F003000228DC
:1058300008D0002080F0010130460CF057FF050031
:1058400003D101E00120F5E7FFDF25212046FDF728
:1058500061FC03208DF80000694605F1E0000EF0C0
:105860001AFC0228A3D00028A1D0FFDF9FE7012067
:10587000CEE703F03AFE9AE72DE9F04387B0994668
:10588000164688460746FDF7DEFD04004BD020781B
:10589000222848D3232846D0E07F000743D4A07FA6
:1058A00000F00300022809D05FF0000080F0010141
:1058B00038460CF01BFF050002D00CE00120F5E794
:1058C000A07F00F00300022805D001210022384605
:1058D0000CF003FF05466946284601F01CF90098C4
:1058E00000B9FFDF45B10098E03505612078222836
:1058F00006D0242804D007E000990020086103E0C6
:1059000025212046FDF706FC0098012141704762E1
:10591000868001A9C0E902890EF0D8FB022802D0D6
:10592000002800D0FFDF07B0BDE8F08370B586B077
:105930000546FDF788FD017822291ED9807F00F0F9
:105940000300022808D0002080F0010128460CF056
:10595000CDFE04002FD101E00120F5E7FFDF2AE0B2
:10596000B4F85E0004F1620630440178427829B14F
:1059700021462846FFF714FCB0B9C9E6ADF804206B
:105980000921284602AB04F016FC03900028F4D04D
:1059900005208DF80000694604F1E0000EF07BFB65
:1059A000022801D000B1FFDF02231022314604F1AA
:1059B0005E000CF058FDB4F860000028D0D1A7E6D6
:1059C00010B586B00446FDF73EFD017822291BD9AB
:1059D000807F00F00300022808D0002080F0010141
:1059E00020460CF083FE040003D101E00120F5E71E
:1059F000FFDF06208DF80000694604F1E0000EF09C
:105A00004AFB002800D0FFDF06B010BD2DE9F05F93
:105A100005460C4600270078904601093E4604F1F1
:105A2000080BBA4602297DD0072902D00A2909D1DC
:105A300046E0686801780A2905D00D2930D00E2982
:105A40002ED0FFDFBBE114271C26002C6BD08088F2
:105A5000A080FDF7F8FC5FEA000900D1FFDF99F8AC
:105A600017005A46400809F11801FDF7BCFC6868A8
:105A7000C0892082696851F8060FC4F8120048688E
:105A8000C4F81600A07E20F0060001E02C020020E1
:105A900040F00100A07699F81E0040F020014DE092
:105AA0001A270A26002CD1D0C088A080FDF7CBFC95
:105AB000050000D1FFDF59462846FFF742FB7EE193
:105AC0000CB1A88BA080287A0B287DD006DC012899
:105AD0007BD0022808D0032804D135E00D2875D0EA
:105AE0000E2874D0FFDF6AE11E270926002CADD0F6
:105AF000A088FDF7A8FC5FEA000900D1FFDF287B42
:105B000000F003000128207A1BD020F00100207251
:105B1000297B890861F341002072297BC90861F360
:105B2000820001E041E1F2E02072297B090961F382
:105B3000C300207299F81E0040F0400189F81E1041
:105B40003DE140F00100E2E713270D26002CAAD02A
:105B5000A088FDF778FC8146807F00F003000228D2
:105B600008D0002080F00101A0880CF0BFFD0500E6
:105B700003D101E00120F5E7FFDF99F81E0000F0F6
:105B80000302022A50D0686F817801F003010129D5
:105B9000217A4BD021F00101217283789B0863F3B5
:105BA000410121728378DB0863F3820121728378DB
:105BB0001B0963F3C3012172037863F30611217299
:105BC000437863F3C71103E061E0A9E090E0A1E04E
:105BD000217284F809A0C178A172022A29D0027921
:105BE000E17A62F30001E1720279520862F3410145
:105BF000E1720279920862F38201E1720279D208BD
:105C000062F3C301E1724279217B62F300012173E7
:105C10004279520862F3410121734279920862F39A
:105C200082012173407928E0A86FADE741F00101BE
:105C3000B2E74279E17A62F30001E17242795208F7
:105C400062F34101E1724279920862F38201E172EA
:105C50004279D20862F3C301E1720279217B62F3D7
:105C6000000121730279520862F341012173027924
:105C7000920862F3820121730079C00860F3C301C6
:105C8000217399F80000232831D9262140E01827F4
:105C90001026E4B3A088FDF7D6FB8346807F00F092
:105CA0000300022809D0002080F00101A0880CF038
:105CB0001DFD5FEA000903D101E00120F4E7FFDFE9
:105CC000E868A06099F8000040F0040189F800102D
:105CD00099F80100800708D5012020739BF8000087
:105CE00023286CD92721584651E084F80CA066E09F
:105CF00015270F265CB1A088FDF7A5FB814606227B
:105D00005946E86808F097FA0120A073A0E041E046
:105D100048463CE016270926E4B3287B20724EE073
:105D2000287B19270E26ACB3C4F808A0A4F80CA051
:105D3000012807D0022805D0032805D0042803D065
:105D4000FFDF0DE0207207E0697B042801F00F01FE
:105D500041F0800121721ED0607A20F00300607251
:105D6000A088FDF770FB05460078212827D023285E
:105D700000D0FFDFA87F00F00300022813D000202E
:105D800080F00101A0880CF0C3FC22212846FDF719
:105D9000C1F914E004E0607A20F00300401CDEE763
:105DA000A8F8006010E00120EAE70CB16888A08044
:105DB000287A68B301280AD002284FD0FFDFA8F85C
:105DC00000600CB1278066800020BDE8F09F152799
:105DD0000F26002CE4D0A088FDF735FB807F00F073
:105DE0000300022808D0002080F00101A0880CF0F8
:105DF0007DFC050003D101E00120F5E7FFDFD5F8C8
:105E00001D000622594608F016FA84F80EA0D6E7BF
:105E100017270926002CC3D0A088FDF714FB814664
:105E2000807F00F00300022808D0002080F00101EC
:105E3000A0880CF05BFC050003D101E00120F5E730
:105E4000FFDF6878800701D5022000E00120207282
:105E500099F800002328B2D9272159E719270E26DF
:105E6000002C9DD0A088FDF7EEFA5FEA000900D172
:105E7000FFDFC4F808A0A4F80CA084F808A0A07A5A
:105E800040F00300A07299F81E10C90961F3820066
:105E9000A07299F81F2099F81E1012EAD11F05D0A0
:105EA00099F8201001F01F0110292BD020F00800D4
:105EB000A07299F81F10607A61F3C3006072697A6A
:105EC00001F003010129A2D140F00400607299F8A9
:105ED0001E0000F003000228E87A16D0217B60F350
:105EE00000012173AA7A607B62F300006073EA7A92
:105EF000520862F341012173A97A490861F3410014
:105F000060735CE740F00800D2E7617B60F300015A
:105F10006173AA7A207B62F300002073EA7A520848
:105F200062F341016173A97A490861F3410020736A
:105F300045E710B5FE4C30B10146102204F12000B7
:105F40001EF0D0FC012084F8300010BD10B50446CE
:105F500000F0D1FDF64920461022BDE81040203166
:105F60001EF0C0BC70B5F24D06004FF0000413D017
:105F7000FBF7A9F908B110240CE00621304608F01F
:105F800041F9411C05D028665FF0010085F85C00EE
:105F900000E00724204670BD0020F7E7007810F0ED
:105FA0000F0204D0012A05D0022A0CD110E000090A
:105FB00009D10AE00009012807D0022805D00328EA
:105FC00003D0042801D007207047087000207047D4
:105FD0000620704705282AD2DFE800F003070F17D4
:105FE0001F00087820F0FF001EE0087820F00F0066
:105FF000401C20F0F000103016E0087820F00F0070
:10600000401C20F0F00020300EE0087820F00F0057
:10601000401C20F0F000303006E0087820F00F003F
:10602000401C20F0F000403008700020704707202E
:1060300070472DE9F041804688B00D46002708469C
:10604000FBF78EF9A8B94046FDF7FDF9040003D02F
:106050002078222815D104E043F2020008B0BDE800
:10606000F08145B9A07F410603D500F00300022866
:1060700001D01020F2E7A07FC10601D4010702D5AC
:106080000DB10820EAE7E17F090701D50D20E5E71A
:1060900000F00300022805D125B12846FEF762FF73
:1060A0000700DBD1A07F00F00300022808D0002009
:1060B00080F0010140460CF019FB060002D00FE011
:1060C0000120F5E7A07F00F0030002280ED0002099
:1060D00080F00101002240460CF0FFFA060007D0D4
:1060E000A07F00F00300022804D009E00120EFE7C0
:1060F0000420B3E725B12A4631462046FEF756FF75
:106100006946304600F007FD009800B9FFDF0099AE
:10611000022006F1E0024870C1F824804A610022A2
:106120000A81A27F02F00302022A1CD0012008711A
:10613000287800F00102087E62F3010008762A78D0
:10614000520862F3820008762A78920862F3C3004C
:1061500008762A78D20862F30410087624212046B3
:10616000FCF7D8FF33E035B30871301D8861307813
:10617000400908777078C0F340004877287800F02D
:106180000102887F62F301008877A27FD20962F35F
:1061900082008877E27F62F3C3008877727862F3C7
:1061A00004108877A878C87701F1210228462031A9
:1061B000FEF71DFF03E00320087105200876252166
:1061C0002046FCF7A7FFA07F20F04000A07701A9A0
:1061D00000980DF07BFF022801D000B1FFDF3846A8
:1061E0003CE72DE9FF4F534A0D4699B09A4607CA3E
:1061F0000AAB002783E807001998FDF724F9060089
:1062000006D03078262806D008201DB0BDE8F08FD3
:1062100043F20200F9E7B07F00F00309B9F1020F81
:106220000AD05DB91B98FEF79DFE0028EDD1B07F26
:1062300000F00300022801D11B9890BBB07F00F052
:106240000300022808D0002080F0010119980CF00A
:106250004DFA040003D101E00120F5E7FFDF852DB1
:1062600028D007DCF5B1812D1ED0822D1ED0832DC4
:1062700008D11DE0862D1FD0882D1FD0892D1FD05D
:106280008A2D1FD00F2020710F281DD003F02AF96E
:10629000E0B101208DF83C00201D10902079B8B1AC
:1062A0005BE111E00020EEE70120ECE70220EAE7E5
:1062B0000320E8E70520E6E70620E4E70820E2E718
:1062C0000920E0E70A20DEE707209EE711209CE78F
:1062D000B9F1020F03D0A56F03D1A06F02E0656F83
:1062E000FAE7606F804632D04FF0010001904FF026
:1062F00002000090214630461B9AFEF757FE1B987D
:10630000007800F00101A87861F30100A870B17F66
:10631000C90961F38200A870F17F61F3C300A8701E
:10632000617861F30410A87020784009287003E0B8
:106330002C020020D44D02006078C0F34000687049
:106340001B988078E87000206871287103E00220B3
:10635000019001200090A87898F80210C0F3C000C6
:10636000C1F3C00108405FEA000B2DD05046FAF798
:10637000AAFF78BBDAF80C00FAF7A5FF50BBDAF8F1
:106380001C00FAF7A0FF28BBDAF80C00A060DAF8CE
:106390001C00E060607898F8012042EA500100BFDC
:1063A00061F34100607098F80210C0B200EA111168
:1063B00061F30000607000202077009906F117005B
:1063C000022908D0012107E0607898F8012002EA4C
:1063D0005001E5E732E0002104EB810148610199B9
:1063E000701C022901D0012100E0002104EB810191
:1063F0004861A87800F00300012857D198F80200FE
:1064000000F00300012851D1B9F1020F04D02A1D78
:10641000691D1B98FEF7EBFD287998F804100840D9
:106420008DF83400697998F8052011408DF83810FE
:1064300008433BD05046FAF746FF08B11020E4E687
:106440000AF110010491B9F1020F17D0084600219A
:1064500004F18C03CDE9000304F5AE7202920DAB9A
:106460005A462046FEF70CFE0028E8D1B9F1020F8B
:1064700008D0504608D14FF0010107E050464FF0D8
:106480000101E5E70498F5E74FF0000104F1A403EA
:10649000CDE9000304F5B072029281F001010EAB68
:1064A0005A462046FEF7ECFD0028C8D160788007E8
:1064B00034D4A87898F80210C0F38000C1F38001AA
:1064C00008432BD0297898F800000AAAB9F1020FE6
:1064D00006D032F811204300DA4002F003070AE048
:1064E00032F810204B00DA4012F0030705D0012FDC
:1064F0000BD0022F0BD0032F07D0BBF1000F0DD014
:10650000012906D0042904D008E00227F5E7012775
:10651000F3E7012801D0042800D10427B07F40F020
:106520008000B077F17F6BF30001F177607880072E
:1065300006D50320A071BBF1000F0ED1002028E08A
:106540000220022F18D0012F18D0042F29D00020AC
:10655000A071B07F20F08000B07725213046FCF795
:10656000D9FD0FA904F1E0000DF095FD10B102284E
:1065700000D0FFDF002048E6A071DFE7A0710D2109
:1065800004F120001EF04FFA207840F00200207045
:1065900001208DF85C0017AA3146199800F094FA92
:1065A000DBE70120A071D8E72DE9F04387B09046E2
:1065B000894604460025FCF746FF060006D03078E1
:1065C000272806D0082007B0BDE8F08343F2020078
:1065D000F9E7B07F00F00300022809D05FF0000067
:1065E00080F0010120460CF081F8040003D101E0A5
:1065F0000120F5E7FFDFA7795FEA090005D0012850
:1066000021D0B9F1020F26D110E0B8F1000F22D14C
:10661000012F05D0022F05D0032F05D0FFDF2DE07D
:106620000C252BE0012529E0022527E04046FAF75A
:106630004AFEB0B9032F0ED11022414604F11D00CD
:106640001EF050F91AE0012F02D0022F03D104E00E
:10665000B8F1000F12D00720B5E74046FAF733FE35
:1066600008B11020AFE7102104F11D001EF0B9F9A8
:106670000621404607F0C6FDC4F81D0020782521FC
:1066800040F0020020703046FCF744FD2078C1073E
:1066900013D020F00100207002208DF8000004F1DA
:1066A0001D0002908DF804506946C3300DF0F3FCD4
:1066B000022803D010B1FFDF00E02577002082E739
:1066C00030B587B00D460446FCF7BDFEA0B1807F13
:1066D00000F00300022812D05FF0000080F00101FA
:1066E00020460CF003F804000ED02846FAF7EBFD24
:1066F00038B1102007B030BD43F20200FAE70120A4
:10670000ECE72078400701D40820F3E7294604F19C
:106710003D00202205461EF0E5F8207840F01000EC
:10672000207001070FD520F00800207007208DF899
:106730000000694604F1E00001950DF0ACFC022870
:1067400001D000B1FFDF0020D4E770B50D4606464A
:10675000FCF779FE18B10178272921D102E043F234
:10676000020070BD807F00F00300022808D00020E6
:1067700080F0010130460BF0B9FF040003D101E0C5
:106780000120F5E7FFDFA079022809D16078C00772
:1067900006D02A4621463046FEF702FD10B10FE032
:1067A000082070BDB4F860000E280BD204F162011D
:1067B00002231022081F0BF020FE012101704570FA
:1067C000002070BD112070BD70B5064614460D4600
:1067D0000846FAF778FD18B92046FAF79AFD08B18D
:1067E000102070BDA6F57F40FF380ED03046FCF774
:1067F0002AFE38B1417822464B08811C1846FCF726
:10680000F2FD07E043F2020070BD2046FDF7F8FDFF
:106810000028F9D11021E01D0FF0ABF9E21D294647
:1068200004F1170000F087F9002070BD2DE9F04158
:1068300004468AB01546884600270846FAF790FDB8
:1068400018B92846FAF78CFD10B110200AB006E4FA
:106850002046FCF7F8FD060003D0307827281AD12F
:1068600002E043F20200F1E7B07F00F003000228EB
:1068700008D0002080F0010120460BF037FF040013
:1068800003D101E00120F5E7FFDF2078400702D5C2
:106890006078800701D40820D8E7B07F00F00300BB
:1068A000022803D0A06F03D1A16F02E0606FFAE766
:1068B000616F407800B19DB1487810B1B8F1000F18
:1068C0000ED0ADB1EA1D06A8E16800F034F910223F
:1068D00006A905F117001DF0D9FF18B1042707E03C
:1068E0000720B3E71022E91D04F12D001DF0FAFF87
:1068F000B8F1000F06D0102208F1070104F11D00C5
:106900001DF0F0FF2078252140F002002070304675
:10691000FCF700FC2078C10715D020F001002070A2
:1069200002208DF8000004F11D0002901030039049
:106930008DF804706946B3300DF0ADFB022803D02A
:1069400010B1FFDF00E0277700207FE7F8B515469C
:106950000E460746FCF777FD040004D02078222875
:1069600004D00820F8BD43F20200F8BDA07F00F07B
:106970000300022802D043F20500F8BD3046FAF7C2
:10698000A2FC18B92846FAF79EFC08B11020F8BD01
:1069900000953288B31C21463846FEF724FC1128A6
:1069A00015D00028F3D1297C4A08A17F62F3C711D2
:1069B000A177297CE27F61F30002E277297C8908D4
:1069C00084F82010A17F21F04001A177F8BDA17FBC
:1069D0000907FBD4D6F80200C4F83600D6F8060042
:1069E000C4F83A003088A0861022294604F1240019
:1069F0001DF078FF287C4108E07F61F34100E077DB
:106A0000297C61F38200E077287C800884F82100EB
:106A1000A07F40F00800A0770020D3E770B50D46B6
:106A200006460BB1072070BDFCF70DFD040007D032
:106A30002078222802D3A07F800604D4082070BDCD
:106A400043F2020070BDADB1294630460AF0C4FDE4
:106A500002F05EFB297C4A08A17F62F3C711A1778F
:106A6000297CE27F61F30002E277297C890884F8BF
:106A7000201004E030460AF0D2FD02F049FBA17F6D
:106A800021F02001A17770BD70B50D46FCF7DBFC4D
:106A9000040005D02846FAF73CFC20B1102070BD58
:106AA00043F2020070BD29462046FEF74AFB002053
:106AB00070BD04E010F8012B0AB100207047491E98
:106AC00089B2F7D20120704770B51546064602F02C
:106AD00009FD040000D1FFDF207820F00F00801CAA
:106AE00020F0F0002030207066802868A060BDE8AB
:106AF000704002F0FABC10B5134C94F83000002836
:106B000008D104F12001A1F110000DF006FB0120D5
:106B100084F8300010BD10B190F8B9202AB10A48AD
:106B200090F8350018B1002003E0B83001E00648C5
:106B300034300860704708B50023009313460A46B6
:106B40000BF0CFFF08BD00002C02002018B18178A7
:106B5000012938D101E010207047018842F6011266
:106B6000881A914231D018DC42F60102A1EB0200F2
:106B700091422AD00CDC41B3B1F5C05F25D06FF44F
:106B8000C050081821D0A0F57060FF381BD11CE060
:106B900001281AD002280AD117E0B0F5807F14D05E
:106BA00008DC012811D002280FD003280DD0FF28BF
:106BB00009D10AE0B0F5817F07D0A0F580700338D5
:106BC00003D0012801D0002070470F2070470A2809
:106BD0001FD008DC0A2818D2DFE800F0191B1F1F9D
:106BE000171F231D1F21102815D008DC0B2812D0D9
:106BF0000C2810D00D2816D00F2806D10DE0112832
:106C00000BD084280BD087280FD00320704700209A
:106C1000704705207047072070470F2070470420F9
:106C20007047062070470C20704743F202007047FF
:106C300038B50C46050041D06946FFF7AFF900288A
:106C400019D19DF80010607861F302006070694608
:106C5000681CFFF7A3F900280DD19DF8001060789B
:106C600061F3C5006070A978C1F34101012903D027
:106C7000022905D0072038BD217821F0200102E04B
:106C8000217841F020012170410704D0A978C9087A
:106C900061F386106070607810F0380F07D0A97823
:106CA000090961F3C710607010F0380F02D16078E5
:106CB000400603D5207840F040002070002038BD09
:106CC00070B504460020088015466068FFF7B0FFE5
:106CD000002816D12089A189884211D8606880785F
:106CE000C0070AD0B1F5007F0AD840F20120B1FBFD
:106CF000F0F200FB1210288007E0B1F5FF7F01D908
:106D00000C2070BD01F201212980002070BD10B55A
:106D10000478137864F3000313700478640864F350
:106D2000410313700478A40864F382031370047899
:106D3000E40864F3C30313700478240964F30413B0
:106D400013700478640964F34513137000788009A4
:106D500060F38613137031B10878C10701D1800741
:106D600001D5012000E0002060F3C713137010BDAF
:106D70004278530702D002F0070306E012F0380F02
:106D800002D0C2F3C20300E001234A7863F3020297
:106D90004A70407810F0380F02D0C0F3C20005E00E
:106DA000430702D000F0070000E0012060F3C502B5
:106DB0004A7070472DE9F04F95B00D00824612D011
:106DC000122128461DF00DFE4FF6FF7B05AA01217A
:106DD000584607F03EF80024264637464FF4205820
:106DE0006FF4205973E0102015B0BDE8F08F00BF9C
:106DF0009DF81E0001280AD1BDF81C1041450BD09A
:106E000011EB09000AD001280CD002280CD0042C68
:106E10000ED0052C0FD10DE0012400E00224BDF8B6
:106E20001A6008E0032406E00424BDF81A7002E0AA
:106E3000052400E00624BDF81A10514547D12C74F2
:106E4000BEB34FF0000810AA4FF0070ACDE9028246
:106E5000CDE900A80DF13C091023CDF81090424671
:106E60003146584607F0A8F808BBBDF83C002A4652
:106E7000C0B210A90DF0C7F9C8B9AE81CFB1CDE944
:106E800000A80DF1080C0AAE40468CE8410213231D
:106E900000223946584607F08FF840B9BDF83C004B
:106EA000F11CC01EC0B22A1D0DF0ADF910B10320B7
:106EB0009AE70AE0BDF82900E881062C05D19DF883
:106EC0001E00A872BDF81C00288100208CE705A8D0
:106ED00006F0CBFF00288BD0FFF779FE84E72DE981
:106EE000F0471C46DDE90978DDF8209015460E00D4
:106EF000824600D1FFDF0CB1208818B1D5B1112036
:106F0000BDE8F087022D01D0012100E0002106F14B
:106F1000140005F08DFEA8F8000002463B46294605
:106F2000504603F048F9C9F8000008B9A41C3C60B9
:106F30000020E5E71320E3E7F0B41446DDE904524E
:106F40008DB1002314B1022C09D101E0012306E028
:106F50000D7CEE0703D025F0010501230D742146B9
:106F6000F0BC03F0B3BF1A80F0BC70472DE9FE4FB0
:106F700091461A881C468A468046FAB102AB4946B9
:106F800003F019F9050019D04046A61C27880BF01C
:106F9000F1FC3246072629463B4600960BF0FFF8E7
:106FA00020882346CDE900504A4651464046FFF727
:106FB000C3FF002020800120BDE8FE8F0020FBE7FA
:106FC0002DE9F04786B082460EA8904690E8B000C2
:106FD000894604AA05A903A88DE807001E462A468B
:106FE00021465046FFF77BFF039901B1012139701B
:106FF000002818D1F94904F1140204AB0860039881
:1070000005998DE8070042464946504606F0C7F903
:10701000A8B1092811D2DFE800F005080510100A10
:107020000C0C0E00002006B06AE71120FBE70720D9
:10703000F9E70820F7E70D20F5E70320F3E7BDF8AF
:1070400010100398CDE9000133462A4621465046E8
:10705000FFF772FFE6E72DE9F04389B00D46DDE961
:10706000108781461C461646142103A81DF0DBFC40
:10707000012002218DF810108DF80C008DF8117090
:10708000ADF8146064B1A278D20709D08DF816006B
:10709000E088ADF81A00A088ADF81800A068079045
:1070A00008A80095CDE90110424603A948466B683F
:1070B000FFF786FF09B0BDE8F083F0B58BB0002480
:1070C0000646069407940727089405A80994019496
:1070D00000970294CDE903400D4610232246304626
:1070E00006F06AFF78B90AA806A9019400970294ED
:1070F000CDE90310BDF8143000222946304606F0D1
:1071000031FD002801D0FFF762FD0BB0F0BD06F0A5
:10711000D1BB2DE9FC410C468046002602F0E2F985
:10712000054620780D287DD2DFE800F0BC0713B3B8
:1071300025BD49496383AF959B00A848006820B1ED
:10714000417841F010014170ADE0404602F0FAF99B
:10715000A9E0042140460BF0C9FA070000D1FFDF87
:1071600007F11401404605F0F7FCA5BB132140468A
:10717000FDF720FC97E0042140460BF0B7FA07002A
:1071800000D1FFDFE088ADF800000020B8819DF855
:107190000000010704D5C00602D5A088B88105E02B
:1071A0009DF8010040067ED5A088F88105B9FFDF73
:1071B00022462946404601F0BDFC022673E0E188E4
:1071C000ADF800109DF8011009060FD5072803D06F
:1071D00006280AD00AE024E0042140460BF086FA93
:1071E000060000D1FFDFA088F0810226CDB9FFDFC5
:1071F00017E0042140460BF079FA070000D1FFDFC9
:1072000007F1140006F08DFB90F0010F02D1E07938
:10721000000648D5387C022640F00200387405B9D3
:10722000FFDF00E03EE022462946404601F082FCB6
:1072300039E0042140460BF059FA017C002D01F0A1
:107240000206C1F340016171017C21F00201017469
:10725000E7D1FFDFE5E702260121404602F0A4F96D
:1072600021E0042140460BF041FA05466068009099
:107270002089ADF8040001226946404602F0B5F9C4
:10728000287C20F0020028740DE0002DC9D1FFDF1A
:10729000C7E7022600214046FBF716F9002DC0D1B2
:1072A000FFDFBEE7FFDF3046BDE8FC813EB50C00E6
:1072B00009D001466B4601AA002006F0FFFE20B16E
:1072C000FFF785FC3EBD10203EBD00202080A07051
:1072D0009DF8050002A900F00700FEF77BFE50B9FB
:1072E0009DF8080020709DF8050002A9C0F3C200B7
:1072F000FEF770FE08B103203EBD9DF808006070E7
:107300009DF80500C109A07861F30410A0709DF8F4
:107310000510890961F3C300A0709DF80410890667
:1073200001D5022100E0012161F342009DF8001027
:1073300061F30000A07000203EBD70B51446064603
:107340000D4651EA040005D075B10846F9F7FFFF74
:1073500078B901E0072070BD2946304606F00FFFDE
:1073600010B1BDE8704032E454B12046F9F7EFFFA8
:1073700008B1102070BD21463046BDE8704095E749
:10738000002070BD2DE9FC5F0C46904605460027A5
:1073900001780822007A3E46B2EB111F7ED104F13B
:1073A0000A0100910A31821E4FF0020A04F1080B13
:1073B0000191092A73D2DFE802F0ECDF05F42727F8
:1073C0007AA9CD00688804210BF090F9060000D15D
:1073D000FFDFB08920B152270726C2E090020020CB
:1073E00051271026002C7DD06888A0800120A07134
:1073F000A88900220099FFF7A0FF002873D1A8896F
:107400002081288AE081D1E0B5F81290072824D1A4
:10741000E87B000621D5512709F1140086B2002C23
:10742000E1D0A88900220099FFF787FF00285AD1F0
:107430006888A08084F806A0A88920810120A07314
:10744000288A2082A4F81290A88A009068884B4667
:10745000A969019A01F04BFBA8E0502709F112003D
:1074600086B2002C3ED0A88900225946FFF765FF5E
:10747000002838D16888A080A889E080287A072869
:1074800013D002202073288AE081E87BC009607352
:10749000A4F81090A88A0090688801E083E080E05A
:1074A0004B4604F11202A969D4E70120EAE7B5F8D6
:1074B0001290512709F1140086B2002C66D068881A
:1074C00004210BF013F983466888A080A889002264
:1074D0000099FFF732FF00286ED184F806A0A88932
:1074E000208101E052E067E00420A073288A208216
:1074F000A4F81290A88A009068884B46A969019A5E
:1075000001F0F5FAA989ABF80E104FE06888FBF797
:107510009AFF0746688804210BF0E8F8064607B989
:10752000FFDF06B9FFDF687BC00702D051271426B2
:1075300001E0502712264CB36888A080502F06D057
:1075400084F806A0287B594601F0E1FA2EE0287B5A
:10755000A11DF9E7FE49A8894989814205D154272F
:1075600006269CB16888A08020E053270BE068883D
:10757000A080A889E08019E0688804210BF0B6F8A3
:1075800000B9FFDF55270826002CF0D1A8F80060CD
:1075900011E056270726002CF8D06888A08000202C
:1075A00013E0FFDF02E0012808D0FFDFA8F8006049
:1075B0000CB1278066800020BDE8FC9F5727072676
:1075C000002CE3D06888A080687AA071EEE7401DA7
:1075D00020F0030009B14143091D01EB4000704751
:1075E00013B5DB4A00201071009848B100246846AA
:1075F0000AF099FE002C02D1D64A009911601CBDF8
:1076000001240020F4E770B50D46064686B0144606
:107610005C2128461DF007FA04B9FFDFA0786874E2
:10762000A2782188284601F09CFA0020A881E881F0
:10763000228805F11401304605F073FA6A460121EB
:10764000304606F006FC19E09DF80300000715D54A
:10765000BDF806103046FFF730FD9DF80300BDF879
:10766000061040F010008DF80300BDF80300ADF8DF
:107670001400FF233046059A06F04CFD684606F0DC
:10768000F4FB0028E0D006B070BD10B50C4601F147
:10769000140005F07DFA0146627C2046BDE81040EA
:1076A00001F094BA30B50446A94891B04FF6FF7581
:1076B000C18905AA284606F0CCFB30E09DF81E00E3
:1076C000A0422AD001282AD1BDF81C00B0F5205FC5
:1076D00003D042F60101884221D1002002AB0AAA60
:1076E0000CA9019083E8070007200090BDF81A104C
:1076F00010230022284606F05FFC38B9BDF82800A8
:107700000BAAC0B20CA90CF07EFD10B1032011B081
:1077100030BD9DF82E00A04201D10020F7E705A85A
:1077200006F0A3FB0028C9D00520F0E770B5054698
:1077300004210AF0DBFF040000D1FFDF04F1140193
:107740000C46284605F008FA21462846BDE8704058
:1077500005F009BA70B58AB00C460646FBF773FE11
:10776000050014D02878222827D30CB1A08890B126
:1077700001208DF80C0003208DF8100000208DF8FA
:10778000110054B1A088ADF81800206807E043F25A
:1077900002000AB070BD0920FBE7ADF818000590A3
:1077A000042130460AF0A2FF040000D1FFDF04F1FB
:1077B000140005F004FA000701D40820E9E701F0FD
:1077C00091FE60B108A802210094CDE9011095F85E
:1077D000232003A930466368FFF7F2FBD9E71120A5
:1077E000D7E72DE9F04FB2F802A0834689B01546DD
:1077F00089465046FBF727FE0746042150460AF00B
:1078000075FF0026044605964FF002080696ADF86F
:107810001C6007B9FFDF04B9FFDF4146504603F0A3
:10782000C0FE50B907AA06A905A88DE80700424680
:10783000214650466368FFF752FB454807AB066098
:10784000DDE9051204F11400CDF80090CDE9032024
:10785000CDE9013197F82320594650466B6805F071
:10786000F7F906000AD0022E04D0032E14D0042EFD
:1078700000D0FFDF09B03046BDE8F08FBDF81C0036
:107880000028F7D00599CDE9001042462146504620
:107890006368FFF751FBEDE7687840F00800687017
:1078A000E8E72DE9F04F99B004464FF0000828486A
:1078B000ADF81C80ADF82080ADF82480A0F80880D9
:1078C000ADF81480ADF81880ADF82C80ADF82880A4
:1078D000007916460D464746012808D0022806D0F2
:1078E000032804D0042802D0082019B0C4E7204699
:1078F000F9F7E9FC80BB2846F9F7E5FC60BB606856
:10790000F9F72EFD40BB606848B160892189884243
:1079100002D8B1F5007F01D90C20E6E780460EAA17
:1079200006A92846FFF7CCF90028DED168688078E0
:10793000C0F34100022808D19DF8190010F0380F5B
:1079400003D02869F9F703FD30B905A9206904E0DF
:10795000900200201400002020E0FFF769F90028C1
:10796000C3D1206948B1607880079DF8150000F008
:10797000380001D5F0B300E0E0BB9DF814008006AC
:107980000ED59DF8150010F0380F03D06068F9F798
:10799000DEFC18B96068F9F7E3FC08B11020A4E731
:1079A0000AA96069FFF744F900289ED1606940B1D7
:1079B0009DF8290000F0070101293CD110F0380F93
:1079C00039D00BA9A069FFF733F900288DD19DF8B4
:1079D000280080062FD49DF82C0080062BD4A069A7
:1079E00050B19DF82D0000F00701012923D110F0BE
:1079F000380F00E01FE01ED0E06818B10078D0B169
:107A00001C2818D20FAA611C2046FFF780F901211B
:107A1000384661F30F2082468DF85210B94642F67F
:107A200003000F46ADF850000DF13F0218A9286879
:107A30000CF008FC08B1072057E79DF8600015A975
:107A4000CDF80090C01CCDE9019100F0FF0B0023A0
:107A50000BF20122514614A806F03EF9F0BBBDF826
:107A600054000C90FD492A8928690092CDE9010152
:107A70006B89BDF838202868069906F02DF90100B9
:107A80007ED120784FF0020AC10601D480062BD5A2
:107A9000ADF80C90606950B90AA906A8FFF768F91B
:107AA0009DF8290020F00700401C8DF829009DF862
:107AB000280008A940F0C8008DF828008DF8527001
:107AC00042F60210ADF8500003AACDF800A0CDE9AF
:107AD0000121002340F2032214A800E01EE00A99CD
:107AE00006F0FAF801004BD1DC484D4608385B46F9
:107AF0000089ADF83D000FA8CDE90290CDF80490C3
:107B0000CDF810904FF007090022CDF80090BDF895
:107B100054104FF6FF7006F025F810B1FFF757F834
:107B2000E3E69DF83C00000625D52946012060F3D8
:107B30000F218DF852704FF42450ADF85000ADF87D
:107B40000C5062789DF80C00002362F300008DF861
:107B50000C006278CDF800A0520862F341008DF865
:107B60000C0003AACDE9012540F2032214A806F077
:107B7000B3F8010004D1606888B32069A8B900E0B7
:107B800086E005A906A8FFF7F3F86078800706D419
:107B90009DF8150020F038008DF8150005E09DF8DF
:107BA000140040F040008DF814008DF8527042F639
:107BB0000110ADF85000208940F20121B0FBF1F234
:107BC00001FB1202606809ABCDF80080CDE901032A
:107BD000002314A8059906F07FF8010058D12078F9
:107BE000C00729D0ADF80C50A06950B90BA906A860
:107BF000FFF7BEF89DF82D0020F00700401C8DF81F
:107C00002D009DF82C008DF8527040F040008DF84A
:107C10002C0042F60310ADF8500007A903AACDF8D6
:107C200000A0CDE90121002340F2032214A80B9902
:107C300006F052F801002BD1E06868B32946012014
:107C400060F30F218DF8527042F60410ADF8500029
:107C5000E068002302788DF8582040788DF85900AC
:107C6000E06816AA4088ADF85A00E06800798DF8FF
:107C70005C00E068C088ADF85D00CDF80090CDE90B
:107C800001254FF4027214A806F026F8010003D073
:107C90000C9800F0C7FF28E67048032108380171EE
:107CA00056B100893080BDF824007080BDF82000F6
:107CB000B080BDF81C00F080002016E670B50125EC
:107CC0008AB016460B46012802D0022816D104E0DD
:107CD0008DF80E504FF4205003E08DF80E5042F610
:107CE0000100ADF80C005BB10024601C60F30F24B0
:107CF00004AA08A918460CF0A5FA18B1072048E50F
:107D0000102046E504A99DF820205448CDE9002123
:107D1000801E02900023214603A802F2012205F0F2
:107D2000DBFF10B1FEF753FF33E54C4808380EB1C6
:107D3000C1883180057100202BE5F0B593B007466E
:107D400001268DF83E6041F60100ADF83C0012AA14
:107D50000FA93046FFF7B2FF002848D13F4C00255D
:107D6000083CE7B31C2102A81CF05DFE9DF808004A
:107D70008DF83E6040F020008DF8080042F60520A6
:107D8000ADF83C000E959DF83A00119520F00600E4
:107D9000801C8DF83A009DF838006A4620F0FF00FC
:107DA0008DF838009DF8390009A920F0FF008DF802
:107DB00039000420ADF82C00ADF830000EA80A9070
:107DC00011A80D900FA80990ADF82E5002A8FFF74A
:107DD00068FD00280BD1BDF80000608100E008E0DC
:107DE000BDF80400A081401CE0812571002013B083
:107DF000F0BD6581A581BDF84800F4E72DE9F74F96
:107E00001649A0B00024083917940A79A146012A1E
:107E100004D0022A02D0082023B02DE5CA8882426D
:107E200001D00620F8E721988A46824201D1072036
:107E3000F2E701202146ADF848004FF6FF788DF8B3
:107E40006E0042F6020B60F30F21ADF84A80ADF8E8
:107E50006CB006918DF8724002E00000980200209C
:107E60001CA9ADF870401391ADF8508012A806F02F
:107E700020F800252E462F460DAB072212A94046BA
:107E800006F01AF878B10A285DD195B38EB3ADF833
:107E90006450ADF866609DF85E008DF8144019AC32
:107EA000012864D06BE09DF83A001FB3012859D136
:107EB000BDF8381059451FD118A809A9019402949A
:107EC000CDE9031007200090BDF8361010230022E2
:107ED000404606F071F8B0BBBDF86000042801D040
:107EE00006284AD1BDF82410219881423AD10F20AA
:107EF00092E73AE0012835D1BDF83800B0F5205FAF
:107F000003D042F6010188422CD1BAF80600BDF830
:107F10003610884201D1012700E0002705B19EB14B
:107F2000219881421ED118A809AA01940294CDE992
:107F30000320072000900D4610230022404606F043
:107F40003BF800B902E02DE04E460BE0BDF86000C2
:107F5000022801D0102810D1C0B217AA09A90CF02C
:107F600052F950B9BDF8369086E7052054E705A9C7
:107F700017A8221D0CF066F908B103204CE79DF804
:107F800014000023001DC2B28DF814202298009224
:107F9000CDE901401BA8069905F09EFE10B902220A
:107FA0008AF80420FEF713FE36E710B50B46401E94
:107FB00088B084B205AA00211846FEF7A8FE00206A
:107FC0000DF1080C06AA05A901908CE8070007200E
:107FD00000900123002221464FF6FF7005F0C2FDFC
:107FE0000446BDF81800012800D0FFDF2046FEF748
:107FF000EEFD08B010BDF0B5F74F044687B03879F4
:108000000E46032804D0042802D0082007B0F0BD93
:1080100004AA03A92046FEF753FE0500F6D16068C6
:108020008078C0F3410002280AD19DF80D0010F0BD
:10803000380F05D02069F9F78AF908B11020E5E773
:10804000208905AA21698DE807006389BDF8102001
:108050002068039905F040FE10B1FEF7B8FDD5E7A2
:1080600016B1BDF814003080042038712846CDE7E1
:10807000F8B50C0006460CD001464FF6FF750023FC
:108080006A46284606F01AF828B100BFFEF79FFDA1
:10809000F8BD1020F8BD69462046FEF7C9FD00284E
:1080A000F8D1A078314600F001032846009A06F086
:1080B00031F8EBE730B587B0144600220DF1080C1B
:1080C00005AD01928CE82C00072200920A46014679
:1080D00023884FF6FF7005F045FDBDF81410218090
:1080E000FEF775FD07B030BD70B50D4604210AF0EE
:1080F000FDFA040000D1FFDF294604F11400BDE8B9
:10810000704004F055BD70B50D4604210AF0EEFA3A
:10811000040000D1FFDF294604F11400BDE87040DF
:1081200004F069BD70B50D4604210AF0DFFA0400C1
:1081300000D1FFDF294604F11400BDE8704004F0CF
:1081400081BD70B5054604210AF0D0FA040000D1C3
:10815000FFDF214628462368BDE870400122FEF774
:1081600005BF70B5064604210AF0C0FA040000D12C
:10817000FFDF04F1140004F00BFD401D20F00305A7
:1081800011E0011D00880022431821463046FEF709
:10819000EDFE00280BD0607CABB2684382B2A068D1
:1081A000011D0AF060F9A06841880029E9D170BD7D
:1081B00070B5054604210AF099FA040000D1FFDFEA
:1081C000214628466368BDE870400222FEF7CEBE15
:1081D00070B50E46054601F085F9040000D1FFDFB9
:1081E0000120207266726580207820F00F00001D4B
:1081F00020F0F00040302070BDE8704001F075B90B
:1082000010B50446012900D0FFDF2046BDE810402C
:108210000121FAF759B92DE9F04F97B04FF0000A54
:108220000C008346ADF814A0D04619D0E06830B1F8
:10823000A068A8B10188ADF81410A0F800A05846B5
:10824000FBF701F9070043F2020961D038782228D0
:108250005CD3042158460AF049FA050005D103E031
:10826000102017B0BDE8F08FFFDF05F1140004F017
:108270008FFC401D20F00306A078012803D00228BF
:1082800001D00720EDE7218807AA584605F0E1FD57
:1082900030BB07A805F0E9FD10BB07A805F0E5FD18
:1082A00048B99DF82600012805D1BDF82400A0F5A5
:1082B0002451023902D04FF45050D2E7E068B0B1F7
:1082C000CDE902A00720009005AACDF804A00492F1
:1082D000A2882188BDF81430584605F043FC10B13F
:1082E000FEF775FCBDE7A168BDF8140008809DF895
:1082F0001F00C00602D543F20140B2E70B9838B127
:10830000A1780078012905D080071AD40820A8E7B1
:108310004846A6E7C007F9D002208DF83C00A868BF
:108320004FF00009A0B1697C4288714391420FD996
:108330008AB2B3B2011D0AF04CF88046A0F800A042
:1083400006E003208DF83C00D5F800804FF00109CD
:108350009DF8200010F0380F00D1FFDF9DF82000BD
:108360001E49C0F3C200084497F8231010F8010C0E
:10837000884201D90F2074E72088ADF8400014A985
:108380000095CDE90191434607220FA95846FEF713
:1083900017FE002891D19DF8500050B9A07801280F
:1083A00007D1687CB3B2704382B2A868011D0AF09D
:1083B00024F8002055E770B5064615460C460846D9
:1083C000FEF7C4FB002805D12A4621463046BDE809
:1083D000704073E470BD11E590020020DE4D020094
:1083E00070B51E4614460D0009D044B1616831B124
:1083F00038B1FC49C988814203D0072070BD1020E4
:1084000070BD2068FEF7A2FB0028F9D13246214654
:108410002846BDE87040FFF744BA70B515460C0019
:1084200006D038B1EF490989814203D0072070BDD9
:10843000102070BD2068FEF789FB0028F9D129467D
:108440002046BDE87040D6E570B5064686B00D46BC
:1084500014461046F8F75DFFD0BB6068F8F780FF60
:10846000B0BBA6F57F40FF3803D03046FAF7EBFFEC
:1084700080B128466946FEF79DFC00280CD19DF886
:1084800010100F2008293DD2DFE801F0080606068B
:10849000060A0A0843F2020006B070BD0320FBE79B
:1084A0009DF80210012908D1BDF80010B1F5C05F98
:1084B000F2D06FF4C052D142EED09DF806100129DF
:1084C0000DD1BDF80410A1F52851062907D200E00E
:1084D00029E0DFE801F0030304030303DCE79DF870
:1084E0000A1001290FD1BDF80810B1F5245FD3D0CF
:1084F000A1F60211B1F50051CED00129CCD002294C
:1085000001D1C9E7FFDF606878B9002305AA2946D1
:10851000304605F0D3FD10B1FEF759FBBCE79DF8DE
:108520001400800601D41020B6E761882246284650
:108530006368FFF7BFFDAFE72DE9F043814687B0E1
:10854000884614461046F8F7E4FE18B1102007B02C
:10855000BDE8F083002306AA4146484605F0AEFD7B
:1085600018B100BFFEF733FBF1E79DF81800C00615
:1085700002D543F20140EAE70025072705A8019547
:1085800000970295CDE9035062884FF6FF7341468C
:10859000484605F011FD060013D16068F8F7B9FEF2
:1085A00060B960680195CDE9025000970495238871
:1085B00062884146484605F0FFFC0646BDF81400B7
:1085C00020803046CEE739B1864B0A889B899A4293
:1085D00002D843F2030070471DE610B586B0814C07
:1085E0000423ADF81430638943B1A4898C4201D2CD
:1085F000914205D943F2030006B010BD0620FBE707
:10860000ADF81010002100910191ADF80030022169
:108610008DF8021005A9029104A90391ADF812206A
:108620006946FFF7F8FDE7E72DE9FC4781460D466F
:108630000846F8F748FE88BB4846FAF704FF5FEAA9
:1086400000080AD098F80000222829D304214846BF
:108650000AF04CF8070005D103E043F20200BDE840
:10866000FC87FFDF07F1140004F0A9FA064628781A
:10867000012803D0022804D00720F0E7B0070FD567
:1086800002E016F01C0F0BD0A8792C1DC00709D0F2
:10869000E08838B1A068F8F716FE18B11020DEE7C0
:1086A0000820DCE721882A780720B1F5847F35D0BF
:1086B0001EDC40F20315A1F20313A94226D00EDC02
:1086C000B1F5807FCBD003DCF9B1012926D1C6E713
:1086D000A1F58073013BC2D0012B1FD113E0012B08
:1086E000BDD0022B1AD0032BB9D0042B16D112E027
:1086F000A1F20912082A11D2DFE802F00B040410DB
:1087000010101004ABE7022AA9D007E0012AA6D076
:1087100004E0320700E0F206002AA0DACDB200F051
:10872000E1FE50B198F82300CDE90005FA8923460F
:1087300039464846FEF78FFC91E711208FE72DE977
:10874000F04F8BB01F4615460C4683460026FAF7BD
:108750007AFE28B10078222805D208200BB081E5E6
:1087600043F20200FAE7B80801D00720F6E7032F2A
:1087700000D100274FF6FF79CCB1022D73D32046EC
:10878000F8F7EEFD30B904EB0508A8F10100F8F7A1
:10879000E7FD08B11020E1E7AD1EAAB22146484628
:1087A00005F05BFD38F8021C88425CD1ADB20D4982
:1087B000B80702D58889401C00E001201FFA80F824
:1087C000F80701D08F8900E04F4605AA4146584678
:1087D00005F03FFB4FF0070A4FF00009DCB32046DD
:1087E0000BE0000090020020408810283BD8361D86
:1087F000304486B2AE4236D2A01902884245F3D345
:1088000051E000BF9DF8170002074CD594B304EB6C
:108810000608361DB8F80230B6B2102B23D89A19C4
:10882000AA4220D8B8F8002091421CD1C0061CD51D
:10883000CDE900A90DF1080C0AAAA11948468CE857
:108840000700B8F800100022584605F08BF920B157
:10885000FEF7BDF982E726E005E0B8F80200BDF8B2
:108860002810884201D00B2078E7B8F80200304485
:1088700086B207E0FFE7C00604D55846FEF71DFCA8
:10888000002888D19DF81700BDF81A1020F01000BC
:108890008DF81700BDF81700ADF80000FF2358460B
:1088A000009A05F037FC05A805F0DFFA18B9BDF805
:1088B0001A10B942A6D90421584609F017FF04003E
:1088C00000D1FFDFA2895AB1CDE900A94D460023AE
:1088D00021465846FEF7BFFB0028BBD1A5813DE7E6
:1088E00000203BE72DE9FF4F8BB01E4617000D46D9
:1088F0004FF0000412D0B00802D007200FB0B1E44E
:10890000032E00D100265DB10846F8F720FD28B9F6
:108910003888691E0844F8F71AFD08B11020EDE701
:10892000C64AB00701D5D18900E00121F0074FF612
:10893000FF7802D0D089401E00E0404686B206AAE9
:108940000B9805F086FA4FF000094FF0070B0DF178
:10895000140A38E09DF81B00000734D5CDF80490C8
:10896000CDF800B0CDF80890CDE9039A4346002237
:108970000B9805F021FB60BB05B3BDF814103A88D5
:1089800021442819091D8A4230D3BDF81E2020F841
:10899000022BBDF8142020F8022BCDE900B9CDE957
:1089A0000290CDF810A0BDF81E10BDF814300022C2
:1089B0000B9805F001FB08B103209FE7BDF81400F8
:1089C0002044001D84B206A805F04FFA20B10A2801
:1089D00006D0FEF7FCF891E7BDF81E10B142B9D9F8
:1089E00034B17DB13888A11C884203D20C2085E7C0
:1089F000052083E722462946404605F02EFC014625
:108A000028190180A41C3C80002077E710B504469B
:108A1000F8F77FFC08B1102010BD8848C08920807D
:108A2000002010BDF0B58BB00D460646142103A8FA
:108A30001BF0F9FF01208DF80C008DF810000020CC
:108A40008DF81100ADF814503046FAF7FCFC48B12F
:108A50000078222812D30421304609F047FE040092
:108A600005D103E043F202000BB0F0BDFFDF04F1DB
:108A70001400074604F0A3F8800601D40820F3E7A9
:108A8000207C022140F00100207409A80094CDE967
:108A90000110072203A930466368FEF791FA20B15E
:108AA000217C21F001012174DEE729463046F9F7E7
:108AB000FCFC08A9384604F071F800B1FFDFBDF8EE
:108AC0002040172C01D2172000E02046A84201D9EF
:108AD0002C4602E0172C00D2172421463046FFF71F
:108AE00012FB21463046F9F706FA0020BCE7F8B53C
:108AF0001C4615460E46069F09F02AFF2346FF1D19
:108B0000BCB231462A46009409F015FBF8BD70B599
:108B10000C4605460E2120461BF063FF00202080F6
:108B20002DB1012D01D0FFDF70BD062000E0052032
:108B3000A07170BD10B548800878134620F00F0072
:108B4000001D20F0F00080300C46087014221946F9
:108B500004F108001BF00BFF00F0C7FC374804606D
:108B600010BD2DE9F047DFF8D890491D064621F0E9
:108B7000030117460C46D9F8000009F0F2FB050086
:108B800000D1FFDF4FF000083560A5F800802146D6
:108B9000D9F8000009F0E5FB050000D1FFDF7560A2
:108BA000A5F800807FB104FB07F1091D0BD0D9F8AF
:108BB000000009F0D6FB040000D1FFDFB460C4F868
:108BC0000080BDE8F087C6F80880FAE72DE9F0419B
:108BD0001746491D21F00302194D06460168144647
:108BE000286809F0E9FB22467168286809F0E4FB6F
:108BF0003FB104FB07F2121D03D0B168286809F0E9
:108C0000DBFB042009F01AFD0446042009F01EFDD8
:108C1000201A012804D12868BDE8F04109F096BB6C
:108C2000BDE8F08110B50C4605F0DFF800B1FFDFBC
:108C30002046BDE81040FDF7CABF000090020020AA
:108C40001400002038B50C468288817B19B1418917
:108C5000914200D90A462280C188121D90B26A460C
:108C600008F0E2FDBDF80000032800D30320C1B2E4
:108C7000208801F00BF838BD38B50C468288817B1E
:108C800019B10189914200D90A462280C188121D7A
:108C900090B26A4608F0C8FDBDF80000022800D373
:108CA0000220C1B2208800F0F1FF401CC0B238BDE4
:108CB0002DE9FE4F82468B46F94814460BF103021C
:108CC000D0E90010CDE9011022F0030268464FF40C
:108CD0009071009209F027FBF24E002C02D1F24A6B
:108CE00000999160009901440091357F05F10105DB
:108CF00004D1E8B20BF020FA00B1FFDF009800EBDE
:108D00000510C01C20F0030100915CB9707AB27AA2
:108D10001044C2B200200870308C80B204F0EDFE26
:108D200000B1FFDF0098316A084400902146684690
:108D300000F06FFF80460098C01C20F003000090F8
:108D4000B37AF27A717A04B1002009F0E2FB00995B
:108D5000084400902146684600F0A3FFD148002750
:108D60003D4690F801900CE0284600F035FF06469D
:108D700081788088F9F756F971786D1C00FB0177CE
:108D8000EDB24D45F0D10098C01C20F003000090DA
:108D900004B100203946F9F750F90099002708443A
:108DA0000090C0483D4690F801900CE0284600F045
:108DB00013FF0646C1788088FEF709FC71786D1CA8
:108DC00000FB0177EDB24D45F0D10098C01C20F0BA
:108DD0000300009004B100203946FEF701FC009921
:108DE0004FF0000908440090AE484D4647780EE029
:108DF000284600F0F1FE0646807B30B106F10800FF
:108E000001F013FF727800FB02996D1CEDB2BD42B8
:108E1000EED10098C01C20F00300009004B10020A7
:108E2000494601F006FF0099084400902146684633
:108E300000F0A9FE0098C01D20F007000090DAF8AD
:108E40000010814204D3A0EB0B01B1F5803F04DB9D
:108E50004FF00408CAF8000004E0CAF80000B8F1B6
:108E6000000F02D04046BDE8FE8F34BB8F49002082
:108E7000009A03F05BF8FBF760FA8A4801AA002128
:108E80001030F8F7EBFA00B1FFDF8648407FFEF7BD
:108E900054FF00B1FFDF83484FF4F67140301BF000
:108EA000C2FD80480421403080F8E91180F8EA11C1
:108EB000062180F8EB11032101710020D3E770B582
:108EC000784C06464034207804EB4015E0780835AD
:108ED00090B9A01990F8E80100280ED0A0780F28CA
:108EE00000D3FFDF202128461BF09DFD687866F344
:108EF000020068700120E070284670BD2DE9F04145
:108F000005460C4600270078052190463E46B1EB09
:108F1000101F00D0FFDF287A50B101280ED0FFDFEC
:108F2000A8F800600CB1278066800020BDE8F081C1
:108F30000127092674B16888A08008E0022714265A
:108F400044B16888A0802869E060A88A2082287BD4
:108F50002072E5E7A8F80060E7E730B5514C012042
:108F6000002120706170207260720322A272E07290
:108F700021732174052121831F21618360744CA119
:108F800061610A2121776077474D4FF4B06020621C
:108F90006868C11C21F00301814200D0FFDF6868CE
:108FA000606030BD30B5404C1568636810339D4239
:108FB00002D20420136030BD3A4B5D785A6802EB50
:108FC0000512107051700320D0801720908001206E
:108FD000D0709070002090735878401C5870606872
:108FE00010306060002030BD70B506462D4800246A
:108FF000457807E0204600F0EFFD0178B14204D04B
:10900000641CE4B2AC42F5D1002070BDF7B5074650
:1090100008780C4610B3FFF7E7FF0546A7F12006D6
:10902000202F06D0052E19D2DFE806F00F2B2B15C6
:109030001A0000F0DCFD0DB1697800E00021401A53
:10904000A17880B20844FF2808D8A07830B1A08861
:10905000022831D202E0608817282DD20720FEBDF9
:10906000207AE0B161881729F8D3A1881729F5D3B0
:10907000A1790029F2D0E1790029EFD0402804D964
:10908000ECE7242F18D1207A48B161884FF6FB70A5
:10909000814202D8A18881420ED90420FEBD0BE096
:1090A000E44D0200AC030020180000200000002066
:1090B0006E5246357800000065B9207802AA012179
:1090C000FFF770FF0028E9D12078FFF78DFF05003A
:1090D00000D1FFDF052E18D2DFE806F0030B0E08E3
:1090E0001100A0786870A088E8800FE06088A880F0
:1090F0000CE0A078A87009E0A078E87006E054F8C9
:10910000020FA8606068E86000E0FFDF0020C5E7AC
:109110001A2835D00DDC132832D2DFE800F01B31DD
:10912000203131272723252D313129313131312F7C
:109130000F00302802D003DC1E2821D10720704701
:109140003A3809281CD2DFE800F0151B0F1B1B1B47
:109150001B1B07000020704743F20400704743F2D6
:1091600002007047042070470D2070470F207047A1
:109170000820704711207047132070470620704761
:109180000320704710B5007800F0010008F03EFBA6
:10919000BDE81040BCE710B5007818B1012801D037
:1091A000072010BD08F082FBBDE81040B0E710B505
:1091B000007800F0010008F032FBBDE81040A7E79E
:1091C0000EB5017801F001018DF80010417801F031
:1091D00001018DF801100178C1F340018DF80210F2
:1091E0004178C1F340018DF80310017889088DF8AA
:1091F0000410417889088DF8051081788DF80610E3
:10920000C1788DF8071000798DF80800684607F0DE
:109210002FFAFFF77DFF0EBD2DE9F84FDFF8F88339
:10922000FE4C00264FF490771FE0012000F07CFDFB
:109230000120FFF744FE05463946D8F8080009F03A
:1092400090F8686000B9FFDF686807F0A2F8B0B175
:109250002846FAF7D8FB284600F06CFD28B93A46B4
:109260006968D8F8080009F0A7F894F9E90104281A
:10927000DBDA022009F0E2F907460025A5E03A46CC
:109280006968D8F8080009F097F8F2E7B8F8021012
:109290004046491C89B2A8F80210B94201D3002106
:1092A00041800221B8F8020009F020FA002864D0B9
:1092B000B8F80200694608F01BFAFFF729FF00B171
:1092C000FFDF9DF8000078B1B8F8020009F052FB0A
:1092D0005FEA000900D1FFDF484608F0C0FD18B181
:1092E000B8F8020002F04CF9B8F8020009F030FBBF
:1092F0005FEA000900D1FFDF484608F0A8FDE0BBA7
:109300000321B8F8020009F0F1F95FEA000B47D138
:10931000FFDF45E0DBF8100010B10078FF2849D0EE
:10932000022000F001FD0220FFF7C9FD82464846F9
:1093300008F099FECAF8040000B9FFDFDAF804006B
:1093400008F061FF002100900170B8F8021050464B
:10935000AAF8021001F016FE484608F056FF00B9C0
:10936000FFDF504600F0E6FC18B99AF8010000074C
:1093700004D50098CBF8100012E024E0DBF81000D0
:1093800038B10178491C11F0FF01017008D1FFDFED
:1093900006E000221146484600F0F3FB00B9FFDF6B
:1093A00094F9EA01022805DBB8F8020001F0AFFDEC
:1093B0000028AFD194F9E901042804DB484608F0FD
:1093C00088FF00B101266D1CEDB2BD4204D294F9B4
:1093D000EA010228BFF65AAF002E7FF422AFBDE8A3
:1093E000F84F032000F0A0BC10B58B4CE06008687B
:1093F0002061AFF2DB10F9F770FD607010BD874897
:1094000000214038017084480170854941607047EF
:1094100070B505464FF080500C46D0F8A410491C9A
:1094200005D1D0F8A810C9430904090C0BD050F895
:10943000A01F01F001012970416821608068A080AF
:10944000287830B970BD062120460CF092FB01202F
:109450002870607940F0C000607170BD70B54FF049
:1094600080540D46D4F88010491C0BD1D4F88410D8
:10947000491C07D1D4F88810491C03D1D4F88C10AA
:10948000491C0CD0D4F880100160D4F884104160DD
:10949000D4F888108160D4F88C10C16002E01021EB
:1094A0000CF067FBD4F89000401C0BD1D4F894006A
:1094B000401C07D1D4F89800401C03D1D4F89C007C
:1094C000401C09D054F8900F286060686860A0685C
:1094D000A860E068E86070BD2846BDE870401021D3
:1094E0000CF047BB4D480079E9E470B54B4CE0788F
:1094F00030B3207804EB4010407A00F0070020449D
:1095000090F9E801002800DCFFDF2078002504EB5B
:109510004010407A00F00700011991F8E801401E60
:1095200081F8E8012078401CC0B220700F2800D1DB
:109530002570A078401CA0700CF012FAE57070BD88
:10954000FFDF70BD3EB50546032109F0CFF80446A4
:10955000284609F0FDF9054604B9FFDF206918B176
:109560000078FF2800D1FFDF01AA6946284600F0F5
:1095700008FB60B9FFDF0AE0002202A9284600F0DC
:1095800000FB00B9FFDF9DF8080000B1FFDF9DF888
:109590000000411E8DF80010EED22069019988422A
:1095A00001D1002020613EBD70B50546A0F57F4089
:1095B0000C46FF3800D1FFDF012C01D0FFDF70BD6A
:1095C000FFF790FF040000D1FFDF207820F00F00AC
:1095D000401D20F0F0005030207065800020207287
:1095E00001202073BDE870407FE72DE9F041164669
:1095F0000D460746FFF776FF040000D1FFDF207815
:1096000020F00F00401D20F0F000503020706780E7
:1096100001202072286805E018000020EC030020DB
:10962000F81300202061A888A0822673BDE8F041CD
:109630005BE77FB5FFF7D8FC040000D1FFDF02A98C
:109640002046FFF7FFFA054603A92046FFF714FB63
:109650008DF800508DF80100BDF80800001DADF830
:109660000200BDF80C00001DADF80400E088ADF864
:109670000600684608F0B2F8002800D0FFDF7FBD82
:109680002DE9F05FF94E8146307810B10820BDE831
:10969000F09F4846F7F73DFE08B11020F7E7F44C7D
:1096A000207808B9FFF759FCA17A607A4D46084442
:1096B000C4B200F09CFAA04207D2201AC1B22A46D6
:1096C0000020FFF76FFC0028E1D17168E848C91C51
:1096D000002721F003017160B3463E463D46BA467D
:1096E0003C4690F801800AE0204600F075FA417887
:1096F000807B0E4410FB0155641CE4B27F1C444582
:10970000F2D1C6EBC601DA4E0AEB870000EB81000E
:10971000F17A00EB850000EB8100DBF804105C4679
:109720004518012229464846FFF7C2FA070012D021
:109730000020FFF759FC05000BD005F1130061680C
:1097400020F00300884200D0FFDF7078401E707068
:10975000656038469BE7002229464846FFF7A8FA8D
:1097600000B1FFDFD9F8000060604FF6FF70608045
:109770000120207000208AE72DE9F0410446BB4813
:1097800017460E46007810B10820BDE8F081084663
:10979000F7F799FD08B11020F7E7B54D287808B91B
:1097A000FFF7DBFB601E1E2807D8012C22D1307882
:1097B000FE281FD828770020E7E7A4F120001F2803
:1097C00005D8E0B23A463146BDE8F0411EE4A4F1C6
:1097D00040001F2805D831462046BDE8F04100F082
:1097E000D1BAA4F1A0001F2804D80020A02C03D0D7
:1097F000A12C06D00720C8E7317801F00101697774
:10980000C3E731680922F82901D38B0701D010463C
:10981000BBE76B7C03F00303012B04D16B8BD733C5
:109820009CB28C42F3D82962AFE72DE9F04781461C
:109830000E460846F7F76DFD48B94846F7F787FD2D
:1098400028B909F1030020F00301494502D0102096
:10985000BDE8F08786484FF0000A4030817869B152
:109860004178804600EB41140834378832460021A5
:10987000204600F06DFA050004D027E0A6F800A00D
:109880000520E5E7B9F1000F24D03088B84201D9AE
:109890000C251FE0607800F00705284600F044FA28
:1098A00008EB0507324697F8E8014946401C87F85F
:1098B000E801204607F5F47700F04AFA05463878C3
:1098C000401E3870032000F02FFA2DB10C2D01D06E
:1098D000A6F800A02846BBE76078644E00F00701B8
:1098E000012923D002290CD0032934D0FFDF98F8B6
:1098F00001104046491CC9B288F801100F2935D023
:1099000036E0616821B1000702D46088FFF71AFED3
:1099100098F8EA014746012802D17078F9F7FCFA75
:1099200097F9EA010428E2DBFFDFE0E7616821B193
:109930004FF49072B06808F03FFD98F8E90147468F
:10994000032802D17078F9F7E7FA97F9E9010428BA
:10995000CDDBFFDFCBE7C00602D56088FFF7F2FD65
:1099600098F9EB010628C2DBFFDFC0E780F801A011
:109970008178491E8170617801F0070101EB0800D0
:1099800090F8E811491C80F8E811A3E770B50D467E
:109990000446F7F798FC18B92846F7F7BAFC08B15F
:1099A000102070BD29462046BDE870400AF0FBBB80
:1099B00070B505460AF01AFCC4B22846F7F7C7FC92
:1099C00008B1102070BD35B128782C7018B1A042B4
:1099D00001D0072070BD2046FDF764FE052805D1A3
:1099E0000AF008FC012801D0002070BD0F2070BDD6
:1099F00070B5044615460E460846F7F764FC18B9DC
:109A00002846F7F786FC08B1102070BD022C03D061
:109A1000102C01D0092070BD2A46314620460AF09C
:109A2000F2FB0028F7D0052070BD70B514460D4636
:109A30000646F7F748FC38B92846F7F76AFC18B924
:109A40002046F7F784FC08B1102070BD2246294655
:109A500030460AF0F7FB0028F7D0072070BD3EB56E
:109A60000446F7F756FC28B110203EBD1800002030
:109A7000AC030020684606F064FDFFF749FB0028B0
:109A8000F3D19DF806002070BDF808006080BDF895
:109A90000A00A0800020E8E770B505460C4608469D
:109AA000F7F755FC20B93CB12068F7F732FC08B154
:109AB000102070BDA08828B121462846BDE870401E
:109AC000FDF748BE092070BD70B504460D46084636
:109AD000F7F7F9FB30B9601E1E2814D82846F7F7AF
:109AE000F2FB08B1102070BD042C01D9072070BD15
:109AF00004B9FFDFF54800EB840050F8041C284649
:109B0000BDE870400847A4F120001F2805D8294669
:109B10002046BDE87040FAF798BBF02CE6D1A86863
:109B2000F7F7D1FB0028DDD1284607F0C4FEBDE8D9
:109B30007040FFF7EDBA70B504460D460846F7F7DA
:109B4000E8FB30B9601E1E2811D82846F7F7BBFB8A
:109B500008B1102070BD012C05D0022C03D0032CBD
:109B600001D0042C01D1062070BD072070BDA4F1E6
:109B700020001F28F9D829462046BDE87040FAF792
:109B8000BCBB08F033B938B50446D148007B00F0BF
:109B90000105D9B904F012FB0DB1226800E00022E2
:109BA000CC484178C06806F0BAFBCA481030C0788B
:109BB0008DF8000010B1012802D004E0012000E07F
:109BC00000208DF80000684606F033FD002D02D01D
:109BD00020682830206038BD30B5BD4D0446687817
:109BE000A04200D8FFDF686800EB041030BD70B5FC
:109BF000B74800252C46467807E02046FFF7ECFFE3
:109C00004078641C2844C5B2E4B2B442F5D1284679
:109C100070BD2DE9F0410C4607464FF0000800F0FA
:109C2000DEF80646FF2801D94FF013083868C01C3B
:109C300020F003023A6054EA080421D1A448F3B2A8
:109C4000072124300CF09AF909E0072C10D2DFE844
:109C500004F0060408080A0406009F4804E09F4830
:109C600002E09F4800E09F480CF0A8F9054600E09C
:109C7000FFDFA54200D0FFDF641CE4B2072CE4D371
:109C8000386800EB0610386040467EE5021D5143FF
:109C9000452900D245210844C01CB0FBF2F0C0B2F7
:109CA00070472DE9FC5F064689484FF000088B4657
:109CB0004746444690F8019022E02046FFF78CFF8B
:109CC000050000D1FFDF687869463844C7B22846EE
:109CD000FEF7B8FF824601A92846FEF7CDFF0346EE
:109CE000BDF804005246001D81B2BDF80000001D01
:109CF00080B208F079FD6A78641C00FB0288E4B247
:109D00004C45DAD13068C01C20F003003060BBF154
:109D1000000F00D000204246394608F073FD31683C
:109D200008443060BDE8FC9F69494031087100205B
:109D3000C870704766494031CA782AB10A7801EB89
:109D400042110831814201D0012070470020704744
:109D50002DE9F04106460078154600F00F0400207A
:109D60001080601E0F46052800D3FFDF57482A46A3
:109D7000183800EB8400394650F8043C3046BDE802
:109D8000F041184770B50C46402802D0412806D152
:109D900020E0A07861780D18E178814201D9072090
:109DA00070BD2078012801D9132070BDFF2D08D87F
:109DB0000AF0B2FB06460BF08BFD301A801EA8425B
:109DC00001DA122070BD4248216881602179017357
:109DD000002070BDBDE87040084600F02BB82DE9AA
:109DE000F047DFF8EC900026344699F8090099F81E
:109DF0000A2099F801700244D5B299F80B2010445A
:109E000000F0FF0808E02046FFF7E6FE817B40787F
:109E100011FB0066641CE4B2BC42F4D199F809104D
:109E200099F80A0029442944414400B1012008441A
:109E300030440DE538B50446407800F003000128B1
:109E400003D002280BD0072038BD606858B1F7F75F
:109E500087FAD0B96068F7F77AFA20B915E0606838
:109E6000F7F731FA88B969462046FCF797F80028D9
:109E7000EAD1607800F00300022808D19DF80000C4
:109E800028B16068F7F763FA08B1102038BD61891E
:109E9000F8290DD8208988420AD8607800F003029A
:109EA0000B48012A06D1D731026A89B28A4201D20F
:109EB000092038BD94E80E0000F1100585E80E0079
:109EC0000AB900210183002038BD0000044E0200C1
:109ED000AC030020180000204B410000FFAC000044
:109EE000E92F00002B3F01002DE9F0410746144601
:109EF0008846084601F022FD064608EB88001C2231
:109F0000796802EBC0000D18688C58B1414638469C
:109F100001F01CFD014678680078C200082305F1B5
:109F200020000CE0E88CA8B14146384601F015FD50
:109F30000146786808234078C20005F1240008F043
:109F400092FA38B1062121726681D0E90010C4E985
:109F5000031009E0287809280BD0052020726681BB
:109F60006868E060002028702046BDE8F04101F0FC
:109F7000DBBC072020726681F4E72DE9F04116462C
:109F80000D460746406801EB85011C2202EBC1012A
:109F90004418204601F003FD40B10021708865F3AC
:109FA0000F2160F31F4106200CF0C2F80920207039
:109FB000324629463846BDE8F04195E72DE9F041A3
:109FC0000E46074600241C21F07816E004EB8403BB
:109FD000726801EBC303D25C6AB1FFF783FA050034
:109FE00000D1FFDF6F802A4621463046FFF7C5FFCC
:109FF0000120BDE8F081641CE4B2A042E6D8002054
:10A00000F7E770B5064600241C21C0780AE000BFBF
:10A0100004EB8403726801EBC303D5182A782AB1D4
:10A02000641CE4B2A042F3D8402070BD2821284629
:10A030001AF0D7FC706880892881204670BD70B501
:10A04000034600201C25DC780DE000BF00EB8006F5
:10A050005A6805EBC6063244167816B1128A8A424F
:10A0600004D0401CC0B28442F0D8402070BDF0B58E
:10A07000044600201C26E5780EE000BF00EB8007B8
:10A08000636806EBC7073B441F788F4202D15B78B9
:10A09000934204D0401CC0B28542EFD84020F0BDAE
:10A0A0000078032801D00020704701207047007815
:10A0B000022801D00020704701207047007807284F
:10A0C00001D000207047012070472DE9F04106467D
:10A0D00088461078F1781546884200D3FFDF2C7847
:10A0E0001C27641CF078E4B2A04201D8201AC4B244
:10A0F00004EB8401706807EBC1010844017821B1C9
:10A100004146884708B12C7073E72878A042E8D10F
:10A11000402028706DE770B514460B880122A240DC
:10A12000134207D113430B8001230A22011D08F0BB
:10A1300064F9047070BD2DE9FF4F81B00878DDE946
:10A140000E7B9A4691460E4640072CD4019808F0A3
:10A1500011FC040000D1FFDF07F1040820461FFABC
:10A1600088F107F050FD050000D1FFDF20462946A9
:10A170006A4607F09AFF0098A0F80370A0F805A0BF
:10A18000284608F040F8017869F306016BF3C7111F
:10A19000017020461FFA88F107F078FD00B9FFDF53
:10A1A000019806F02EF806EB0900017F491C0177A3
:10A1B00005B0BDE8F08F2DE9F84F0E469A4691465E
:10A1C0000746032108F092FA0446008DDFF8B885AF
:10A1D000002518B198F80000B0421ED1384608F0AA
:10A1E000C9FB070000D1FFDF09F10401384689B23D
:10A1F00007F009FD050010D0384629466A4607F0E9
:10A2000054FF009800210A460180817006F0B2F8E0
:10A210000098C01DCAF8000021E098F80000B04284
:10A2200016D104F1260734F8341F012000FA06F98C
:10A2300011EA090F00D0FFDF2088012340EA09005E
:10A2400020800A22391D384608F0F2F8067006E030
:10A25000324604F1340104F12600FFF75CFF0A21C5
:10A2600088F800102846BDE8F88FFEB515460C4664
:10A27000064602AB0C220621FFF79DFF002827D0DF
:10A280000299607812220A70801C487008224A8065
:10A29000A07002982988052381806988C180A988D7
:10A2A0000181E988418100250C20CDE900050622C5
:10A2B00021463046FFF73FFF2946002266F31F4143
:10A2C000F02310460BF08AFE6078801C607001203D
:10A2D000FEBDFEB514460D460622064602AB1146EB
:10A2E000FFF769FF002812D0029B1320002118708D
:10A2F000A8785870022058809C800620CDE9000183
:10A300000246052329463046FFF715FF0120FEBD12
:10A310002DE9FE430C46804644E002AB0E220721A5
:10A320004046FFF748FF002841D060681C2267784C
:10A330008678BF1C06EB860102EBC1014518029826
:10A340001421017047700A214180698A0181E98ADC
:10A350004181A9888180A9898181304601F0EEFA86
:10A36000029905230722C8806F70042028700025F9
:10A370000E20CDE9000521464046FFF7DCFE2946C8
:10A3800066F30F2168F31F41F023002206200BF033
:10A3900025FE6078FD49801C607062682046921C32
:10A3A000FFF793FE606880784028B6D10120BDE8B1
:10A3B000FE83FEB50D46064638E002AB0E220721AD
:10A3C0003046FFF7F8FE002835D068681C23C178B6
:10A3D00001EB810203EBC20284180298152202707D
:10A3E000627842700A224280A2894281A2888281D8
:10A3F000084601F0A3FA014602988180618AC18073
:10A40000E18A0181A088B8B10020207000210E20CF
:10A41000CDE900010523072229463046FFF78BFED0
:10A420006A68DB492846D21CFFF74FFE6868C0788F
:10A430004028C2D10120FEBD0620E6E72DE9FE43FB
:10A440000C46814644E0204601F093FAD0B302ABBB
:10A45000082207214846FFF7AEFE0028A7D0606813
:10A460001C2265780679AD1C06EB860102EBC10162
:10A4700047180298B7F81080062101704570042132
:10A480004180304601F05AFA01460298052307221E
:10A49000C180A0F804807D70082038700025CDE9C7
:10A4A000000521464846FFF746FE294666F30F2180
:10A4B00069F31F41F023002206200BF08FFD607826
:10A4C000801C60706268B3492046121DFFF7FDFDD5
:10A4D000606801794029B6D1012068E72DE9F34F82
:10A4E00083B00E4680E0304601F043FA002875D074
:10A4F00071681C2091F8068008EB880200EBC2000E
:10A500000C184146304601F028FA0146A078C300F5
:10A5100070684078C20004F1240007F0C0FF0746CD
:10A520008088E18B401A80B2002581B3AA46218B36
:10A53000814200D808468146024602AB07210398B3
:10A54000FFF739FE010028D0BAF1000F03D0029ABC
:10A55000B888022510808B46E28B3968A9EB05008C
:10A560001FFA80FA0A440398009208F003FAED1DDE
:10A57000009A59465346009507F011FEE08B50446F
:10A5800080B2E083B988884209D1012508E0FFE75D
:10A59000801C4FF0010A80B2C9E7002008E60025C0
:10A5A000CDE90095238A072231460398FFF7C3FDC2
:10A5B000E089401EE0818DB1A078401CA0707068D9
:10A5C000F178427811FB02F1CAB2816901230E30A1
:10A5D00007F013FF80F800800020E08372686E4966
:10A5E0003046921DFFF771FD7068817940297FF434
:10A5F0007AAF0120DCE570B5064648680D46144682
:10A600008179402910D104EB84011C2202EBC101A5
:10A61000084401F0E5F9002806D0686829468471ED
:10A620003046BDE8704059E770BDFEB50C460746A0
:10A63000002645E0204601F09CF9D8B360681C2252
:10A64000417901EB810102EBC1014518688900B92C
:10A65000FFDF02AB082207213846FFF7ACFD0028D8
:10A6600033D00299607816220A70801C487004204A
:10A6700048806068407901F061F90146029805233D
:10A68000072281806989C1800820CDE90006214622
:10A690003846FFF750FD6078801C6070A889698992
:10A6A0000844B0F5803F00D3FFDFA88969890844DA
:10A6B000A8816E81626839492046521DFFF705FD69
:10A6C000606841794029B5D10120FEBD30B5438C89
:10A6D000458BC3F3C704002345B1838B641EED1A79
:10A6E000C38A6D1E1D4495FBF3F3E4B22CB10089BF
:10A6F00018B1A04200D8204603444FF6FF708342B1
:10A7000000D3034613800C7030BD2DE9FC41074691
:10A7100016460D46486802EB86011C2202EBC10179
:10A7200044186A4601A92046FFF7D0FFA089618935
:10A7300001448AB2BDF80010914212D0081A00D527
:10A74000002060816868407940280AD1204601F0E5
:10A750003DF9002805D06868294646713846FFF75C
:10A7600064FFBDE8FC812DE9FE4F89468046154611
:10A770005088032107F0BAFF8346B8F8020040284A
:10A780000ED240200DE000002C000020A1A000000F
:10A79000AFA00000BDA00000E1B90000CDB90000ED
:10A7A000403880B282460146584601F0E2F800285F
:10A7B0007ED00AEB8A001C22DBF8041002EBC000FA
:10A7C0000C18204601F0EBF8002877D1B8F800000B
:10A7D000E18A88423CD8A189D1B348456ED1002690
:10A7E0005146584601F0B2F8218C0F18608B48B9D9
:10A7F000B9F1020F62D3B8F804006083618A88421D
:10A8000026D80226A9EB06001FFA80F9B888A28B89
:10A81000801A002814DD4946814500DA084683B2D3
:10A8200068886968029139680A44CDE9003208F005
:10A830008FF8DDE90121F61D009B009607F07BFCF7
:10A84000A18B01EB090080B2A083618B884207D9FC
:10A85000688803B052465946BDE8F04F01F0DDB8B4
:10A860001FD14FF009002872B8F802006881D7E9BB
:10A870000001C5E90401608BA881284601F054F865
:10A880005146584601F062F80146DBF804000823FF
:10A890000078C20004F1200007F0E5FD0020A0834D
:10A8A0006083A0890AF0FF02401EA081688800E052
:10A8B00004E003B05946BDE8F04F26E7BDE8FE8F3F
:10A8C0002DE9F041064615460F461C461846F6F798
:10A8D000FAFC18B92068F6F71CFD08B1102013E443
:10A8E0007168688C0978B0EBC10F01D313200BE4B9
:10A8F0003946304601F02AF801467068082300788E
:10A90000C20005F1200007F078FDD4E90012C0E98B
:10A9100000120020E3E710B50446032107F0E6FE2D
:10A920000146007800F00300022805D02046BDE86B
:10A93000104001F1140298E48A8A2046BDE81040D4
:10A94000C7E470B50446032107F0D0FE0546014672
:10A950002046FFF773FD002816D029462046FFF752
:10A9600064FE002810D029462046FFF722FD00286B
:10A970000AD029462046FFF7CBFC002804D0294600
:10A980002046BDE87040A9E570BD2DE9F0410C46B8
:10A9900080461EE0E178427811FB02F1CAB281697B
:10A9A00001230E3007F05FFD077860681C22C17933
:10A9B000491EC17107EB8701606802EBC1014618AF
:10A9C0003946204600F0D5FF18B1304600F0E0FFD0
:10A9D00020B16068C1790029DCD180E7FEF782FDF3
:10A9E000050000D1FFDF0A202872384600F0A6FFDC
:10A9F00068813946204600F0B0FF014660680823B0
:10AA00004078C20006F1240007F02DFDD0E90010C7
:10AA1000C5E90310A5F80280284600F085FFB0784C
:10AA200000B9FFDFB078401EB07058E770B50C4633
:10AA30000546032107F05AFE01464068C2792244C8
:10AA4000C2712846BDE870409FE72DE9FE4F82465F
:10AA5000507814460F464FF0000800284FD00128C8
:10AA600007D0022822D0FFDF2068B8606068F86055
:10AA700024E702AB0E2208215046FFF79CFB00287A
:10AA8000F2D00298152105230170217841700A2126
:10AA90004180C0F80480C0F80880A0F80C8062886B
:10AAA00082810E20CDE90008082221E0A6783046F8
:10AAB00000F044FF054606EB86012C22786802EB85
:10AAC000C1010822465A02AB11465046FFF773FBFC
:10AAD0000028C9D002980721017021784170042113
:10AAE000418008218580C680CDE9001805230A46EB
:10AAF00039465046FFF71FFB87F80880DEE6A67848
:10AB0000022516B1022E13D0FFDF2A1D914602AB9B
:10AB100008215046FFF74FFB0028A5D002980121DD
:10AB2000022E0170217841704580868002D005E0B8
:10AB30000625EAE7A188C180E1880181CDE9009876
:10AB40000523082239465046D4E710B504460321B0
:10AB500007F0CCFD014600F108022046BDE8104098
:10AB600073E72DE9F05F0C4601281DD0957992F826
:10AB70000480567905EB85011F2202EBC10121F00B
:10AB8000030B08EB060111FB05F14FF6FF7202EA19
:10AB9000C10909F1030115FB0611F94F21F0031A50
:10ABA00040B101283DD124E06168E57891F800804A
:10ABB0004E78DFE75946786807F0D3FB606000B94C
:10ABC000FFDF5946606819F02EFFE570514678683E
:10ABD00007F0C7FB6168486100B9FFDF6068426940
:10ABE00002EB09018161606880F80080606846704E
:10ABF00017E0606852464169786807F0DDFB5A4605
:10AC00006168786807F0D8FB032007F017FD044659
:10AC1000032007F01BFD201A012802D1786807F0F5
:10AC200095FB0BEB0A00BDE8F09F024600210220D5
:10AC300097E773B5D24D0A202870009848B10024D8
:10AC40004FEA0D0007F06FFB002C01D100996960FD
:10AC50007CBD01240020F5E770B50C46154638216F
:10AC6000204619F0E0FE012666700A2104F11C005E
:10AC700019F0D9FE05B9FFDF297A207861F30100C8
:10AC80002070A879002817D02A4621460020FFF717
:10AC900068FF6168402088706168C87061680871E9
:10ACA0006168487161688871616828880881616895
:10ACB000688848816068868170BDC878002802D0A5
:10ACC000002201204DE7704770B50546002165F36D
:10ACD0001F4100200BF02CFA0321284607F006FD47
:10ACE000040000D1FFDF21462846FFF767F900285E
:10ACF00004D0207840F010002070012070BD2DE9B4
:10AD0000FF4180460E460F0CFEF7ECFB050007D016
:10AD10006F800321384607F0E9FC040008D106E003
:10AD200004B03846BDE8F0411321F9F743BEFFDF18
:10AD30005FEA080005D0B8F1060F18D0FFDFBDE8C4
:10AD4000FF8120782A4620F0080020700020ADF80E
:10AD5000020002208DF800004FF6FF70ADF80400ED
:10AD6000ADF8060069463846F9F71BFAE7E7C6F37F
:10AD7000072101EB81021C23606803EBC202805CA7
:10AD8000042803D008280AD0FFDFD8E7012000906C
:10AD90004FF440432A46204600F008FECFE704B0B7
:10ADA0002A462046BDE8F041FFF7E7B82DE9F05FFD
:10ADB0000027B0F80A9090460C4605463E46B9F189
:10ADC000400F01D2402001E0A9F140001FFA80FAB3
:10ADD000287AC01E08286BD2DFE800F00D04192085
:10ADE00058363C4772271026002C6CD0D5E9030159
:10ADF000C4E902015CE070271226002C63D00A220D
:10AE000005F10C0104F1080019F0B1FD50E07127C3
:10AE10000C26002C57D0E868A06049E07427102663
:10AE20009CB3D5E90301C4E902016888032107F056
:10AE30005DFC8346FEF756FB02466888508051460B
:10AE40005846FFF751F833E075270A26ECB1A88978
:10AE500020812DE076271426BCB105F10C0004F109
:10AE6000080307C883E8070022E07727102664B1AB
:10AE7000D5E90301C4E902016888032107F036FC23
:10AE800001466888FFF781FD12E01CE07327082661
:10AE9000CCB16888032107F029FC01460078C00680
:10AEA00006D56888FFF78AF810B96888F8F78FFD2B
:10AEB000A8F800602CB12780A4F806906680688806
:10AEC000A0800020AFE6A8F80060FAE72DE9FC4179
:10AED0000C461E4617468046032107F007FC054630
:10AEE0000A2C0AD2DFE804F0050505050505090965
:10AEF0000907042303E0062301E0FFDF0023CDE977
:10AF00000076224629464046FFF715F929E438B570
:10AF10000546A0F57F40FF3830D0284607F018FDE1
:10AF2000040000D1FFDF204607F09DF8002815D06F
:10AF300001466A46204607F0B8F800980321B0F8A9
:10AF40000540284607F0D2FB0546052C03D0402CCF
:10AF500005D2402404E0007A80B1002038BD403C96
:10AF6000A4B2214600F005FD40B1686804EB8401FD
:10AF70003E2202EBC101405A0028EFD0012038BD2B
:10AF80002C0000202DE9F04F054689B0408807F0DD
:10AF9000DFFC040000D1FFDF06AA2046696800F04C
:10AFA000C1FC069C001F34F8031F21806388638066
:10AFB000228881B28A4205D1042B0AD0052B1DD0EC
:10AFC000062B15D02A462046FFF7CDFB09B0BDE879
:10AFD000F08F1646241D2A4621463046F7F74FFAD1
:10AFE0000828F3D12A4621463046FCF7FAFBEDE764
:10AFF0006888211D6B68FAF73FFCE7E71746688809
:10B00000032107F073FB4FF000088DF8048006461B
:10B01000ADF80680042FD9D36279002AD6D02079E2
:10B020004FF6FF794FF01C0A13282CD008DC0128BA
:10B0300078D0062847D0072875D0122874D106E0AA
:10B04000142872D0152871D016286DD1ACE10C2FC0
:10B050006AD1307800F00301022965D140F0080080
:10B0600030706079B07001208DF804002089ADF84F
:10B0700008006089ADF80A00A089ADF80C00E089ED
:10B08000ADF80E0019E0B07890429FD130780107FA
:10B090009CD5062F9AD120F0080030706888414670
:10B0A00060F31F4100200BF043F802208DF80400EC
:10B0B000ADF808902089ADF80A0068882A4601A9F1
:10B0C000F9F76FF882E7082F80D12789B4F80A9042
:10B0D000402F01D2402001E0A7F1400080B280461D
:10B0E0000146304600F045FC08B3716808EB880063
:10B0F0002C2202EBC000095A4945E3D1FE4807AAB9
:10B10000D0E90210CDE9071060798DF81C0008F035
:10B11000FF048DF81E4068883146FFF796FC2A46EA
:10B12000214639E0B6E014E03CE039E0E6E0F248E0
:10B13000D0E90010CDE907106079ADF820708DF8E6
:10B140001C00ADF82290688807AA3146FFF77DFC05
:10B150003CE7082FB6D16089B4F80880402801D2B6
:10B16000402000E0403887B23946304600F001FC0C
:10B170000028A7D007EB870271680AEBC2000844D9
:10B18000028A42459ED1017808299BD14078617995
:10B19000884297D1F9B22A463046FEF7EEFE15E70F
:10B1A0000E2F07D0CDF81C80CDF8208060798DF867
:10B1B0001C00C8E76189E7898B46B4F80C903046DB
:10B1C000FEF73DFFABF14001402901D309204AE0E1
:10B1D000B9F1170F01D3172F01D20B2043E04028FC
:10B1E0000ED000EB800271680AEBC20008440178BF
:10B1F000012903D1407861798842A9D00A2032E040
:10B200003046FEF7FEFE014640282BD001EB8103BD
:10B2100072680AEBC30002EB0008012288F80020E4
:10B22000627988F80120706822894089B84200D983
:10B230003846248A03232B72AA82EF812882A5F83C
:10B240000C906C82084600F079FB6881A8F8149095
:10B25000A8F81870A8F80E40A8F810B0284600F01A
:10B2600063FBB3E6042005212972A5F80A80E88172
:10B2700001212973A049D1E90421CDE90721617990
:10B280008DF81C10ADF81E00688807AA3146FFF73C
:10B29000DCFBE3E7062FE4D3B078904215D1307899
:10B2A000010712D520F0080030706888414660F32D
:10B2B0001F4100200AF03CFF02208DF80400208985
:10B2C000ADF80800ADF80A90F7E604213046FEF725
:10B2D000CEFE04464028C4D00220830300902A46B4
:10B2E0002146304600F062FB4146688864F30F2136
:10B2F00060F31F4106200AF01BFF67E60E2FB0D156
:10B3000004213046FEF7B3FE81464028A9D04146CD
:10B31000688869F30F2160F31F4106200AF008FFD7
:10B32000208A0790E08900907068A7894089B84218
:10B3300000D938468346B4F80A80208905904846EB
:10B3400000F0FCFA6881079840B10220079B00904A
:10B350002A464946304600F029FB37E6B8F1170F78
:10B360001ED3172F1CD30420287200986882EF8107
:10B37000A5F810B0A5F80C8009EB89020AEBC20011
:10B380007168009A0C180598A4F81480A4F818B0F5
:10B39000E2812082284600F0C7FA0620207015E6D8
:10B3A00001200B230090D3E7082FA6D12189304636
:10B3B000FEF745FE074640289FD007EB87027168DD
:10B3C0000AEBC2000844804600F0E9FA002894D154
:10B3D0006489B8F80E002044B0F5803F05D3688832
:10B3E0003A46314600F019FBF0E5002C85D0A8F86C
:10B3F0000E0068883A463146FFF7FDF808202872AB
:10B40000384600F09BFA6881AC8127E770B50D469D
:10B410000646032107F06AF9040004D020780007EB
:10B4200004D5112070BD43F2020070BD2A462146AA
:10B430003046FEF71AFF18B9286860616868A06195
:10B44000207840F008002070002070BD70B50D46D7
:10B450000646032107F04AF9040004D020780007CB
:10B4600004D4082070BD43F2020070BD2A46214674
:10B470003046FEF72EFF00B9A582207820F00800A4
:10B480002070002070BD2DE9F04F0E4691B080462F
:10B49000032107F02BF90446404607F06BFA0746F4
:10B4A0000020079008900990ADF830000A900290B3
:10B4B0000390049004B9FFDF0DF108091FBBFFDF03
:10B4C00021E038460BA9002206F090FC9DF82C00E4
:10B4D00000F07F050A2D00D3FFDF6019017F491EB0
:10B4E00001779DF82C0000060DD52A460CA907A867
:10B4F000FEF711FE02E00000144E020019F80510DC
:10B50000491C09F80510761EF6B2DAD204F13400AF
:10B51000FA4D04F1260BDFF8E8A304F12A070690A0
:10B5200010E05846069900F06AFA064628700A2884
:10B5300000D3FFDF5AF8261040468847E08CC05DF4
:10B54000B04202D0208D0028EBD10A202870EC4DAB
:10B550004E4628350EE00CA907A800F050FA044624
:10B56000375D55F8240000B9FFDF55F8242039462F
:10B5700040469047BDF81E000028ECD111B026E5EA
:10B5800010B5032107F0B2F8040000D1FFDF0A2153
:10B5900004F11C0019F047FA207840F004002070F4
:10B5A00010BD10B50C46032107F0A0F82044007F21
:10B5B000002800D0012010BD2DE9F84F894615461E
:10B5C0008246032107F092F8070004D02846F5F7D9
:10B5D0007AFE40B903E043F20200BDE8F88F484626
:10B5E000F5F797FE08B11020F7E7786828B1698869
:10B5F0000089814201D90920EFE7B9F800001C2435
:10B6000018B1402809D2402008E03846FEF7F9FC7E
:10B610008046402819D11320DFE7403880B28046A9
:10B620000146384600F0A5F948B108EB8800796872
:10B6300004EBC000085C012803D00820CDE70520FA
:10B64000CBE7FDF74FFF06000BD008EB88007968C9
:10B6500004EBC0000C18B9F8000020B1E88910B163
:10B6600013E01120B9E72888172802D36888172823
:10B6700001D20720B1E7686838B12B1D2246414648
:10B680003846FFF71DF90028A7D104F10C026946DE
:10B690002046FFF71BF8288860826888E082B9F8A6
:10B6A000000030B102202070E889A080E889A0B1B4
:10B6B0002BE003202070A889A08078688178402939
:10B6C00005D180F8028039465046FEF721FE4046FB
:10B6D00000F034F9A9F8000021E07868218B408956
:10B6E000884200D908462083A6F802A004203072C0
:10B6F000B9F800007081E0897082F181208B30827E
:10B70000A08AB081304600F00FF97868C1784029EE
:10B7100005D180F8038039465046FEF74AFE0020E6
:10B720005BE770B50D460646032106F0DFFF040017
:10B7300003D0402D04D2402503E043F2020070BD47
:10B74000403DADB2294600F014F958B105EB850132
:10B750001C22606802EBC101084400F020F918B116
:10B76000082070BD052070BD2A462146304600F0F5
:10B7700054F9002070BD2DE9F0410D461646804673
:10B78000032106F0B3FF0446402D01D2402500E01E
:10B79000403DADB28CB1294600F0EBF880B105EB2D
:10B7A00085011C22606802EBC1014718384600F091
:10B7B000F6F838B10820BDE8F08143F20200FAE75C
:10B7C0000520F8E733463A4629462046FFF778F841
:10B7D0000028F0D1EAB221464046FEF796FF00204D
:10B7E000E9E72DE9F0410D4616468046032106F0B3
:10B7F0007DFF0446402D01D2402500E0403DAFB220
:10B8000024B13046F5F75FFD38B902E043F202009B
:10B81000D1E73068F5F757FD08B11020CBE739467E
:10B82000204600F0A6F860B107EB87011C22606893
:10B8300002EBC1014518284600F0B1F818B1082004
:10B84000B9E70520B7E7B088A98A884201D90C205A
:10B85000B1E76168E88C4978B0EBC10F01D31320E0
:10B86000A9E73946204600F078F8014660680823C9
:10B870004078C20005F1240006F0BFFDD6E90012B1
:10B88000C0E90012FAB221464046FEF7B4FE00209D
:10B8900091E72DE9F0470D461F469046814603216A
:10B8A00006F024FF0446402D01D2402001E0A5F11E
:10B8B000400086B23CB14DB13846F5F748FD50B175
:10B8C0001020BDE8F08743F20200FAE76068C8B1D3
:10B8D000A0F80C8024E03146204600F04AF888B1F8
:10B8E00006EB86011C22606802EBC1014518284660
:10B8F00000F055F840B10820E3E700002C000020DC
:10B900002C4E02000520DCE7A5F80880F2B22146A3
:10B910004846FEF7FAFE1FB1A889698908443880B5
:10B920000020CEE706F0C1BB017821F00F01491CD1
:10B9300021F0F00110310170FDF7D7BD10B50446BC
:10B94000402800D9FFDF4034A0B210BD40684269F2
:10B950000078484302EBC0007047C2784068037823
:10B9600012FB03F24378406901FB032100EBC100A5
:10B970007047C2788A4209D9406801EB81011C22D4
:10B9800002EBC101405C08B1012070470020704704
:10B990000078062801D90120704700207047007800
:10B9A000062801D00120704700207047F0B401EB59
:10B9B00081061C27446807EBC6063444049D05260F
:10B9C0002670E3802571F0BCFEF78EBA10B5418970
:10B9D00011B1FFF7DDFF08B1002010BD012010BD3F
:10B9E00010B5C18C8278B1EBC20F04D9C18911B1F5
:10B9F000FFF7CEFF08B1002010BD012010BD10B52B
:10BA00000C4601230A22011D06F02DFD0078218835
:10BA1000012282409143218010BDF0B402EB8205E7
:10BA20001C264C6806EBC505072363554B681C793B
:10BA3000402C03D11A71F0BCFEF700BDF0BC70477A
:10BA400010B5EFF3108000F0010472B6F7484178AA
:10BA5000491C41704078012801D109F0A9FF002C50
:10BA600000D162B610BD70B5F04CA07848B9012580
:10BA7000A570FFF7E5FF09F0ACFF20B1002009F049
:10BA800076FF002070BD4FF08040E570C0F8045391
:10BA9000F7E770B5EFF3108000F0010572B6E34CE4
:10BAA000607800B9FFDF6078401E6070607808B988
:10BAB00009F082FF002D00D162B670BDDB4810B5E1
:10BAC000817821B10021C1708170FFF7E2FF002071
:10BAD00010BD10B5044609F07CFFD44989780840B0
:10BAE00000D001202060002010BD10B5FFF7A8FF96
:10BAF00009F06FFF02220123CC49540728B1CC483A
:10BB0000026023610320087202E00A72C4F8043361
:10BB10000020887110BD2DE9F84FDFF810934278AE
:10BB2000817889F80420002689F80510074689F8ED
:10BB300006600078DFF8FCB2354620B1012811D04C
:10BB4000022811D0FFDF09F056FF4FF0804498B172
:10BB500009F058FFB0420FD1304609F057FF0028D6
:10BB6000FAD041E00126EEE7FFF76AFF5846016888
:10BB7000C907FCD00226E6E70120E060C4F80451C2
:10BB8000AD490E600107D1F84412AB4AC1F342310E
:10BB900024321160A849343108604FF0020AC4F819
:10BBA00004A3A060A5480168C94341F3001101F155
:10BBB0000108016841F01001016000E020BFD4F8E5
:10BBC00004010028FAD0304609F020FF0028FAD0FE
:10BBD000B8F1000F04D19948016821F0100101600B
:10BBE000C4F808A3C4F8045199F805004E4680B182
:10BBF000387870B909F0EDFE80460AF081F86FF0F0
:10BC00000042B8F1000F02D0C6E9032001E0C6E906
:10BC10000302DBF80000C00701D009F0D6FE387837
:10BC200010B13572BDE8F88F4FF01808C4F80883DA
:10BC30000127A7614FF4A070ADF80000BDF8000027
:10BC4000411EADF80010F9D2C4F80C51C4F81051DF
:10BC50007648C01D09F0ECFE3570FFF746FF6761BE
:10BC60007549307920310860C4F80483DAE770B58B
:10BC7000050000D1FFDF4FF080424FF0FF30C2F8E7
:10BC800008030021C2F80011C2F80411C2F80C1117
:10BC9000C2F81011654C617009F0A7FE10B10120C7
:10BCA000A070607063480068C00701D009F08DFE85
:10BCB0002846BDE870402EE75C48007A002800D096
:10BCC000012070472DE9FC5F5D48D0F800905C4A88
:10BCD0005C49083211608406D4F8080100B10120E3
:10BCE000D4F8001111B14FF0010801E04FF0000845
:10BCF000D4F8041101B101210191D4F80C1101B162
:10BD000001210091D4F8101101B10121474D8A465B
:10BD100095F800B0002620B1C4F80861012009F0B0
:10BD200026FE4248C01D09F08BFE00B1FFDF01274F
:10BD3000B8F1000F10D0C4F80873E87818B1EE70AD
:10BD4000002009F014FE287A022805D10320287269
:10BD50003748022101602761019808B1C4F80461E5
:10BD6000009850B1C4F80C61287A032800D0FFDF96
:10BD70002F4806602F72FFF78CFEBAF1000F07D034
:10BD8000C4F81061287A012801D100F05DF86761DC
:10BD9000BBF1000F07D02E70287A012801D1FFF7E0
:10BDA000A4FEFFF776FE2148C01D09F05FFE24497E
:10BDB000091DC1F80090BDE8FC9F1C4810B5C01DCE
:10BDC00009F03EFE194940B1012008704FF0E02112
:10BDD000C1F80002BDE8104032E6087A012801D11E
:10BDE000FFF783FE1148BDE81040C01D09F03EBEBC
:10BDF00070B50E4CA07808B909F0DEFD012085076A
:10BE0000A861207A002603280AD100BFD5F80C01CA
:10BE100020B9002009F0FAFD0028F7D1C5F80C611F
:10BE200026724FF0FF30C5F8080370BD3C000020BB
:10BE3000340C00400C0400401805004010ED00E0F8
:10BE4000100502400100000170B5134C6079F0B19B
:10BE5000012803D0A179401E814218DA09F0B9FD0A
:10BE6000054609F04DFF6179012902D9A179491CE4
:10BE7000A1710DB1216900E0E168411A022902DADD
:10BE800011F1020FD1DC0DB1206100E0E060BDE8EE
:10BE900070402AE6C9E700003C00002010B52020D1
:10BEA00000F07FF8202000F08DF84D49202081F827
:10BEB0000004F5F7A3FA4B4908604B48D0F8041387
:10BEC00041F00101C0F80413D0F8041341F080716F
:10BED000C0F80413424901201C39C1F8000110BD0B
:10BEE00010B5202000F05DF83E480021C838016000
:10BEF000001D01603D4A481E10603B4AC2F808031D
:10BF0000384B1960C2F80001C2F860013849086076
:10BF1000BDE81040202000F055B834493548091FCD
:10BF20000860704731493348086070472D48C83869
:10BF30000160001D521E026070472C4901200860FC
:10BF4000BFF34F8F70472DE9F0412849D0F8188092
:10BF500028480860244CD4F800010025244E6F1EA8
:10BF600028B14046F5F7A8F940B9002111E0D4F80E
:10BF7000600198B14046F5F79FF948B1C4F8005107
:10BF8000C4F860513760BDE8F041202000F01AB8D5
:10BF900031684046BDE8F04118F070BDFFDFBDE8F4
:10BFA000F08100280DDB00F01F02012191404009C3
:10BFB000800000F1E020C0F88011BFF34F8FBFF385
:10BFC0006F8F7047002809DB00F01F0201219140AC
:10BFD0004009800000F1E020C0F8801270470000A6
:10BFE00020E000E0C80602400000024018050240C0
:10BFF00000040240010000010F4A12680D498A4204
:10C000000CD118470C4A12680A4B9A4206D101B566
:10C0100009F048FEFFF781FFBDE8014007490968C4
:10C020000958084706480749054A064B704700006B
:10C0300000000000BEBAFECA540000200400002028
:10C040008013002080130020F8B51D46DDE9064767
:10C050000E000AD006F08EFC2346FF1DBCB231460E
:10C060002A46009406F09BF8F8BDD01922461946DE
:10C0700018F038FC2046F8BD70B50D460446102176
:10C0800018F0AFFC258117206081A07B40F00A00EA
:10C09000A07370BD4FF6FF720A80014602200AF0BD
:10C0A00047B8704700897047827BD30701D1920758
:10C0B00003D4808908800020704705207047827B68
:10C0C000920700D58181704701460020098841F61A
:10C0D000FE52114200D00120704700B50346807B1C
:10C0E000C00701D0052000BD59811846FFF7ECFFBD
:10C0F000C00703D0987B40F004009873987B40F011
:10C1000001009873002000BD827B520700D509B161
:10C110004089704717207047827B61F3C3028273A6
:10C1200070472DE9FC5F0E460446017896460120D3
:10C1300000FA01F14DF6FF5201EA020962684FF67A
:10C14000FF7B1188594502D10920BDE8FC9FB9F158
:10C15000000F05D041F6FE55294201D00120F4E739
:10C1600041EA090111801D0014D000232B7094F8BE
:10C1700000C0052103221F464FF0020ABCF10E0F3A
:10C1800076D2DFE80CF0F909252F47646B774791E9
:10C1900093B4D1D80420D8E7616820898B7B9B07B2
:10C1A00067D517284AD30B89834247D38989172932
:10C1B00001D3814242D185F800A0A5F80100328068
:10C1C000616888816068817B21F002018173C6E02B
:10C1D000042028702089A5F801006089A5F80300D3
:10C1E0003180BCE0208A3188C01D1FFA80F84145AB
:10C1F00024D3062028702089A5F801006089A5F8BD
:10C200000300A089A5F805000721208ACDE90001D7
:10C21000636941E00CF0FF00082810D00820287066
:10C220002089A5F801006089A5F8030031806A1D06
:10C23000694604F10C0008F005F810B15EE010202A
:10C24000EDE730889DF800100844308087E00A2030
:10C2500028702089A5F80100328044E00C20287065
:10C260002089A5F801006089A5F8030031803AE033
:10C2700082E064E02189338800EB41021FFA82F8F2
:10C2800043453BD3B8F1050F38D30E222A700BEA91
:10C290004101CDE90010E36860882A467146FFF746
:10C2A000D3FEA6F800805AE04020287060893188CB
:10C2B000C01C1FFA80F8414520D32878714620F031
:10C2C0003F00123028702089A5F801006089CDE96F
:10C2D000000260882A46E368FFF7B6FEA6F80080F1
:10C2E000287840063BD461682089888037E0A0899F
:10C2F0003288401D1FFA80F8424501D204273DE0F4
:10C30000162028702089A5F801006089A5F803008F
:10C31000A089CDE9000160882A4671462369FFF7AC
:10C3200093FEA6F80080DEE718202870207A687057
:10C33000A6F800A013E061680A88920401D40527DA
:10C340001CE0C9882289914201D0062716E01E21EF
:10C35000297030806068018821F400510180B9F1B2
:10C36000000F0BD0618878230022022009F036FEEE
:10C3700061682078887006E0338003276068018850
:10C3800021EA090101803846DFE62DE9FF4F85B03B
:10C390001746129C0D001E461CD03078C10703D0F2
:10C3A00000F03F00192801D9012100E000212046BA
:10C3B000FFF7AAFEA8420DD32088A0F57F41FF39E0
:10C3C00008D03078410601D4000605D5082009B010
:10C3D000BDE8F08F0720FAE700208DF800008DF807
:10C3E000010030786B1E00F03F0C0121A81E4FF0B9
:10C3F000050A4FF002094FF0030B9AB2BCF1200F6F
:10C4000075D2DFE80CF08B10745E7468748C749CC9
:10C4100074B674BB74C974D574E2747474F274F035
:10C4200074EF74EE748B052D78D18DF80090A078A0
:10C430008DF804007088ADF8060030798DF80100A1
:10C44000707800F03F000C2829D00ADCA0F102002F
:10C45000092863D2DFE800F0126215621A621D62D9
:10C460002000122824D004DC0E281BD01028DBD199
:10C470001BE016281FD01828D6D11FE0207880078F
:10C4800001E020784007002848DAEFE02078000734
:10C49000F9E72078C006F6E720788006F3E72078F1
:10C4A0004006F0E720780006EDE72088C005EAE7BF
:10C4B00020884005E7E720880005E4E72088C004DD
:10C4C000E1E72078800729D5032D27D18DF800B02A
:10C4D000B6F8010082E0217849071FD5062D1DD34B
:10C4E00081B27078012803D0022817D102E0CAE097
:10C4F000022000E0102004228DF8002072788DF8D0
:10C500000420801CB1FBF0F2ADF8062092B2424349
:10C510008A4203D10397ADF80890A7E07AE020782B
:10C52000000777D598B282088DF800A0ADF80420F6
:10C53000B0EB820F6ED10297ADF8061096E021782D
:10C54000C90667D5022D65D381B206208DF800009B
:10C55000707802285ED300BFB1FBF0F28DF80400C2
:10C56000ADF8062092B242438A4253D1ADF808900A
:10C570007BE0207880064DD5072003E02078400638
:10C580007FD508208DF80000A088ADF80400ADF834
:10C590000620ADF8081068E02078000671D5092063
:10C5A000ADF804208DF80000ADF8061002975DE0AC
:10C5B0002188C90565D5022D63D381B20A208DF883
:10C5C0000000707804285CD3C6E72088400558D561
:10C5D000012D56D10B208DF80000A088ADF8040085
:10C5E00044E021E026E016E0FFE72088000548D57A
:10C5F000052D46D30C208DF80000A088ADF804006E
:10C60000B6F803006D1FADF80850ADF80600ADF8A0
:10C610000AA02AE035E02088C00432D5012D30D1AF
:10C620000D208DF8000021E02088800429D4B6F880
:10C630000100E080A07B000723D5032D21D33078B3
:10C6400000F03F001B2818D00F208DF80000208834
:10C6500040F40050A4F80000B6F80100ADF8040062
:10C66000ED1EADF80650ADF808B003976946059881
:10C67000F5F750FC050008D016E00E208DF80000FC
:10C68000EAE7072510E008250EE0307800F03F00CB
:10C690001B2809D01D2807D00220059909F048FD64
:10C6A000208800F400502080A07B400708D5204659
:10C6B000FFF70AFDC00703D1A07B20F00400A073A0
:10C6C000284684E61FB5022806D101208DF8000017
:10C6D00088B26946F5F71EFC1FBD0000F8B51D467F
:10C6E000DDE906470E000AD006F044F92346FF1D97
:10C6F000BCB231462A46009405F051FDF8BDD01970
:10C700002246194618F0EEF82046F8BD2DE9FF4FF5
:10C710008DB09B46DDE91B57DDF87CA00C46082B4D
:10C7200005D0E06901F002F950B11020D2E028886C
:10C73000092140F0100028808AF80010022617E036
:10C74000E16901208871E2694FF420519180E1692B
:10C750008872E06942F601010181E069002181737C
:10C760002888112140F0200028808AF80010042633
:10C7700038780A900A2038704FF0020904F1180046
:10C780004D460C9001F095FBB04681E0BBF1100FD7
:10C790000ED1022D0CD0A9EB0800801C80B2022122
:10C7A000CDE9001005AB52461E990D98FFF796FF94
:10C7B000BDF816101A98814203D9F74800790F90F6
:10C7C00004E003D10A9808B138702FE04FF002015D
:10C7D000CDE900190DF1160352461E990D98FFF789
:10C7E0007DFF1D980088401B801B83B2C6F1FF00AF
:10C7F000984200D203461E990BA8D9B15FF00002FF
:10C80000DDF878C0CDE9032009EB060189B2CDE956
:10C8100001C10F980090BDF8161000220D9801F08C
:10C82000CBFB387070B1C0B2832807D0BDF81600BA
:10C8300020833AE00AEB09018A19E1E7022011B0EE
:10C84000BDE8F08FBDF82C00811901F0FF08022D22
:10C850000DD09AF80120424506D1BDF82010814242
:10C8600007D0B8F1FF0F04D09AF801801FE08AF8D2
:10C870000180C94800680178052902D1BDF8161069
:10C88000818009EB08001FFA80F905EB080085B2EA
:10C89000DDE90C1005AB0F9A01F00EFB28B91D98CD
:10C8A0000088411B4145BFF671AF022D13D0BBF18B
:10C8B000100F0CD1A9EB0800801C81B20220CDE939
:10C8C000000105AB52461E990D98FFF707FF1D9812
:10C8D0000580002038700020B1E72DE9F8439C4620
:10C8E000089E13460027B26B9AB3491F8CB2F18F92
:10C8F000A1F57F45FF3D05D05518AD882944891D18
:10C900008DB200E000252919B6F83C800831414578
:10C9100020D82A44BCF8011022F8021BBCF80310EE
:10C9200022F8021B984622F8024B914606F010F8B6
:10C930004FF00C0C41464A462346CDF800C005F0A6
:10C94000FAFBF587B16B00202944A41D214408801F
:10C9500003E001E0092700E083273846BDE8F883BB
:10C9600010B50B88848F9C420CD9846BE018048826
:10C9700044B1848824F40044A41D23440B80106037
:10C98000002010BD0A2010BD2DE9F0478AB0002517
:10C99000904689468246ADF8185007274BE0059827
:10C9A00006888088000446D4A8F8006007A801958E
:10C9B00000970295CDE903504FF4007300223146F1
:10C9C000504601F0F9FA04003CD1BDF81800ADF86A
:10C9D0002000059804888188B44216D10A0414D432
:10C9E00001950295039521F400410097049541F4C7
:10C9F000804342882146504601F0B4F804000BD130
:10CA00000598818841F40041818005AA08A948461B
:10CA1000FFF7A6FF0400DCD000970598029501956A
:10CA2000039504950188BDF81C300022504601F0A2
:10CA300099F80A2C06D105AA06A94846FFF790FFE7
:10CA40000400ACD0ADF8185004E00598818821F4BA
:10CA50000041818005AA06A94846FFF781FF00280A
:10CA6000F3D00A2C03D020460AB0BDE8F08700209E
:10CA7000FAE710B50C46896B86B051B10C218DF8E0
:10CA80000010A18FADF80810A16B01916946FAF76B
:10CA900040FB00204FF6FF71A063E187A08706B03E
:10CAA00010BD2DE9F0410D460746896B0020069E1A
:10CAB0001446002911D0012B0FD1324629463846A1
:10CAC000FFF762FF002808D1002C06D03246294625
:10CAD0003846BDE8F04100F038BFBDE8F0812DE9EF
:10CAE000FC411446DDE9087C0E46DDE90A15521DBD
:10CAF000BCF800E092B2964502D20720BDE8FC8166
:10CB0000ACF8002017222A70A5F80160A5F80330C0
:10CB10000522CDE900423B462A46FFF7DFFD002013
:10CB2000ECE770B50C4615464821204617F07BFF10
:10CB300004F1080044F81C0F00204FF6FF71E0617B
:10CB400061842084A5841720E08494F82A0040F0B2
:10CB50000A0084F82A0070BD4FF6FF720A80014671
:10CB6000032009F0E5BA30B585B00C460546FFF75D
:10CB700080FFA18E284629B101218DF80010694659
:10CB8000FAF7C7FA0020E0622063606305B030BDA9
:10CB9000B0F84000704700005800002090F8462090
:10CBA000920703D4408808800020F3E70620F1E7CD
:10CBB00090F846209207EDD5A0F84410EAE7014628
:10CBC000002009880A0700D5012011F0F00F01D0DC
:10CBD00040F00200CA0501D540F004008A0501D5E5
:10CBE00040F008004A0501D540F010000905D1D5F4
:10CBF00040F02000CEE700B5034690F84600C0079D
:10CC000001D0062000BDA3F842101846FFF7D7FF59
:10CC100010F03E0F05D093F8460040F0040083F872
:10CC2000460013F8460F40F001001870002000BDC8
:10CC300090F84620520700D511B1B0F84200A9E79C
:10CC40001720A7E710F8462F61F3C3020270A1E78F
:10CC50002DE9FF4F9BB00E00DDE92B34DDE929788B
:10CC6000289D24D02878C10703D000F03F00192860
:10CC700001D9012100E000212046FFF7D9FFB04291
:10CC800015D32878410600F03F010CD41E290CD0A2
:10CC9000218811F47F6F0AD13A8842B1A1F57F4211
:10CCA000FF3A04D001E0122901D1000602D5042088
:10CCB0001FB0C5E5F9491D984FF0000A08718DF8BD
:10CCC00018A08DF83CA00FAA0A60ADF81CA0ADF822
:10CCD00050A02978994601F03F02701F5B1C04F1B7
:10CCE000180C4FF0060E4FF0040BCDF858C01F2A59
:10CCF0007ED2DFE802F07D7D107D267DAC7DF47D67
:10CD0000F37DF27DF17DF47DF07D7D7DEF7DEE7D27
:10CD10007D7D7D7DED0094F84610B5F80100890712
:10CD200001D5032E02D08DF818B022E34FF4006134
:10CD3000ADF85010608003218DF83C10ADF8400034
:10CD4000D8E2052EEFD1B5F801002083ADF81C0024
:10CD5000B5F80310618308B1884201D901207FE151
:10CD60000020A07220814FF6FF702084169801F0F9
:10CD7000A0F8052089F800000220029083460AAB43
:10CD80001D9A16991B9801F097F890BB9DF82E00FC
:10CD9000012804D0022089F80100102003E00120BE
:10CDA00089F8010002200590002203A90BA807F0D2
:10CDB00049FAE8BB9DF80C00059981423DD13A88BB
:10CDC000801CA2EB0B01814237DB02990220CDE9E6
:10CDD00000010DF12A034A4641461B98FFF77EFCED
:10CDE00002980BF1020B801C80B217AA03A901E084
:10CDF000A0E228E002900BA807F024FA02999DF81F
:10CE00000C00CDE9000117AB4A4641461B98FFF7DD
:10CE100065FC9DF80C100AAB0BEB01001FFA80FBC0
:10CE200002981D9A084480B2029016991B9800E05F
:10CE300003E001F041F80028B6D0BBF1020F02D0A8
:10CE4000A7F800B053E20A208DF818004FE2002145
:10CE50000391072EFFF467AFB5F801002083ADF80A
:10CE60001C00B5F80320628300283FF477AF90429E
:10CE70003FF674AF0120A072B5F8050020810020B4
:10CE8000A073E06900F052FD78B9E1690120887172
:10CE9000E2694FF420519180E1698872E06942F6BD
:10CEA00001010181E06900218173F01F20841E9837
:10CEB000606207206084169800F0FBFF072089F865
:10CEC00000000120049002900020ADF82A0028E024
:10CED0001DE2A3E13AE1EAE016E2AEE086E049E0D5
:10CEE0000298012814D0E0698079012803D1BDF8A7
:10CEF0002800ADF80E00049803ABCDE900B04A4617
:10CF000041461B98FFF7EAFB0498001D80B204908D
:10CF1000BDF82A00ADF80C00ADF80E00059880B2FF
:10CF200002900AAB1D9A16991B9800F0C5FF28B90C
:10CF300002983988001D05908142D1D202980128BB
:10CF400081D0E0698079012805D0BDF82810A1F5CD
:10CF50007F40FF3803D1BDF82800ADF80E000498DB
:10CF600003ABCDE900B04A4641461B98FFF7B6FB3C
:10CF70000298BBE1072E02D0152E7FF4D4AEB5F88F
:10CF800001102183ADF81C10B5F80320628300293D
:10CF90003FF4E4AE91423FF6E1AE0121A1724FF0C1
:10CFA000000BA4F808B084F80EB0052E07D0C0B26C
:10CFB000691DE26907F027F900287FF444AF4FF6B6
:10CFC000FF70208401A906AA14A8CDF800B081E85A
:10CFD00085032878214600F03F031D9A1B98FFF730
:10CFE00095FB8246208BADF81C0080E10120032ECA
:10CFF000C3D14021ADF85010B5F801102183ADF830
:10D000001C100AAAB8F1000F00D00023CDE90203DA
:10D0100004921D98CDF80480009038880022401EAC
:10D0200083B21B9800F0C8FF8DF8180090BB0B204E
:10D0300089F80000BDF8280037E04FF0010C052EFC
:10D040009BD18020ADF85000B5F801102183B5F8D0
:10D0500003002084ADF81C10B0F5007F03D9072031
:10D060008DF8180085E140F47C4222840CA8B8F1C8
:10D07000000F00D00023CDE90330CDE9018C1D98CD
:10D0800000903888401E83B21B9800F095FF8DF801
:10D09000180028B18328A8D10220BDE05800002044
:10D0A0000D2189F80010BDF83000401C1EE1032E50
:10D0B00004D248067FF537AE002017E1B5F801101D
:10D0C000ADF81C102878400602D58DF83CE002E04F
:10D0D00007208DF83C004FF000080320CDE902083E
:10D0E0001E9BCDF810801D980193A6F1030B0090B4
:10D0F0001FFA8BF342461B9800F034FD8DF81800A0
:10D100008DF83C80297849060DD52088C00506D5C4
:10D11000208BBDF81C10884201D1C4F82480404601
:10D120008DF81880E2E0832801D14FF0020A4FF415
:10D130008070ADF85000BDF81C002083A4F820B02A
:10D140001E986062032060841321CCE0052EFFF45A
:10D15000EAADB5F80110ADF81C10A28F62B3A2F5CC
:10D160007F43FE3B28D008228DF83C204FF0000B77
:10D170000523CDE9023BDDF878C0CDF810B01D9A4B
:10D1800080B2CDF804C040F400430092B5F803200B
:10D190001B9800F0E7FC8DF83CB04FF400718DF85F
:10D1A0001800ADF85010832810D0F8B1A18FA1F568
:10D1B0007F40FE3807D0DCE00B228DF83C204FF694
:10D1C000FE72A287D2E7A4F83CB0D2E000942B46CE
:10D1D00031461E9A1B98FFF780FB8DF8180008B1A6
:10D1E00083284BD1BDF81C00208355E700942B46C3
:10D1F00031461E9A1B98FFF770FB8DF81800E8BBAC
:10D20000E18FA06B0844811D8DE8820343888288EA
:10D2100001881B98FFF763FC824668E095F801805F
:10D22000022E70D15FEA080002D0B8F1010F6AD176
:10D2300009208DF83C0007A800908DF840804346F7
:10D24000002221461B98FFF72CFC8DF842004FF07E
:10D25000000B8DF843B050B9B8F1010F12D0B8F1FE
:10D26000000F04D1A18FA1F57F40FF380AD0A08F15
:10D2700040B18DF83CB04FF4806000E037E0ADF88D
:10D2800050000DE00FA91B98F9F743FF82468DF877
:10D290003CB04FF48060ADF85000BAF1020F06D0F8
:10D2A000FC480068C07928B18DF8180027E0A4F880
:10D2B000188044E0BAF1000F03D081208DF81800E7
:10D2C0003DE007A800904346012221461B98FFF746
:10D2D000E8FB8DF8180021461B98FFF7CAFB9DF864
:10D2E000180020B9192189F80010012038809DF814
:10D2F0003C0020B10FA91B98F9F70BFF8246BAF149
:10D30000000F33D01BE018E08DF818E031E02078F2
:10D31000000712D5012E10D10A208DF83C00E088BC
:10D32000ADF8400003201B9908F002FF0820ADF87B
:10D330005000C1E648067FF5F6AC4FF0040A20889D
:10D34000BDF8501008432080BDF8500080050BD573
:10D35000A18FA1F57F40FE3806D11E98E062289883
:10D360002063A6864FF0030A5046A1E49DF81800FA
:10D3700078B1012089F80000297889F80110BDF8FA
:10D380001C10A9F802109DF8181089F80410052047
:10D3900038802088BDF8501088432080E4E72DE9CC
:10D3A000FF4F8846087895B0012181404FF209006F
:10D3B000249C0140ADF820102088DDF88890A0F56D
:10D3C0007F424FF0000AFF3A06D039B1000705D579
:10D3D000012019B0BDE8F08F0820FAE7239E4FF036
:10D3E000000B0EA886F800B018995D460988ADF8C4
:10D3F0003410A8498DF81CB0179A0A718DF838B00E
:10D40000086098F8000001283BD0022809D00328C2
:10D410006FD1307820F03F001D303070B8F8040034
:10D42000E08098F800100320022904D1317821F01F
:10D430003F011B31317094F84610090759D505ABEF
:10D44000B9F1000F13D0002102AA82E80B000720D7
:10D45000CDE90009BDF83400B8F80410C01E83B24D
:10D460000022159800F0A8FD0028D1D101E0F11CA0
:10D47000EAE7B8F80400A6F80100BDF81400C01CE3
:10D4800004E198F805108DF81C1098F804000128A4
:10D4900006D04FF4007A02282CD00328B8D16CE1D2
:10D4A0002188B8F8080011F40061ADF8201020D0F0
:10D4B00017281CD3B4F84010814218D3B4F8441094
:10D4C000172901D3814212D1317821F03F01C91CC3
:10D4D0003170A6F801000321ADF83410A4F844001F
:10D4E00094F8460020F0020084F8460065E1052526
:10D4F0007EE177E1208808F1080700F4FE60ADF8CE
:10D50000200010F0F00F1BD010F0C00F03D03888AF
:10D51000228B9042EBD199B9B878C00710D0B96886
:10D520000720CDE902B1CDF804B00090CDF810B0DD
:10D53000FB88BA883988159800F014FB0028D6D1EA
:10D540002398BDF82010401C80294ED006DC1029FD
:10D550000DD020290BD0402987D124E0B1F5807F60
:10D560006ED051457ED0B1F5806F97D1DEE0C80610
:10D5700001D5082000E0102082460DA907AA052049
:10D58000CDE902218DF83800ADF83CB0CDE9049624
:10D5900008A93888CDE9000153460722214615988D
:10D5A000FFF7B4F8A8E09DF81C2001214FF00A0A0B
:10D5B000002A9BD105ABB9F1000F00D00020CDE9C6
:10D5C00002100720CDE90009BDF834000493401E85
:10D5D00083B2218B0022159800F0EEFC8DF81C0020
:10D5E0000B203070BDF8140020E09DF81C200121B4
:10D5F0004FF00C0A002A22D113ABB9F1000F00D072
:10D600000020CDE902100720CDE900090493BDF800
:10D610003400228C401E83B2218B159800F0CCFC84
:10D620008DF81C000D203070BDF84C00401CADF88A
:10D63000340005208DF83800208BADF83C00BCE0AC
:10D640003888218B88427FF452AF9DF81C004FF040
:10D65000120A00281CD1606AA8B1B878C0073FF44C
:10D6600046AF00E018E0BA680720CDE902B2CDF875
:10D6700004B00090CDF810B0FB88BA88159800F07F
:10D6800071FA8DF81C00132030700120ADF83400C1
:10D6900093E00000580000203988208B8142D2D1CD
:10D6A0009DF81C004FF0160A0028A06B08D0E0B3CC
:10D6B0004FF6FF7000215F46ADF808B0019027E0FB
:10D6C00068B1B978C907BED1E18F0DAB0844821D9E
:10D6D00003968DE80C0243888288018809E0B878B7
:10D6E000C007BCD0BA680DAB03968DE80C02BB88AE
:10D6F000FA881598FFF7F3F905005ED0072D72D070
:10D7000076E0019005AA02A92046FFF729F9014613
:10D71000E28FBDF80800824201D00029F1D0E08FED
:10D72000A16B084407800198E08746E09DF81C0043
:10D730004FF0180A40B1208BC8B1388820832146A9
:10D740001598FFF796F938E004F118000090237E51
:10D75000012221461598FFF7A4F98DF81C00002836
:10D76000EDD1192030700120ADF83400E7E7052530
:10D7700021461598FFF77DF93AE0208800F4007003
:10D78000ADF8200050452DD1A08FA0F57F41FE3986
:10D7900001D006252CE0D8F808004FF0160A48B151
:10D7A000A063B8F80C10A1874FF6FF71E187A0F8CD
:10D7B00000B002E04FF6FF70A087BDF8200030F403
:10D7C0007F611AD0782300220320159908F006FC07
:10D7D00098F8000020712088BDF8201008432080B0
:10D7E0000EE000E007252088BDF820108843208047
:10D7F000208810F47F6F1CD03AE02188814321807B
:10D800009DF8380020B10EA91598F9F782FC05465D
:10D810009DF81C000028EBD086F801A00120307094
:10D82000208B70809DF81C0030710520ADF834000D
:10D83000DEE7A18EE1B118980DAB0088ADF8340099
:10D840002398CDE90304CDE90139206B0090E36A08
:10D85000179A1598FFF7FCF9054601208DF8380056
:10D860000EA91598F9F755FC00B10546A4F834B097
:10D8700094F8460040070AD52046FFF7A0F910F0BB
:10D880003E0F04D114F8460F20F0040020701898C1
:10D89000BDF83410018028469BE500B585B003280B
:10D8A00006D102208DF8000088B26946F9F731FCF4
:10D8B00005B000BD10B5384C0B782268012B02D0A2
:10D8C000022B2AD111E013780BB1052B01D10423CF
:10D8D000137023688A889A802268CB88D380226854
:10D8E0000B891381498951810DE08B8893802268CF
:10D8F000CB88D38022680B8913814B8953818B8914
:10D900009381096911612168F9F703FC22680021FC
:10D910000228117003D0002800D0812010BD832080
:10D9200010BD806B002800D001207047817801294C
:10D9300009D10088B0F5205F03D042F6010188428A
:10D9400001D10020704707207047F0B587B0002450
:10D9500015460E460746ADF8184011E005980088B8
:10D96000288005980194811DCDE902410721049486
:10D970000091838842880188384600F0F3F830B976
:10D9800005AA06A93046FEF7EBFF0028E6D00A28D4
:10D9900000D1002007B0F0BD5800002010B58B78F2
:10D9A00083B102789A4205D10B885BB102E08B7992
:10D9B000091D4BB18B789A42F9D1B0F801300C882F
:10D9C000A342F4D1002010BD812010BD072826D02D
:10D9D00012B1012A27D103E0497801F0070102E0E2
:10D9E0004978C1F3C20105291DD2DFE801F003180F
:10D9F000080C12000AB10320704702207047042867
:10DA00000DD250B10DE0052809D2801E022808D39E
:10DA100003E0062803D0032803D005207047002028
:10DA200070470F20704781207047C0B282060BD428
:10DA3000000607D5FE48807A4143C01D01EBD000A7
:10DA400080B27047084670470020704770B5138851
:10DA50000B800B781C0625D5F54CA47A844204D89B
:10DA600043F010000870002070BD956800F00706B4
:10DA700005EBD0052D78F54065F304130B70137892
:10DA8000D17803F0030341EA032140F20123B1FB03
:10DA9000F3F503FB15119268E41D00FB012000EB78
:10DAA000D40070BD906870BD37B51446BDF8041041
:10DAB00011809DF804100A061ED5C1F30013DC493D
:10DAC000A568897A814208D8FE2811D1C91DC908E4
:10DAD0005A42284616F07DFF0AE005EBD00100F01F
:10DAE0000702012508789540A84393401843087021
:10DAF000207820F0100020703EBD2DE9F04107464F
:10DB0000C81C0E4620F00300B04202D08620BDE8BB
:10DB1000F081C74D002034462E60AF802881AA7264
:10DB2000E8801AE0E988491CE980810614D4E1788C
:10DB300000F0030041EA002040F20121B0FBF1F2C5
:10DB400001FB12012068FFF770FF2989084480B2A9
:10DB50002881381A3044A0600C3420784107E1D481
:10DB60000020D4E72DE9FF4F89B01646DDE9168A7B
:10DB70000F46994623F44045084600F00DFB04008B
:10DB80000FD0099804F078FD0290207800060AD59D
:10DB9000A748817A0298814205D887200DB0BDE858
:10DBA000F08F0120FAE7224601A90298FFF74EFF05
:10DBB000834600208DF80C004046B8F1070F1AD0BC
:10DBC00001222146FFF702FF0028E7D12078400616
:10DBD00011D502208DF80C00ADF81070BDF80400CE
:10DBE000ADF81200ADF814601898ADF81650CDF8E5
:10DBF0001CA0ADF818005FEA094004D500252E46A8
:10DC0000A84601270CE02178E07801F0030140EA02
:10DC1000012040F20121B0FBF1F2804601FB1287A6
:10DC20005FEA494009D5B84507D1A178207901F0CC
:10DC3000030140EA0120B04201D3BE4201D90720CE
:10DC4000ACE7A8191FFA80F9B94501D90D20A5E75D
:10DC50009DF80C0028B103A90998F9F758FA002893
:10DC60009CD1B84507D1A0784FEA192161F3010092
:10DC7000A07084F804901A9800B10580199850EAB1
:10DC80000A0027D0199830B10BEB06002A461999E3
:10DC900016F028FE0EE00BEB06085746189E099872
:10DCA00004F056FE2B46F61DB5B2394642460095A5
:10DCB00004F041FA224601A90298FFF7C7FE9DF839
:10DCC0000400224620F010008DF80400DDE9011068
:10DCD000FFF7EAFE002061E72DE9FF4FDFF85091E2
:10DCE00082461746B9F80610D9F8000001EB410149
:10DCF00000EB810440F20120B2FBF0F185B000FBA3
:10DD000011764D46DDF84C8031460698FFF78DFEC2
:10DD100029682A898B46611A0C3101441144AB8869
:10DD200089B28B4202D8842009B038E70699CDB277
:10DD3000290603D5A90601D50620F5E7B9F806C0DE
:10DD40000CF1010C1FFA8CFCA9F806C0149909B15A
:10DD5000A1F800C0A90602D5C4F8088007E0104465
:10DD600080B2A9F80800191A01EB0B00A060224646
:10DD7000FE200699FFF798FEE77026712078390A91
:10DD800061F30100320AA17840F0040062F301015E
:10DD9000A17020709AF802006071BAF80000E0806B
:10DDA00000262673280602D599F80A7000E001279C
:10DDB000A80601D54FF000084D4600244FF0070992
:10DDC0000FE0CDE902680196CDF800900496E9884D
:10DDD0002046129B089AFFF7C5FE0028A4D1641CB8
:10DDE000E4B2BC42EDD300209EE72DE9F047804627
:10DDF00000F0D2F9070005D0002644460C4D40F251
:10DE0000012919E00120BDE8F087204600F0C4F99F
:10DE10000278C17802F0030241EA0222B2FBF9F370
:10DE200009FB13210068FFF700FE304486B201E0D1
:10DE3000F8050020641CA4B2E988601E8142E4DC7D
:10DE4000A8F10100E8802889801B28810020387013
:10DE5000D9E710B5144631B1491E218004F00CFCFD
:10DE6000A070002010BD012010BD10B5D24904469D
:10DE70000088CA88904201D30A2010BD096800EBCF
:10DE8000400001EB80025079A072D0882081917807
:10DE9000107901F0030140EA0120A081A078E11C83
:10DEA000FFF7D4FD20612088401C2080E080002006
:10DEB00010BD0121018270472DE9FF4F85B04FF65B
:10DEC000FF788246A3F8008048681F460D46807898
:10DED0008DF8060048680088ADF8040000208DF831
:10DEE0000A00088A0C88A04200D304462C8241E034
:10DEF000288A401C2882701D6968FFF74FFDB8BB57
:10DF00003988414501D1601E38806888A04236D3E7
:10DF1000B178307901F0030140EA012901A9701DAF
:10DF2000FFF73CFD20BB298941452CD0002231461A
:10DF30000798FFF74BFDD8B92989494518D1E968F9
:10DF40000391B5F80AC0D6F808B05046CDF800C025
:10DF500004F0FEFCDDF800C05A460CF1070C1FFA75
:10DF60008CFC4B460399CDF800C004F0AEF850B1DC
:10DF7000641CA4B2204600F00FF90600B8D1641E5C
:10DF80002C820A20D0E67C807079B871F088B88045
:10DF90003178F07801F0030140EA01207881A7F898
:10DFA0000C90504604F068FB324607F10801FFF779
:10DFB0004DFD38610020B7E62DE9FF4F87B081465F
:10DFC0001C469246DDF860B0DDF85480089800F0F9
:10DFD000E3F805000CD0484604F04EFB297809060A
:10DFE00008D57549897A814204D887200BB0D6E5D7
:10DFF0000120FBE7CAF309062A4601A9FFF726FD1F
:10E000000746149807281CD000222946FFF7DEFC9B
:10E010000028EBD12878400613D501208DF80800A0
:10E020000898ADF80C00BDF80400ADF80E00ADF88E
:10E030001060ADF8124002A94846F9F768F80028C8
:10E04000D4D12978E87801F0030140EA0121AA78C7
:10E05000287902F0030240EA0220564507D0B1F5C4
:10E06000007F04D9611E814201DD0B20BEE786429C
:10E0700001D90720BAE7801B85B2A54200D9254601
:10E08000BBF1000F01D0ABF80050179818B1B919C7
:10E090002A4616F027FCB8F1000F0DD03E44484642
:10E0A0004446169F04F066FC2146FF1DBCB2324672
:10E0B0002B46009404F073F8002097E72DE9F04117
:10E0C00007461D461646084600F066F804000BD0C9
:10E0D000384604F0D1FA2178090607D53649897AFD
:10E0E000814203D8872012E5012010E522463146FF
:10E0F000FFF7ACFC65B12178E07801F0030140EA5C
:10E100000120B0F5007F01D8012000E00020287038
:10E110000020FCE42DE9F04107461D46164608465E
:10E1200000F03AF804000BD0384604F0A5FA217844
:10E13000090607D52049897A814203D88720E6E479
:10E140000120E4E422463146FFF7AEFCFF2D14D057
:10E150002178E07801F0030240EA022040F2012237
:10E16000B0FBF2F302FB130015B900F2012080B2FC
:10E17000E070000A60F3010121700020C7E410B5CF
:10E180000C4600F009F828B1C18821804079A070C0
:10E19000002010BD012010BD0749CA88824209D362
:10E1A00040B1096800EB40006FF00B0202EB800009
:10E1B0000844704700207047F805002010B508F0AB
:10E1C00079F9F4F773FB07F0FFFFBDE8104008F0A2
:10E1D000C7B8202834BF012000207047012303FA6C
:10E1E00000F04FF0A042002914BFC2F80C05C2F89D
:10E1F000080570474FF0A041012202FA00F0C1F873
:10E200001805704770B50346002002466FF02F05D1
:10E210000EE09C5CA4F130060A2E02D34FF0FF30D2
:10E2200070BD00EB800005EB4000521C2044D2B2D0
:10E230008A42EED370BD30B50A230BE0B0FBF3F495
:10E2400003FB1404B0FBF3F08D183034521E05F8B4
:10E25000014CD2B2002AF1D130BD30B500234FF6C7
:10E26000FF7510E0040A44EA002084B2C85C6040F4
:10E27000C0F30314604005EA00344440E0B25B1C84
:10E2800084EA40109BB29342ECD330BD2DE9F041BB
:10E29000FE4B0026012793F860501C7893F864C069
:10E2A000B8B183F88D40A3F88E1083F88C2083F8E2
:10E2B0008A70BCF1000F0CBF83F8906083F8905017
:10E2C000F3488068008804F043FBBDE8F04103F0A8
:10E2D000D9BF4FF6FF7083F88D40A3F88E0083F806
:10E2E0008C2083F88A70BCF1000F14BF83F8905023
:10E2F00083F89060BDE8F08170B5E54E0446306863
:10E3000090F898100025012919D090F89210012951
:10E3100024D090F8681001292AD090F88A10012999
:10E320001CBF002070BD657017212170D0F88C10C3
:10E330006160B0F89010218180F88A5016E0657015
:10E340001C212170D0F899106160D0F89D10A16057
:10E3500090F8A110217380F8985007E065700721AC
:10E360002170D0F89410616080F89250012070BD47
:10E3700065701421217000F16A012022201D16F021
:10E38000B1FA01212172306880F86850BF48B0F8B6
:10E390006C20A0F89420B268537B80F8963080F807
:10E3A0009210108804F0D4FA03F07BFFDEE7B8483F
:10E3B000006890F86810002914BFB0F86C004FF6A0
:10E3C000FF70704770B5B24C06462068002808BF41
:10E3D000FFDF0025206845706660002808BFFFDF6A
:10E3E0002068417800291CBFFFDF70BDA42116F012
:10E3F0001AFB2068FF2101707F2180F8361013215D
:10E400004184282180F86510012180F8581080F897
:10E410005D5008F02DFDBDE8704007F002BF9C493B
:10E420000968097881420CBF012000207047984894
:10E43000006890F82200C0F34000704794480068DC
:10E4400090F8220000F0010070479148006890F8B1
:10E450002200C0F3001070472DE9F0438C48D0F83B
:10E4600000C09CF82400BCF82240C0F38001C0F337
:10E470004002114400F001000144C4F30010F0B167
:10E48000132C17D009DC102C02BF824830F8110081
:10E49000BDE8F083122C0DD008E0152C08BF7E4893
:10E4A00009D01D2C04BF7D48BDE8F083FFDF0020AC
:10E4B000BDE8F0837A4830F81100BDE8F0839CF89D
:10E4C0005A209CF85B002E2600234FF47A774FF0F9
:10E4D00014084FF04009022A04BF4AF2D745B5FBA1
:10E4E000F7F510D0012A04BF4AF22F75B5FBF7F5F6
:10E4F00010D04AF62315B5FBF7F5082A08BF4E469B
:10E5000013D0042A18D01E46082A0ED0042A13D08D
:10E51000022A49D003F12806042A0FD0082A1CBF7A
:10E520004FF01908082204D00AE04FF0140806F54D
:10E53000A8764FF0400203E006F5A8764FF01002EF
:10E5400018FB026212FB0152C1EB0111554D01EBA8
:10E55000810105EB8101114414F0010F4FF4C872E1
:10E560004FF4BF7504BFC4F34006002E6FD0C4F350
:10E57000400601F5A571EEB1082804BF17464026F4
:10E580000CD0042804BF2F46102607D0022807BF4E
:10E5900003F11807042603F12807082606EB86086E
:10E5A00008EB86163E441BE003F118064FF01908ED
:10E5B0000422C5E7082804BF164640270CD00428CB
:10E5C00004BF2E46102707D0022807BF03F1180604
:10E5D000042703F12806082707EB871706EB8706B1
:10E5E00031449C31082804BF164640270CD004282B
:10E5F00004BF2E46102707D0022807BF03F11806D4
:10E60000042703F128060827C7EBC70707EB4707CE
:10E6100006EB47063144983114F0010F18D0082852
:10E6200008BF40200CD0042804BF2A46102007D081
:10E63000022807BF03F11802042003F12802082072
:10E6400000EB400303EB0010104401444FE052E0A4
:10E65000082804BF144640260CD0042804BF2C46CA
:10E66000102607D0022807BF03F11804042603F17F
:10E670002804082606EB8616BCF83CC004EB86048A
:10E680002144BCF1EB0F32D90EE00000040600205B
:10E6900060000020904E0200984E02008E89130008
:10E6A000884E0200D4FEFFFF44F255240CF10B0CFF
:10E6B0000CFB04FC4FEA9C5C082807D0042802D01D
:10E6C000022805D008E02A46102008E0402006E095
:10E6D00003F11802042002E003F12802082000EBF5
:10E6E000801002EB800000F5A5700CFB001101F218
:10E6F0006510BDE8F08301F5A574082804BF16462F
:10E7000040210CD0042804BF2E46102107D0022837
:10E7100007BF03F11806042103F12806082101EBC5
:10E720008111BCF844C006EB81012144BCF1EB0F20
:10E73000DDD944F255240CF10B0C0CFB04FC4FEA20
:10E740009C5C0828C2D00428BDD00228C4D1BFE7F1
:10E75000FE4840F271210068806A48437047FB48D8
:10E76000006890F83500002818BF0120704710B5E8
:10E77000F74C207B022818BF032808D1207D04F124
:10E7800015010DF07EF908281CBF012010BD207B6B
:10E79000002816BF022800200120BDE8104008F024
:10E7A00045BFEB4908737047E849096881F83000B4
:10E7B00070472DE9F047E54C2168087B002816BF1B
:10E7C000022800200120487301F10E0108F018FF13
:10E7D0002168087B022816BF03280122002281F845
:10E7E0002F204FF0080081F82D00487B01F10E0327
:10E7F0004FF001064FF00007012804BF5B7913F0CA
:10E80000C00F0AD001F10E03012804D1587900F09D
:10E81000C000402801D0002000E0012081F82E0037
:10E82000002A04BF91F8220010F0040F07D0087DE1
:10E8300001F115010DF025F9216881F82D002068FE
:10E84000476006F095F82168C14D4FF000098860D7
:10E8500095F82D000DF031F9804695F82F0000282D
:10E8600018BFB8F1000F04D095F82D000CF0ECFEA5
:10E8700068B195F8300000281CBF95F82E000028DC
:10E880001DD0697B05F10E0001290ED012E06E73D8
:10E890004A4605F10E01404608F007FF95F82D1095
:10E8A00005F10E000DF000FA09E0407900F0C0001B
:10E8B000402831D0394605F10E0008F02DFF2068C0
:10E8C000C77690F8220010F0040F08BFBDE8F0876B
:10E8D000002795F82D000CF06BFF050008BFBDE880
:10E8E000F08710210DF073FF002818BFBDE8F087F6
:10E8F00020683A4600F11C01C676284608F0D5FE8D
:10E90000206800F11C0160680EF07EFA6068BDE8C6
:10E91000F04701210EF093BA0DF003FA4A4605F1D3
:10E920000E0108F0C2FECAE7884A1268137B037022
:10E93000D2F80E000860508A8880704778B5844904
:10E940000446824D407B08732A68207810706088E6
:10E95000ADF8000080B200F00101C0F3400341EACD
:10E960004301C0F3800341EA8301C0F3C00341EADD
:10E97000C301C0F3001341EA0311C0F3401341EA9D
:10E980004311C0F3801041EA80105084E07D0128DB
:10E9900008BF012603D0022814BFFFDF0226286823
:10E9A00080F85A60607E012808BF012603D0022843
:10E9B00014BFFFDF0226286880F85B60217B80F8A7
:10E9C0002410418C1D290CBF002161688162617D8A
:10E9D00080F83510A17B002916BF022900210121F2
:10E9E0000175D4F80F10C0F81510B4F81310A0F882
:10E9F0001910A17EB0F8662061F30302A0F866202A
:10EA0000E17E012918BF002180F83410002078BD74
:10EA10004E480068408CC0F3001131B1C0F3800053
:10EA2000002804BF1F20704702E0C0F3400109B175
:10EA30000020704710F0010F14BFEE20FF20704738
:10EA400042480068408CC0F3001119B1C0F3800047
:10EA500028B102E0C0F3400008B100207047012057
:10EA600070473A49002209680A664B8C1D2B0CBF7F
:10EA700081F8642081F8640070470023334A1268EB
:10EA800082F859309164A2F84C00012082F85900B4
:10EA900070472E4A0023126882F85830A2F85400BA
:10EAA0000120116582F8580070472849096881F8EB
:10EAB0005D0070472548006890F95D007047234865
:10EAC000006890F82200C0F3401070471F480068AB
:10EAD00090F82200C0F3C0007047012070471B4827
:10EAE000006890F85B00704770B508F0A2F908F074
:10EAF00081F908F04EF808F0D7F8144C2068016E40
:10EB0000491C016690F83300002530B108F0B0F9D7
:10EB100007F087FB206880F833502068457090F834
:10EB2000371021B1BDE87040042009F049BA90F8CF
:10EB3000641001B3006E81421DD8042009F040FA30
:10EB4000206890F8220010F0010F03E06000002020
:10EB50000406002007D0A06843220188BDE8704069
:10EB60000120FFF793BBBDE8704043224FF6FF71D1
:10EB70000020FFF78BBBBDE87040002009F020BAF1
:10EB80002DE9F047FF4E814682B030680F464FF0C6
:10EB90000008458C15F0030F10D015F0010F05F09B
:10EBA000020005D0002808BF4FF0010806D004E09D
:10EBB000002818BF4FF0020800D1FFDF4FF0000A15
:10EBC000544615F0010F05F002000DD080B915F084
:10EBD000040F0DD04AF00800002F1CBF40F00100C8
:10EBE00040F0020440D090E010B115F0040F0DD0B9
:10EBF00015F0070F10D015F0010F05F0020036D008
:10EC0000002808BF15F0040F27D03DE0002F18BFE3
:10EC10004AF0090479D134E02FB14AF0080415F024
:10EC2000200F14D071E0316805F02002B1F84400E3
:10EC3000104308BF4AF0010467D04AF0180415F0E9
:10EC4000200F62D191F85A1008295AD156E0316844
:10EC500091F85A10082951D153E04AF00800002FCA
:10EC600018BF40F0010450D140F010044DE00028DE
:10EC700018BF15F0040F07D0002F18BF4AF00B047F
:10EC800043D14AF0180440E015F0030F3CD115F0D1
:10EC9000040F39D077B131684AF0080091F85A1062
:10ECA00008290CBF40F0020420F0020415F0200FE8
:10ECB00022D02AE0316805F02002B1F84400104368
:10ECC00008BF4AF0030420D04AF0180015F0200FC6
:10ECD00009D000BF91F85A10082914BF40F002046F
:10ECE00020F0020411E091F85A20082A14BF40F0E5
:10ECF000010020F00100EDE7082902D024F0010412
:10ED000003E044F0010400E0FFDF15F0400F1BD0EA
:10ED1000C7B93168B1F84400002804BF488C10F02E
:10ED2000010F0BD110F0020F08BF10F0200F05D11A
:10ED300015F0010F08BF15F0020F03D091F85A002B
:10ED4000082801D044F040047068A0F800A00178C1
:10ED500021F02001017007210EF022F84146706871
:10ED60000EF015FA214670680EF01DFA14F0010F2E
:10ED70000AD006230022844970680EF0EEF930684C
:10ED8000417B70680EF04EF814F0020F18D0D6E9EF
:10ED90000010B9F1000F4FF006034FF0010207D049
:10EDA0001C310EF0DAF9012170680EF048F807E026
:10EDB00015310EF0D2F93068017D70680EF03FF821
:10EDC00014F0040F18BFFFDF14F0080F17D0CDF8B0
:10EDD00000A03068BDF800100223B0F866000209F8
:10EDE00062F30B01ADF800109DF80110032260F3EF
:10EDF00007118DF80110694670680EF0AEF9012F09
:10EE000061D13068B0F84410E9B390F82200C0F343
:10EE10004000C0BB70680EF0B6F9401CC7B2306845
:10EE2000B0F84420B0F85610551AC7F1FF018D42D2
:10EE3000A8BF0D46AA423AD990F8220010F0010F5F
:10EE400035D144F01004214670680EF0ACF9F81C7E
:10EE5000C0B2ED1E284482B23068B0F86610036E6E
:10EE6000090951FA83F190F85C30484F1944BC46C7
:10EE70000023E1FB07C31B096FF0240C03FB0C11FB
:10EE800080F85C1000E01EE090F85B00012101F0CA
:10EE900025F80090BDF800009DF80210032340EA19
:10EEA00001400190042201A970680EF056F9306803
:10EEB000AAB2016C70680EF0A4F93068B0F8561070
:10EEC0002944A0F8561014F0400F06D0D6E90010DF
:10EED000012306225D310EF040F914F0200F18BF17
:10EEE000FFDF0020002818BFFFDF02B0BDE8F08779
:10EEF0002DE9F843234C2068002808BFFFDF206875
:10EF0000417839BB0178FF2924D0002680F8316090
:10EF1000A0F85660867080F83760304607F0D8FE5B
:10EF200007F062FB206890F95D0007F029FC1848A3
:10EF300007F02CFC174807F0B1FE606807F0CBFE25
:10EF4000206890F8240010F0010F06D0252007F06B
:10EF500025FC09E00C20BDE8F88310F0020F18BF73
:10EF6000262076D007F01AFC206890F85A10252049
:10EF700007F006FB206880F82C6007F0A3FE2068ED
:10EF80000AE00000600000201206002053E4B36E87
:10EF9000844E0200814E020090F85A10002007F0C3
:10EFA000F3FC0F21052007F0BFFB206890F82E101E
:10EFB000002901BF90F82F10002990F8220010F0CE
:10EFC000040F75D005F0D4FC0546206829468068FA
:10EFD00006F0E7F9DFF82C84074690FBF8F008FB11
:10EFE00010704142284605F0C4F92168886097FBFB
:10EFF000F8F04A68104448600CF040FD0146206873
:10F00000426891426FD8C0E90165FF4D4FF0010899
:10F0100095F82D000CF051FD814695F82F00012741
:10F02000002818BFB9F1000F04D095F82D000CF09E
:10F030000BFBA8B195F8300000281CBF95F82E00F6
:10F04000002825D0697B05F10E00012916D01AE0B1
:10F05000FFE710F0040F14BF2720FFDF82D183E702
:10F060003A466F7305F10E01484608F01EFB95F80D
:10F070002D1005F10E000CF017FE09E0407900F0AC
:10F08000C000402815D0414605F10E0008F044FBB1
:10F09000206890F8220010F0040F24D095F82D007D
:10F0A0000CF086FB05001ED010210DF090FB40B146
:10F0B00019E00CF036FE3A4605F10E0108F0F5FABB
:10F0C000E6E720683A4600F11C01C776284608F0BA
:10F0D000ECFA206800F11C0160680DF095FE01213A
:10F0E00060680DF0ACFE2068417B0E3007F000FB3D
:10F0F000206890F8581059B3B0F85410A0F8441094
:10F10000016D016490F82210C1F30011E9B9B0F863
:10F11000660002210509ADF80050684606F00AFDB8
:10F1200028B1BDF80000C0F30B00A84204D1BDF81F
:10F130000000401CADF800002168BDF80000B1F8E7
:10F14000662060F30F12A1F86620206880F85860EE
:10F15000206890F8591031B1B0F84C108187816C5B
:10F16000816380F85960B0F86610026E090951FA9F
:10F1700082F190F85C20DFF894C2114463460022CB
:10F18000E1FB0C3212096FF0240302FB031180F83B
:10F190005C100CF0F6FC032160680CF075FD216832
:10F1A00081F833000020BDE8F883994988607047F2
:10F1B0002DE9F043964C83B0226892F831303BB190
:10F1C000508C1D2808BFFFDF03B0BDE8F0438BE47F
:10F1D00001260027F1B1054692F85C0007F0DEFA3F
:10F1E000206890F85B10FF2007F0CAF920684FF400
:10F1F000A57190F85B20002007F08EFC206890F845
:10F20000221011F0030F00F02D81002D00F0248159
:10F2100000F028B992F822108046D07EC1F3001188
:10F22000002956D0054660680780017821F020014A
:10F230000170518C132937D01FDC102908BF02211F
:10F2400044D0122908BF062140D0FFDF6E4D606810
:10F2500005F10E010DF0CAFD697B60680DF0E2FD5D
:10F260002068418C1D2918BF152965D0B0F84420AD
:10F27000016C60680DF0EFFD5EE0152918BF1D29D7
:10F28000E3D14FF001010DF08BFD6068017841F092
:10F2900020010170216885B11C310DF0B5FD0121FF
:10F2A00060680DF0CCFDD1E700210DF079FD6068BC
:10F2B000017841F020010170C8E715310DF0A4FD7F
:10F2C0002068017D60680DF0BAFDBFE70DF068FDB4
:10F2D000BCE70021FFF754FC6068C17811F03F0FD4
:10F2E0002AD0017911F0100F26D00DF057FD2368B8
:10F2F000024693F82410C1F38000C1F3400C60442F
:10F3000001F0010100EB010C93F82C10C1F3800017
:10F31000C1F34005284401F001010844ACEB0000B2
:10F32000C1B293F85A0000F0D9FD009003230422E3
:10F33000694660680DF011FF2068002590F82410E0
:10F3400090F82C0021EA000212F0010F18BF0125ED
:10F350000ED111F0020F04D010F0020F08BF0225E9
:10F3600006D011F0040F03D010F0040F08BF0425DD
:10F37000B8F1000F2BD0012D1BD0022D08BF262085
:10F380001BD0042D14BFFFDF272016D0206890F873
:10F390005A10252007F0F4F8206890F82210C1F3E5
:10F3A000001169B101224FF49671002007F0B4FBFF
:10F3B0000DE0252007F0F2F9E8E707F0EFF9E5E7BF
:10F3C00090F85A204FF49671002007F0A5FB2068B2
:10F3D00090F82C10294380F82C1090F8242032EA61
:10F3E00001011CD04670418C13292BD026DC10293A
:10F3F00004BF03B0BDE8F083122923D0C1F300108D
:10F40000002807E040420F000406002053E4B36EDA
:10F410006000002018BFFFDF03B0BDE8F083418C1F
:10F420001D2908BF80F82C70DCD0C1F30011002921
:10F4300014BF80F8316080F83170D3E7152918BF08
:10F440001D29DBD190F85A2003B04FF00101BDE82F
:10F45000F043084607F049BD90F85B2001210846BB
:10F4600007F043FD2168002DC87E7CD04A8C3D46C4
:10F47000C2F34000002808BF47F0080512F0400F13
:10F4800018BF45F04005002819BFD1F83890B1F8F1
:10F490003C80D1F84090B1F8448060680721078033
:10F4A0000DF07EFC002160680DF071FE2946606859
:10F4B0000DF079FE15F0080F15D02068BDF800108A
:10F4C0000223B0F86600020962F30B01ADF80010E8
:10F4D0009DF80110032260F307118DF801106946B1
:10F4E00060680DF03AFE60680DF016FD2168C0F10D
:10F4F000FE00B1F85620A8EB02018142A8BF0146E8
:10F50000CFB2D019404542D245F0100160680DF0ED
:10F510004AFE60680DF000FD2168C0F1FE00B1F800
:10F520005610A8EB01018142A8BF0146CFB2606826
:10F530000DF029FE3844421C2068B0F86610036EB6
:10F54000090951FA83F190F85C30FF4D1944AC463B
:10F550000023E1FB05C31B096FF0240C03FB0C1116
:10F5600080F85C1000E038E090F85B00012100F0CA
:10F57000B5FC0090BDF800009DF80210032340EA9E
:10F5800001400190042201A960680DF0E6FD2168A8
:10F5900091F8220010F0400F05D0012306225D31C2
:10F5A00060680DF0DAFD20683A46B0F8560000EBCE
:10F5B000090160680DF025FE2068B0F85610394446
:10F5C000A0F8561007F053FF002818BFFFDF20688F
:10F5D0004670867003B0BDE8F0830121FFF7D0FAD2
:10F5E000F0E7DA4810B50068417841B90078FF28A3
:10F5F00005D000210846FFF7DBFD002010BD07F015
:10F6000018FC07F0F7FB07F0C4FA07F04DFB0C20DD
:10F6100010BD10B5CD4C206890F8220010F0010FFD
:10F620001CBFA06801884FF03C0212BF01204FF6BA
:10F63000FF710020FEF72AFE2168012081F83700C3
:10F6400010BDC249096881F8320070472DE9F041C8
:10F65000002608F081FC002800F0F380BB4C2068F5
:10F66000417800270125012906D0022901D003296C
:10F670007BD0FFDFBDE8F081817802270029418C33
:10F6800037D0C1F34002002A08BF11F0010F6DD03E
:10F6900090F85B204FF001014FF0000007F025FCCF
:10F6A000216891F82200C0F34000002814BF0C200C
:10F6B000222091F85B1006F063FF2068477090F8F5
:10F6C000330020B106F099FD402007F0BEFB206812
:10F6D00090F83400002818BF07F0E4FB00219620C2
:10F6E00007F04CFB07F0BAFE002818BFFFDFBDE8AB
:10F6F000F081C1F3001282B110293ED090F833009E
:10F7000020B106F07AFD402007F09FFB206890F8BA
:10F71000221011F0040F35D042E090F8242090F828
:10F720002C309A4229D1B0F84400002808BF11F0CB
:10F73000010F05D111F0020F08BF11F0200F7DD08D
:10F740004FF001014FF00000FFF732FD2068418CBF
:10F7500011F0010F04BFC1F3400100290AD1B0F834
:10F760005610B0F84420914201E032E026E018BF84
:10F77000BDE8F08180F83150B9E7BDE8F0410021E3
:10F78000012015E590F83510012914BF0329102632
:10F7900046F00E0190F85A204FF0000007F0A5FB4C
:10F7A000206890F83400002818BF07F07BFB002188
:10F7B000962007F0E3FA2068477098E7B0F85610F3
:10F7C000B0F8440081423CD0BDE8F0410121084638
:10F7D000EEE48178D9B1418C11F0010F1CD080F892
:10F7E000685090F86A20B0F86C100120FEF74EFDCA
:10F7F0002068477007F01DFB07F0FCFA07F0C9F915
:10F8000007F052FABDE8F041032008F0D9BB817837
:10F81000BDE8F0410120CBE411F0020F08BFFFDF8B
:10F820003FF465AFB0F85610808F814209D00121B6
:10F830000846FFF7BDFC0320216800E001E04870A6
:10F8400055E7BDE8F041FFF74FB9FFF74DB910B5E7
:10F850003E4C206890F8341049B1363007F02DFB4B
:10F8600018B921687F2081F8360007F011FB206865
:10F8700090F8330018B107F0FBFA06F0D2FC08F05C
:10F880006BFBA8B1206890F82210C1F3001179B188
:10F890004078022818BFFFDF00210120FFF788FC15
:10F8A0002068417800291EBF40780128FFDF10BD85
:10F8B000BDE81040FFF718B92DE9F047234C0F467B
:10F8C00080462168B8F1030F488C08BFC0F340059B
:10F8D00008D000F0010591F83200002818BF4FF061
:10F8E000010901D14FF0000906F04CFF0646B8F1BE
:10F8F000030F0CBF4FF002084FF0010835EA090072
:10F9000008BFBDE8F087206890F8330068B10CF0BC
:10F910001BF938700146FF2807D06068C01C0CF046
:10F92000ECF838780CF01DF9064360680178C1F3F3
:10F93000801221680B7D9A420DD10622C01C153120
:10F9400014F0A4FF002803E053E4B36E600000202D
:10F9500008BF012000D000203978FF2906D0C8B99F
:10F96000206890F82D00884216D113E0A0B161689C
:10F9700011F8030BC0F380100CF083F805460CF06F
:10F98000E3F938B128460BF013FF18B110210CF041
:10F990001EFF08B1012000E00020216891F822102C
:10F9A00011F0040F01D0F0B11AE0CEB9FE4890F882
:10F9B0003500002818BF404515D1616811F8030BC8
:10F9C000C0F380100CF05DF804460CF0BDF938B1BE
:10F9D00020460BF0EDFE18B110210CF0F8FE10B12E
:10F9E0000120BDE8F0870020BDE8F0872DE9F04F49
:10F9F000EE4D074683B0286800264078022818BFDD
:10FA0000FFDF28684FF07F0990F8341049B1363095
:10FA100007F053FA002804BF286880F8369007F0F2
:10FA200037FA68680DF0DEF90446002F00F0048212
:10FA300068680DF062FB002800F0FE8106F070FEA1
:10FA4000002800F0F981FF20DFF864B3DFF8588365
:10FA500000274FF0010A062C80F00082DFE804F056
:10FA6000EFEFEF03EFF78DF8000069460320FFF793
:10FA700023FF002800F0E480296891F8340010B1D9
:10FA800091F89800D0B12868817801294CD0686835
:10FA9000042107800DF084F908F10E0168680DF06B
:10FAA000A5F998F80D1068680DF0BCF92868828FE8
:10FAB000816B68680DF0F3F900F04DB99DF8000016
:10FAC00081F898A00A7881F89920FF280FD001F1D9
:10FAD0009B029A310BF0FAFF002808BFFFDF28686D
:10FAE00090F89A1041F0020180F89A100DE06868D1
:10FAF0000278C2F3801281F89A20D0F80320C1F86E
:10FB00009B20B0F80700A1F89F00286800F1A1042D
:10FB100090F836007F2808BFFFDF286890F836107D
:10FB2000217080F83690AEE790F822009BF80490A0
:10FB3000C0F38014686864F38619072107800DF00C
:10FB40002FF9002168680DF022FB494668680DF026
:10FB50002AFB0623002208F10E0168680DF0FDFA69
:10FB60002868417B68680DF05DF968680DF0D4F98C
:10FB700029688A8FC0F1FE018A42B8BF1146CFB210
:10FB8000BA423DD9F81EC7B249F0100A514668681A
:10FB90000DF009FB68680DF0F6FA3844431C28683C
:10FBA000B0F86610026E090951FA82F190F85C20F3
:10FBB000DFF800920A44C8464FF0000CE2FB098CC3
:10FBC0004FEA1C116FF0240C01FB0C2180F85C1033
:10FBD00090F85B001A46012100F080F90190BDF811
:10FBE00004009DF80610032340EA0140029004221D
:10FBF00002A968680DF0B1FA514668680DF0D3FAB1
:10FC000034B1D5E90010012306225D310DF0A5FACB
:10FC100028683A46816B68680DF0F3FA2868A0F806
:10FC20005670818F8F420CBF0121002180F8311066
:10FC300007F01DFC002818BFFFDF8CE007E00DE196
:10FC400028688078002840F0F98000F0F5B88DF839
:10FC5000000068680178C1F38019D0F803100191A1
:10FC6000B0F80700ADF8080069460520FFF724FE4C
:10FC70000028286873D08178002972D090F85BA0A2
:10FC8000D5E90104D0F80F10C4F80E10B0F8131025
:10FC90006182417D2175817D6175B0F81710E18227
:10FCA000B0F819106180B0F81B10A180B0F81D10D9
:10FCB000E18000F11F0104F1080014F0C8FF68683A
:10FCC00090F8241001F01F01217690F824004009DB
:10FCD00084F8740184F854A084F855A0286890F83A
:10FCE000651084F8561090F85D0084F857009DF870
:10FCF0000010A86800F050F9022008F061F9686867
:10FD0000DBF800400DF1040A078008210DF048F8E7
:10FD1000002168680DF03BFA214668680DF043FA4F
:10FD20000623002208F10E0168680DF016FA286813
:10FD3000417B68680DF076F8494668680DF07FF8F9
:10FD400006230122514668680DF007FA07F08FFB81
:10FD5000002818BFFFDF03202968487070E066E0C4
:10FD6000FFE76868AC684FF001080278617BC2F376
:10FD7000401211406173D0F80F10C4F80E10B0F8A3
:10FD800013106182417D2175817D6175B0F8171076
:10FD9000E182B0F819106180B0F81B10A180B0F8B2
:10FDA0001D10E18008E00000040600206000002033
:10FDB0007C4E020053E4B36E00F11F0104F1080011
:10FDC00014F045FF686890F8241001F01F012176B7
:10FDD00090F82400400984F8740184F8548084F871
:10FDE0005580286890F8651084F8561090F85D00EA
:10FDF00084F857009DF80010A86800F0CDF8286836
:10FE000080F868A090F86A20B0F86C100120FEF726
:10FE10003DFA2868477007F00CF806F0EBFF06F093
:10FE2000B8FE06F041FF012008F0CAF808E090F89B
:10FE30002200C0F3001008B1012601E0FEF754FED5
:10FE4000286890F8330018B107F012F806F0E9F9C5
:10FE500066B100210120FFF7ABF910E0286890F8A7
:10FE60002200C0F300100028E8D0E5E72868817878
:10FE7000012904D190F85B10FF2006F081FB28686F
:10FE80004178002919BF4178012903B0BDE8F08FFE
:10FE90004078032818BFFFDF03B0BDE8F08F70B5CE
:10FEA000794C06460D462068807858B106F030FB44
:10FEB00021680346304691F85B202946BDE8704032
:10FEC00008F03BBE06F024FB21680346304691F85B
:10FED0005A202946BDE8704008F02FBE78B50C4680
:10FEE00000210091082804BF4FF4C87040210DD0B4
:10FEF000042804BF4FF4BF70102107D0022807BFA9
:10FF000001F11800042101F128000821521D02FB13
:10FF100001065D489DF80010006890F85C2062F3CF
:10FF2000050141F040058DF8005090F85B00012874
:10FF300004BF9DF8020020F0E0002AD0022818BF7C
:10FF4000FFDF21D025F080008DF80000C4EB041005
:10FF500000EB80001E2101EB800006FB04044B48EF
:10FF6000844228BFFFDF4A48A0FB0410BDF80110FF
:10FF7000000960F30C01ADF80110BDF800009DF818
:10FF8000021040EA014078BD9DF8020020F0E00038
:10FF900020308DF80200D5E72DE9F0413A4D0446B6
:10FFA0000E46286890F86800002818BFFFDF002779
:10FFB000286880F86A702188A0F86C106188A0F821
:10FFC0008210A188A0F88410E188A0F8861094F827
:10FFD000741180F8881090F82F1049B1427B00F11D
:10FFE0000E01012A04D1497901F0C001402934D021
:10FFF00090F8301041B1427B00F10E01012A04BF9C
:020000040001F9
:10000000497911F0C00F28D000F1760014F016FEE7
:100010006868FF2E0178C1F380116176D0F8031073
:10002000C4F81A10B0F80700E08328681DD0C16733
:10003000E18BA0F8801000F17002511E30460BF0E9
:1000400045FD002808BFFFDF286890F86F1041F0D9
:10005000020180F86F10BDE8F081D0F80E10C0F8F2
:100060007610418AA0F87A10D2E7C767A0F88070AE
:10007000617E80F86F10D4F81A100167E18BA0F848
:100080007410BDE8F081000060000020C4BF0300D0
:10009000898888880178406829B190F8141190F80F
:1000A000730038B901E001F0BFBC19B1042901D0D7
:1000B000012070470020704770B50C4605460621A8
:1000C00002F014FB606008B1002006E0072128461A
:1000D00002F00CFB606018B101202070002070BDA0
:1000E000022070BD2DE9FC470C4606466946FFF725
:1000F000E3FF00287DD19DF8000050B1FEF757F9CD
:10010000B0427CD02146304609F09CFE002873D1D5
:100110002DE00DF0F5FAB04271D02146304612F0D4
:10012000F2FD002868D1019D95F8D80022E0012059
:1001300000E00020804695F837004FF0010A4FF0AC
:100140000009F0B195F8380080071AD584F80190BD
:1001500084F800A084F80490E68095F839102172A4
:10016000698F6181A98FA18185F8379044E0019D55
:1001700095F8140158350028DBD1E87E0028D8D046
:10018000D5E7304602F0F6FB070000D1FFDF384626
:1001900001F006FE40B184F801900F212170E68045
:1001A000208184F804A027E0304602F0D1FB07004C
:1001B00000D1FFDFB8F1000F21D0384601F047FE33
:1001C000B8B19DF8000038B90198D0F80001418815
:1001D000B14201D180F80090304607F090F984F8E0
:1001E00001900C21217084F80490E680297F21720F
:1001F00000E004E085F81B900120BDE8FC870020AA
:10020000FBE71CB56946FFF757FF00B1FFDF684603
:1002100001F016FCFA4900208968A1F8DA001CBD3B
:100220002DE9FC4104460E46062002F007FA054679
:10023000072002F003FA2844C7B20025A8463E442E
:1002400017E02088401C80B22080B04202D3404694
:10025000A4F8008080B2B84204D3B04202D2002099
:10026000BDE8FC816946FFF727FF0028F8D06D1C28
:10027000EDB2AE42E5D84FF6FF7020801220EFE7D6
:1002800038B54FF6FF70ADF800000DE00621BDF85F
:10029000000002F03DFA04460721BDF8000002F01C
:1002A00037FA0CB100B1FFDF00216846FFF7B8FF55
:1002B0000028EBD038BD70B507F08EF90BF0CDF902
:1002C000D04C4FF6FF7600256683A683CEA025701E
:1002D00001680079A4F14002657042F8421FA11C38
:1002E0001071601C12F02FFE25721B2060814FF4EC
:1002F000A471A181E08121820321A1740422E2740E
:10030000A082E082A4F13E00218305704680BC48B3
:100310000C300570A4F110000570468070BD70B5FA
:10032000B74C16460D466060217007F0CFF8FFF716
:10033000A7FFFFF7C0FF207810F0F1FAB4480DF0E6
:1003400053FE2178606812F0A3FD20780AF010FCBB
:10035000284608F09CF9AE48FEF734F8217860682A
:1003600009F056FE3146207813F078F8BDE8704069
:100370000BF073B910B501240AB1002010BD21B1F2
:10038000012903D00024204610BD02210CF076FF85
:10039000F9E72DE9F047040000D1FFDF9948022179
:1003A0001C308146FFF73CFF00B1FFDF954D062072
:1003B000B5F81C8002F042F90646072002F03EF92B
:1003C0003044C6B2701CC7B2A88BB04228D12046B8
:1003D0000DF00CF9B0B1207818283FD12079012810
:1003E0003CD1E088062102F081F9040000D1FFDF52
:1003F000208807F084F82088062102F089F940B3AC
:10040000FFDF2BE0287860B3002666701420207090
:100410002021201D14F007FB022020712E701DE00A
:10042000B84217D12046FDF767FFD0B120781728D2
:1004300014D1207968B1E088072102F057F940B162
:10044000008807F05CF8E088072102F061F900B14C
:10045000FFDF03E02146FFF745FE10B10120BDE8B4
:10046000F08702214846FFF7DBFE10B9A98B414512
:10047000AAD12046BDE8F04713F036B810B501F018
:100480007AFA08B10C2010BD0BF03AF9002010BD2B
:1004900010B50446007818B1012801D0122010BD13
:1004A00001F07AFA20B10BF0DBFA08B10C2010BD94
:1004B000207801F027FAE21D04F11703611CBDE862
:1004C00010400BF0C2B910B5044601F054FA08B15F
:1004D0000C2010BD207828B1012803D0FF280BD0B4
:1004E000122010BD01F00EFA611C0BF0C9F808B122
:1004F000002010BD072010BD01200BF0FBF8F7E72E
:1005000010B50BF0B0FA08B1002010BD302010BDBE
:1005100010B5044601F040FA08B10C2010BD204689
:100520000BF09BFA002010BD10B501F035FA20B198
:100530000BF096FA08B10C2010BD0BF0EBF900207F
:1005400010BDFF2181704FF6FF7181802C494968F1
:100550000A7882718A88028149884181012141702B
:10056000002070471CB5002412F1080F15D00CDCD8
:1005700012F1280F11D012F1140F0ED012F1100F3A
:100580000BD012F10C0F0ED107E012F1040F04D0C2
:100590001AB1032A01D0042A05D1012806D0022865
:1005A00008D003280AD0122420461CBD1046FEF7AE
:1005B0007CFAF9E710460DF0BDFCF5E70846144655
:1005C0006946FFF779FD08B10224EDE79DF80000C8
:1005D000019880F857400024E6E710B51346012241
:1005E0000CF032F9002010BD10B5044610F07CFF6D
:1005F00005280FD0204610F081F9002010BD000022
:100600006C000020E8070020FFFFFFFF1F00000034
:10061000A80600200C20F1E710B5044601F0BCF953
:1006200008B10C20EAE72146002006F0D6FF0020A2
:10063000E4E710B5044610F0EFF950B108F0ABFA5A
:1006400038B1207808F049F820780DF067FF0020D5
:10065000D4E70C20D2E710B5044601F09DF908B1AB
:100660000C20CBE72146012006F0B7FF0020C5E7AC
:1006700038B504464FF6FF70ADF80000A079E17977
:10068000884216D02079FDF7A4FD90B16079FDF77E
:10069000A0FD70B10022A079114613F0F5FA40B91F
:1006A0000022E079114613F0EFFA10B9207A0728FA
:1006B00001D9122038BD08F07BFA60B910F014FFA0
:1006C00048B900216846FFF7ABFD20B1204605F090
:1006D00032FF002038BD0C2038BD2DE9FC41817867
:1006E00005461A2925D00EDC16292DD2DFE801F0A7
:1006F0002C2C2C2C2C212C2C2C2C2C2C2C2C2C2C45
:100700002C2C2C2121212A291ED00BDCA1F11E0129
:100710000C2919D2DFE801F0181818181818181841
:100720001818180D3A3904290ED2DFE801F00D022D
:100730000D022888B0F5706F06D201276946FFF7D1
:10074000BBFC18B102208BE5122089E59DF8000062
:1007500001F0DFF8019C08B1FC3401E004F5BC7441
:100760009DF8000001F0D5F8019E08B1FD3601E0CA
:1007700006F279166846FFF78DFC08B1207808B1BB
:100780000C206DE52770A8783070684601F058F9A4
:10079000002065E57CB50D466946FFF78DFC002617
:1007A00018B12E602E7102207CBD9DF8000001F072
:1007B000B0F8019C9DF80000583401F0AAF80198A7
:1007C00084F8406081682960017B297194F84010A9
:1007D0000029F5D100207CBD70B50D460446018985
:1007E000002380880CF09CF9696A81421DD2401A6E
:1007F000401CA1884008091A8AB2A2802189081ADF
:100800002081668895F8541010460CF063F98642F2
:1008100000D230466080E68895F8551020890CF0AB
:1008200059F9864200D23046E08070BDF0B585B0FF
:100830000D46064603A9FFF73FFC00282DD19DF881
:100840000C0060B300220499FB20B1F84A30FB2B66
:1008500000D30346B1F84C40FB20FB2C00D30446E8
:10086000DFF8A8CA9CE8811000900197CDF808C075
:10087000ADF80230ADF806406846FFF7ADFF6E8078
:10088000BDF80400E880BDF808006881BDF80200EA
:10089000A880BDF806002881002005B0F0BD012227
:1008A000D1E72DE9F04186B0044600886946FFF79C
:1008B00003FC002876D12189E08801F0D0F80028D7
:1008C00070D1A188608801F0CAF800286AD1218916
:1008D000E08801F0D2F8002864D1A188608801F096
:1008E000CCF807005ED1208802A9FFF79FFF00B176
:1008F000FFDFBDF8101062880920914252D3BDF885
:100900000C10E28891424DD3BDF81210BDF80E20B4
:1009100023891144A2881A44914243D39DF80010C0
:10092000019D4FF00008012640F6480041B185F8CE
:10093000A361019991F8E61105F5D17541B91AE065
:1009400085F80D61019991F8301105F5867509B1A9
:100950003A2724E0E18869806188E9802189814221
:1009600000D30146A980A188814200D2084628818F
:10097000012201990FE0E18869806188E98021897D
:10098000814200D30146A980A188814200D2084655
:100990002881019900222846FFF71EFF2E7085F856
:1009A0000180384606B0BDE8F0817AE710B504460C
:1009B00000F0F2FF20B10BF053F808B10C201DE657
:1009C000207800F09FFFE279611C0BF0CAF908B1B2
:1009D000002013E6022011E610B503780446002B30
:1009E000406813460A46014608D001200CF0C9F9B8
:1009F0006168496A884203D90120FFE50020F5E7D4
:100A00000020FBE5887800B90320C97801B90321EB
:100A1000107019700020704710B586B00446008829
:100A200003A9FFF749FB002806D1A08830B10128AF
:100A300004D0022802D0122006B0DFE56B4602AADD
:100A4000214603A8FFF7DEFF0028F5D19DF80C3002
:100A500000220121002B049B06D083F8AD11049BDA
:100A600093F8FA314BBB20E083F81711049B93F8FD
:100A70003C313BB9049B93F816311BB9049B93F8A6
:100A80007D300BB13A200CE0049B83F81611049BD7
:100A90009DF8081083F81811049B9DF8001083F846
:100AA0001911049981F81721C6E7049B93F8AC311A
:100AB0001BB9049B93F87D300BB13A200CE0049BEA
:100AC00083F8AC11049B9DF8081083F8AE11049BC9
:100AD0009DF8001083F8AF11049981F8AD21ABE7C0
:100AE00010B504460020A17801B90120E2780AB9C6
:100AF00040F0020000F0CBFF002803D12046BDE803
:100B0000104089E77AE52DE9F04104460078012894
:100B100004D018B1022801D003281ED1607828B172
:100B2000012803D0022801D0032816D1E07B10B998
:100B3000A078012811D1A07830F005020DD110F075
:100B4000050F0AD0400801D011202CE7E078E68894
:100B500062890F4618B1012801D0122023E7104600
:100B600000F0A5FF302558B13946304600F0A9FF06
:100B700030B1A07B0028F0D00728EED8002012E783
:100B8000284610E71FB5044600F0E8FE10B10C201F
:100B900004B033E5022104F10A0000F09CFFA078C4
:100BA0008DF80800A0788DF8000060788DF80400BA
:100BB00020788DF80300A07B8DF80500E07B00B164
:100BC00001208DF80600A078C0070DD0E07801283C
:100BD00013D0A0B15FF000008DF80100E088ADF8FF
:100BE0000A006089ADF80C0002A80FF021FF002870
:100BF000CED168460DF097FCCAE70220ECE7012051
:100C0000EAE710B504460121FFF77DFF002803D174
:100C10002046BDE81040B5E7F0E40278012A01D093
:100C2000BAB118E042783AB1012A05D0022A12D1AD
:100C300089B1818879B100E059B1418849B1808892
:100C400038B101EB8101490000EB8000B1EB002FCE
:100C500001D2002070471220704770B5044600781A
:100C60000D46012809D010F03FFC052803D00FF0F5
:100C7000F0FD002800D00C2070BD0DF034FB88B1D1
:100C80000DF046FB0DF02CFC0028F5D125B1607865
:100C90000DF0DCFB0028EFD1A1886088BDE8704032
:100CA0000FF0E1BE122070BD10B504460121FFF720
:100CB000B4FF002804D12046BDE810400121CCE754
:100CC0009CE42DE9F0470746B0F84C50FB209246D3
:100CD0000E46FB2D00D30546DFF83486B8F80A002F
:100CE000A84200D2054697F85510284600F025FE88
:100CF000B8F80C10814200D208468146B7F84A4045
:100D0000FB20FB2C00D30446B8F80E00A04200D212
:100D1000044697F85410204600F00FFEB8F8101063
:100D2000814200D208464FF4A4721B2C01D090429D
:100D300003D11B2D25D0914523D0F580A6F808902E
:100D40007480B080524639463046FFF745FD012099
:100D50003070F0881B38E02800D9FFDF70881B381E
:100D6000E02800D9FFDF30894FF4E064A0F5A470DB
:100D7000A04200D9FFDFB088A0F5A470A04200D93E
:100D8000FFDFBDE8F087F0B5871FDDE9056540F6B8
:100D90007B44A74213D28F1FA74210D288420ED89D
:100DA000B2F5FA7F0BD2A3F10A00241FA04206D2AB
:100DB000521C4A43B2EB830F01DAAE4201D9002044
:100DC000F0BD0120F0BD2DE9FC41477A884604467C
:100DD00017F0050F7FD0F8087DD1780701D51120D5
:100DE000B1E494F83A0008B9012F74D100252E46D9
:100DF000F8071BD088F00105208A294600F057FE2D
:100E000048B36089294600F05CFE20B3208A6189DE
:100E1000884260D8A18EE08DCDE90001238D628CDF
:100E2000A18BE08AFFF7AFFFA8B10125B8070ED567
:100E300004EB4500828EC18DCDE90012038D428CFA
:100E4000818BC08AFFF79FFF28B12E466D1CB8F139
:100E5000000F02D023E0302075E4228A012119E03E
:100E6000B14203D004EB4100008A024404EB41008C
:100E7000C38A878ABB422ED1838B478BBB422AD140
:100E8000438C078CBB4226D1038DC08C834222D178
:100E9000491CC9B2A942E3D3608990421BD3207890
:100EA00010B1012817D10EE0A078B8F1000F08D0DA
:100EB00048B1012807D0022805D003280BD102E051
:100EC00009E00028EDD1607838B1012805D002286A
:100ED00003D0032801D0122035E4002033E40021A0
:100EE00071E70178C90702D0406812F0D0BA12F059
:100EF0009DBA2DE9F0438DB00D46AFF6F402D2E96C
:100F0000008701462846FFF75EFF00280CD100F05D
:100F100025FD40B9FE4E307828B90CF0F1FBA0F564
:100F20007F41FF3903D00C200DB0BDE8F0830321D1
:100F300005F1100000F0CFFDF54808AA3E380890F2
:100F4000F4480990F248062110380A900BA801F0E5
:100F50009BFB040035D003210BF013FAB18AA4F8EF
:100F60004A10F28AA4F84C20F37C0093B146B37C7B
:100F7000208801F076FC00B1FFDF208806F0BEFA81
:100F8000218804F10E0000F011FDE3A004F1120627
:100F900000680490032104A804F0C2FD002004A905
:100FA0000A5C3254401CC0B20328F9D3A88B60807D
:100FB000688CA080288DE080687AC10703D0012169
:100FC00006E00920B0E7800701D5022100E00021FA
:100FD000B9F818000A460FF0DBFD0146A062204672
:100FE0000FF0E4FD002684F85E6084F85F60A87866
:100FF00000F088FC6076D5F80300C4F81A00B5F854
:101000000700E083C4F808802773012084F80801F2
:10101000024604F586712046FFF753FE8DF8006006
:101020000121684604F07CFD9DF8000000F00701F6
:10103000C0F3C1021144C0F3401008448DF8000011
:10104000401D2076092801D2083020760021204654
:101050000BF097F968780DF051F9A9782878EA1C17
:101060000DF01FF948B10DF053F9A9782878EA1C62
:101070000DF0C6F9060002D038E0122636E0687A94
:1010800000F001010020CA0700D00120890701D526
:1010900040F002000DF0EEF8060027D121460320B3
:1010A0000DF0D8F9060021D1687A00F001018DF821
:1010B0000810C00705D06889ADF80A00288AADF885
:1010C0000C0002A80FF0B4FC064695F83A0000B1F7
:1010D00001200DF0E1F84EB90DF002FA060005D13D
:1010E000A98F20460FF046FC060008D0208806F0A5
:1010F00006FA2088062101F00BFB00B1FFDF304625
:1011000012E701460020F4E638B58148007878B946
:1011100010F0EAF9052805D00CF0F2FAA0F57F41AD
:10112000FF3905D068460FF0E2FC040002D00CE065
:101130000C2038BD0098008806F0E1F900980621DF
:10114000008801F0E5FA00B1FFDF204638BD1CB58C
:1011500082894189CDE900120389C288818840884B
:10116000FFF711FE08B100201CBD30201CBD70B57A
:101170000546FFF7ECFF00280ED12888062101F074
:10118000B5FA040007D000F04FFC20B1D4F80001FC
:10119000017831B901E0022070BDD4F84C11097812
:1011A00009B13A2070BD05218171D4F800110020E9
:1011B0000881D4F80011A8884881D4F80011E88883
:1011C0008881D4F800112889C881D4F800010289E7
:1011D00041898A4204D88279082A01D88A4201D3F7
:1011E000122070BD29884180D4F8001102200870B7
:1011F000002070BD3EB504460BF0B8FAB0B14448CB
:101200000125A0F140024570236842F8423F23794E
:101210000021137141706946062001F0F0F900B118
:10122000FFDF684601F0C9F910B10EE012203EBDA3
:10123000BDF80440029880F80851684601F0BDF9F5
:1012400018B9BDF80400A042F4D100203EBD70B52D
:1012500005460088062101F049FA040007D000F095
:10126000E3FB20B1D4F80011087830B901E0022086
:1012700070BDD4F84C01007808B13A2070BD9620BA
:10128000005D10F0010F1BD0D5F802004860D5F8C2
:1012900006008860D4F80001698910228181D4F8A1
:1012A000000105F10C010E3004F5807413F01AFBF7
:1012B000216803200870216828884880002070BDBC
:1012C0000C2070BD38B504460078EF2856D86088E9
:1012D000ADF80000009800F00FFCD0B3618808075B
:1012E00008D4D4E90120824248D8202A46D3B0F558
:1012F000804F43D8207B60B307283FD8607B70B114
:1013000001280CD002280AD0032807E0A04E0200D2
:10131000E807002078000020112233002ED14A0770
:1013200003D4022801D0032805D1A07B08B10128ED
:1013300024D1480707D4607D28B1012803D00228B2
:1013400001D003281AD1C806E07D03D5012815D1A4
:1013500010E013E0012801D003280FD1C80609D4FA
:10136000607E012803D0022801D0032806D1A07E88
:101370000F2803D8E07E18B1012801D0122038BD13
:10138000002038BDF8B515460E46044607F010FC9F
:1013900008B10C20F8BD2046FFF794FF0028F9D1D2
:1013A000E07D03280BD0A078C00602D4607E03281D
:1013B00005D0FDF77FFB3070A07515B10CE0112052
:1013C000F8BDFF208DF8000069460020FDF761FBA5
:1013D00069460020FDF751FB2046BDE8F840FDF7C7
:1013E000ADBA0022CEE770B50C46054612B11F29F2
:1013F00007D80CE0FF2C04D8FDF727F818B11F2CF4
:1014000001D9122070BD2846FDF709F808B1002067
:1014100070BD422070BD10B50446408810B1FDF784
:101420000FFB78B12078618800F001026078FFF747
:10143000DAFF002805D1FDF7EBFA6288824203D972
:1014400007203DE412203BE410466168FDF721FBD4
:10145000002035E410B50446408810B1FCF7E7FFE2
:1014600070B12078618800F001026078FFF7BBFF5F
:10147000002804D160886168FDF7FFFA00201FE4AE
:1014800012201DE47CB5054640784224012808D886
:10149000A878FCF7C4FF20B128781224012802D0D4
:1014A00090B120467CBDFDF711FB20B1A888002833
:1014B000F7D08028F5D8FDF710FB60B168780028D8
:1014C000EFD02878012808D006F038F9044607F054
:1014D0003BF8002872D00C207CBDFDF748F910B90C
:1014E000FDF7EDFA90B307F063FB0028F3D1FCF7AA
:1014F0005EFFA0F57F41FF39EDD1FDF75AF9AE88C7
:1015000042F210704643A879FDF7ABFAFCF796FF5C
:10151000F8B10022072101A801F0B6F804001FD09D
:10152000F6480321846020460AF0E4FD2046FDF7DA
:101530003CFEF34DA88AA4F84A00E88AA4F84C00BF
:10154000FCF783FF70B1288B01210FE0FFE7122029
:101550007CBD3146002007F0C3F868B3FFDF37E0F9
:1015600009207CBDFDF7BBFA0146288B07F06DF919
:101570000146A0620022204606F0E3F8FCF765FF72
:1015800008B9FDF7ACFAE87C0090AB7CEA8AA98A3E
:10159000208801F066F900B1FFDF208805F0AEFF7A
:1015A0003146204607F09CF800B1FFDF002204F529
:1015B000D1712046FFF785FB0AE0FFE744B12088A0
:1015C00005F09DFF2088072101F0A2F800B1FFDFA0
:1015D00000207CBD002155E770B50D46072101F0C4
:1015E00085F8040003D094F87B0110B10AE00220D2
:1015F00070BD94F86500142801D0152802D194F824
:10160000C80108B10C2070BD1022294604F5BE7037
:1016100013F068F9012084F87B01002070BD10B53B
:10162000072101F063F818B190F87B1111B107E0C0
:10163000022006E790F86510142903D0152901D07F
:101640000C20FEE6022180F87B110020F9E62DE94E
:10165000FC410C464BF68032122194421CD8DCB17E
:101660006946FEF729FD002815D19DF8000000F01D
:1016700050F9019E9DF80000583600F04AF9019D8E
:10168000AD1C2F882246394630460AF0EEFC2888E9
:10169000B842F6D100201FE408461DE47CB504469C
:1016A00000886946FEF708FD002810D19DF800006B
:1016B00000F02FF9019D9DF80000583500F029F940
:1016C0000198A27890F82C10914201D10C207CBD99
:1016D0007F212972A9720021E972E17880F82D102A
:1016E000217980F82E10A17880F82C1000207CBD84
:1016F0001CB50C466946FEF7DFFC00280AD19DF8B0
:10170000000000F006F9019890F8730000B1012084
:10171000207000201CBD7CB50D4614466946FEF7BE
:10172000CBFC002809D19DF8000000F0F2F80198E8
:1017300090F82C00012801D00C207CBD9DF8000001
:1017400000F0E7F8019890F86010297090F86100B7
:10175000207000207CBD70B50D461646072100F0B4
:10176000C5FF18B381880124C388428804EB410473
:10177000AC4217D842F210746343A4106243B3FB27
:10178000F2F2521E94B24FF4FA72944200D9144607
:10179000A54200D22C46491C641CB4FBF1F24A431A
:1017A000521E91B290F8B4211AB901E0022070BD26
:1017B00001843180002070BD10B50C46072100F077
:1017C00095FF48B180F8E74024B190F8E51009B1E1
:1017D00007F051F8002034E6022032E6017899B192
:1017E000417889B141881B290ED381881B290BD3ED
:1017F000C188022908D342490268403941F8522F72
:1018000040684860002070471220704710B50446B9
:101810000FF0BAF9204606F0E7FF002011E610B5F8
:1018200006F0E5FF00200CE62DE9F04115460F46D5
:1018300006460122114638460FF0AAF90446012156
:10184000384607F002F8844200D2044601213046AF
:10185000653C00F063F806460121002000F05EF8C8
:10186000304401219630844206D900F19601201AB5
:10187000B0FBF1F0401C81B229800020BDE8F0816E
:1018800010B5044600F088F808B10C20D9E5601CBA
:101890000AF042FA207800F00100FCF785FF20787A
:1018A00000F001000CF02FFD0020CAE510B506F095
:1018B00098FF0020C5E510B50446072000F0B0FEF3
:1018C00008B10C20BDE52078C00711D00022607857
:1018D000114612F0D9F908B11220B2E5A06808F05B
:1018E000F6FE6078D4F8041008F0FAFE0020A8E5AF
:1018F000002008F0ECFE00210846F5E76C0000200F
:10190000E807002018B1022801D00120704700200C
:10191000704708B1002070470120704710B50129B9
:1019200004D0022905D0FFDF20468AE5C0005030F0
:1019300001E080002C3084B2F6E711F00C0F04D0E7
:101940004FF4747101EB801006E0022902D0C00050
:10195000703001E080003C3080B2704710B50FF06D
:10196000C3FD042805D00FF0BFFD052801D00020DD
:1019700067E5012065E510B5FFF7F0FF10B10CF049
:1019800073FD28B907F014F920B1FCF7E8FE08B19F
:10199000012056E5002054E510B5FFF7DFFF18B928
:1019A00007F006F9002800D001204AE52DE9FE43A2
:1019B00000250F4680460A260421404604F0D9F847
:1019C00040460AF0AFFE062000F038FE044616E05E
:1019D0006946062000F013FE0BE000BFBDF80400CE
:1019E000B84206D00298042241460E3012F04EFF53
:1019F00050B1684600F0E1FD0500EFD0641E002CF8
:101A000006DD002DE4D005E040460AF094FEF5E73F
:101A100005B9FFDFD8F800000AF031FB761E01D0CF
:101A20000028C9D0BDE8FE8390F8D81090F8730064
:101A300020B919B1042901D0012070470020704756
:101A4000017800290AD0416891F8E520002A05D0E4
:101A5000002281F8E520406806F00DBF70471B3872
:101A6000E12806D2B1F5A47F03D344F2902081424D
:101A700001D91220704700207047FB2803D840F698
:101A80004800814201D9112070470020704770B58D
:101A900014460546012200F053F8002806D12146DD
:101AA0002846BDE87040002200F04AB870BD042806
:101AB00003D321B9B0F5804F01D900207047012030
:101AC0007047042803D321B9B0F5804F01D9002015
:101AD00070470120704710B500224FF4C84408E059
:101AE00030F81230A34200D9234620F81230521C9D
:101AF000D2B28A42F4D3A4E480B2C1060BD4010767
:101B00001CD481064FEAC07101D5B9B900E099B182
:101B1000800713D410E0410610D481060ED4C1070B
:101B20004FEA807104D0002902DB400704D405E0AD
:101B3000010703D4400701D40120704700207047FB
:101B40000AB1012200E00222024202D1880802D139
:101B500009B10020704711207047000030B505889A
:101B600025F4004421448CB24FF4004194420AD23F
:101B7000121B92B21B339A4201D2A94307E005F42B
:101B80000041214303E0A21A92B2A943114301800C
:101B900030BD0844083050434A31084480B2704791
:101BA00070B51D4616460B46044629463046049A33
:101BB000FFF7EFFF0646B34200D2FFDF28212046A1
:101BC00012F031FF4FF6FF70A082283EB0B2657769
:101BD0006080B0F5004F00D9FFDF618805F13C005F
:101BE000814200D2FFDF60880835401B343880B264
:101BF00020801B2800D21B2020800020A07770BDF1
:101C00008161886170472DE9F05F0D46C188044607
:101C100000F12809008921F4004620F4004800F072
:101C200062FB10B10020BDE8F09F4FF0000A4FF0BA
:101C3000010BB0450CD9617FA8EB0600401A0838AB
:101C4000854219DC09EB06000021058041801AE07D
:101C50006088617F801B471A083F0DD41B2F00DA74
:101C6000FFDFBD4201DC294600E0B9B2681A020478
:101C7000120C04D0424502DD84F817A0D2E709EB2C
:101C800006000180428084F817B0CCE770B50446A6
:101C900000F12802C088E37D20F400402BB11044FD
:101CA0000288438813448B4201D2002070BD002576
:101CB0008A4202D30180458008E0891A0904090C90
:101CC000418003D0A01D00F01EFB08E0637F008868
:101CD0000833184481B26288A01DFFF73FFFE57505
:101CE000012070BD70B5034600F12804C5888088C6
:101CF00020F400462644A84202D10020188270BD7C
:101D000098893588A84206D3401B75882D1A20442F
:101D1000ADB2C01E05E02C1AA5B25C7F2044304451
:101D2000401D0C88AC4200D90D809C8924B1002450
:101D300014700988198270BD0124F9E770B5044652
:101D400000F12801808820F400404518208A0028EE
:101D500025D0A189084480B2A08129886A881144CD
:101D6000814200D2FFDF2888698800260844A189C3
:101D7000884212D1A069807F2871698819B1201D1D
:101D800000F0C1FA08E0637F28880833184481B264
:101D90006288201DFFF7E2FEA6812682012070BD29
:101DA0002DE9F041418987880026044600F1280585
:101DB000B94218D004F10A0821F4004028444188AF
:101DC00019B1404600F09FFA08E0637F00880833AD
:101DD000184481B262884046FFF7C0FE761C6189D4
:101DE000B6B2B942E8D13046BDE8F0812DE9F04104
:101DF00004460B4627892830A68827F40041B4F80A
:101E00000A8001440D46B74201D10020ECE70AB137
:101E1000481D106023B1627F691D184612F062FDF3
:101E20002E88698804F1080021B18A1996B200F061
:101E30006AFA06E0637F62880833991989B2FFF76E
:101E40008DFE474501D1208960813046CCE78188ED
:101E5000C088814201D1012070470020704701896C
:101E60008088814201D1012070470020704770B501
:101E70008588C38800F1280425F4004223F400413A
:101E800014449D421AD08389058A5E192588638887
:101E9000EC18A64214D313B18B4211D30EE0437F4A
:101EA00008325C192244408892B2801A80B22333EF
:101EB000984201D211B103E08A4201D1002070BDE5
:101EC000012070BD2DE9F0478846C188044600898D
:101ED00021F4004604F1280720F4004507EB060929
:101EE00000F001FA002178BBB54204D9627FA81B3B
:101EF000801A002503E06088627F801B801A083802
:101F000023D4E28962B1B9F80020B9F802303BB1BC
:101F1000E81A2177404518DBE0893844801A09E047
:101F2000801A217740450ADB607FE1890830304420
:101F300039440844C01EA4F81280BDE8F087454526
:101F400003DB01202077E7E7FFE761820020F4E769
:101F50002DE9F74F044600F12805C088884620F493
:101F6000004A608A05EB0A0608B1404502D200200B
:101F7000BDE8FE8FE08978B13788B6F8029007EBAC
:101F80000901884200D0FFDF207F4FF0000B50EAAC
:101F9000090106D088B33BE00027A07FB946307125
:101FA000F2E7E18959B1607F294408305044084480
:101FB000B4F81F1020F8031D94F821108170E289F5
:101FC00007EB080002EB0801E1813080A6F802B0BF
:101FD00002985F4650B1637F30880833184481B25D
:101FE0006288A01DFFF7BAFDE78121E0607FE189EB
:101FF00008305044294408442DE0FFE7E089B4F854
:102000001F102844C01B20F8031D94F82110817074
:1020100009EB0800E28981B202EB0800E081378019
:1020200071800298A0B1A01D00F06DF9A4F80EB067
:10203000A07F401CA077A07D08B1E088A08284F832
:1020400016B000BFA4F812B084F817B001208FE7D3
:10205000E0892844C01B30F8031DA4F81F108078C5
:1020600084F82100EEE710B5818800F1280321F4FF
:1020700000442344848AC288A14212D0914210D0E5
:10208000818971B9826972B11046FFF7E8FE50B9D3
:102090001089283220F400401044197900798842D0
:1020A00001D1002010BD184610BD00F12803407F6B
:1020B00008300844C01E1060088808B9DB1E136091
:1020C00008884988084480B270472DE9F04100F142
:1020D0002806407F1C4608309046431808884D88E3
:1020E000069ADB1EA0B1C01C80B2904214D9801A9F
:1020F000A04200DB204687B298183A46414612F0CB
